 jdwp

 Timestamp is b6253b36 (reproducible build file hash)

 Preferred load address is 0000000180000000

 Start         Length     Name                   Class
 0001:00000000 0002b130H .text$mn                CODE
 0001:0002b130 00000036H .text$mn$00             CODE
 0001:0002b166 00000092H .text$x                 CODE
 0002:00000000 000002b0H .idata$5                DATA
 0002:000002b0 00000038H .00cfg                  DATA
 0002:000002e8 00000008H .CRT$XCA                DATA
 0002:000002f0 00000008H .CRT$XCZ                DATA
 0002:000002f8 00000008H .CRT$XIA                DATA
 0002:00000300 00000008H .CRT$XIZ                DATA
 0002:00000308 00000008H .CRT$XPA                DATA
 0002:00000310 00000008H .CRT$XPZ                DATA
 0002:00000318 00000008H .CRT$XTA                DATA
 0002:00000320 00000010H .CRT$XTZ                DATA
 0002:00000328 00000000H .gehcont$y              DATA
 0002:00000328 00000000H .gfids$y                DATA
 0002:00000330 00007b50H .rdata                  DATA
 0002:00007e80 00000000H .rdata$CastGuardVftablesA DATA
 0002:00007e80 00000000H .rdata$CastGuardVftablesC DATA
 0002:00007e80 00000118H .rdata$voltmd           DATA
 0002:00007f98 000002b8H .rdata$zzzdbg           DATA
 0002:00008250 00000008H .rtc$IAA                DATA
 0002:00008258 00000008H .rtc$IZZ                DATA
 0002:00008260 00000008H .rtc$TAA                DATA
 0002:00008268 00000008H .rtc$TZZ                DATA
 0002:00008270 00000f70H .xdata                  DATA
 0002:000091e0 00000064H .edata                  DATA
 0002:00009244 000000dcH .idata$2                DATA
 0002:00009320 00000018H .idata$3                DATA
 0002:00009338 000002b0H .idata$4                DATA
 0002:000095e8 0000061aH .idata$6                DATA
 0003:00000000 00000840H .data                   DATA
 0003:00000840 00000f28H .bss                    DATA
 0004:00000000 00001bf0H .pdata                  DATA
 0005:00000000 00000060H .rsrc$01                DATA
 0005:00000060 00000390H .rsrc$02                DATA

  Address         Publics by Value              Rva+Base               Lib:Object

 0000:00000000       __AbsoluteZero             0000000000000000     <absolute>
 0000:00000000       ___safe_se_handler_count   0000000000000000     <absolute>
 0000:00000000       ___safe_se_handler_table   0000000000000000     <absolute>
 0000:00000000       __arm64x_extra_rfe_table   0000000000000000     <absolute>
 0000:00000000       __arm64x_extra_rfe_table_size 0000000000000000     <absolute>
 0000:00000000       __arm64x_native_entrypoint 0000000000000000     <absolute>
 0000:00000000       __arm64x_redirection_metadata 0000000000000000     <absolute>
 0000:00000000       __arm64x_redirection_metadata_count 0000000000000000     <absolute>
 0000:00000000       __dynamic_value_reloc_table 0000000000000000     <absolute>
 0000:00000000       __enclave_config           0000000000000000     <absolute>
 0000:00000000       __guard_check_icall_a64n_fptr 0000000000000000     <absolute>
 0000:00000000       __guard_eh_cont_count      0000000000000000     <absolute>
 0000:00000000       __guard_eh_cont_table      0000000000000000     <absolute>
 0000:00000000       __guard_fids_count         0000000000000000     <absolute>
 0000:00000000       __guard_fids_table         0000000000000000     <absolute>
 0000:00000000       __guard_iat_count          0000000000000000     <absolute>
 0000:00000000       __guard_iat_table          0000000000000000     <absolute>
 0000:00000000       __guard_longjmp_count      0000000000000000     <absolute>
 0000:00000000       __guard_longjmp_table      0000000000000000     <absolute>
 0000:00000000       __hybrid_auxiliary_iat     0000000000000000     <absolute>
 0000:00000000       __hybrid_auxiliary_iat_copy 0000000000000000     <absolute>
 0000:00000000       __hybrid_code_map          0000000000000000     <absolute>
 0000:00000000       __hybrid_code_map_count    0000000000000000     <absolute>
 0000:00000000       __x64_code_ranges_to_entry_points 0000000000000000     <absolute>
 0000:00000000       __x64_code_ranges_to_entry_points_count 0000000000000000     <absolute>
 0000:00000100       __guard_flags              0000000000000100     <absolute>
 0000:00000000       __ImageBase                0000000180000000     <linker-defined>
 0001:000033d0       createFrameID              00000001800043d0 f   FrameID.obj
 0001:000033ec       getFrameNumber             00000001800043ec f   FrameID.obj
 0001:000033f0       validateFrameID            00000001800043f0 f   FrameID.obj
 0001:00005af8       __local_stdio_printf_options 0000000180006af8 f i SDE.obj
 0001:00005b00       convertLineNumberTable     0000000180006b00 f   SDE.obj
 0001:000061c8       searchAllSourceNames       00000001800071c8 f   SDE.obj
 0001:000062f8       setGlobalStratumId         00000001800072f8 f   SDE.obj
 0001:00006300       snprintf                   0000000180007300 f i SDE.obj
 0001:00009c84       __acrt_initialize          000000018000ac84 f   MSVCRT:ucrt_stubs.obj
 0001:00009c84       __acrt_thread_attach       000000018000ac84 f   MSVCRT:ucrt_stubs.obj
 0001:00009c84       __acrt_thread_detach       000000018000ac84 f   MSVCRT:ucrt_stubs.obj
 0001:00009c84       __acrt_uninitialize        000000018000ac84 f   MSVCRT:ucrt_stubs.obj
 0001:00009c84       __acrt_uninitialize_critical 000000018000ac84 f   MSVCRT:ucrt_stubs.obj
 0001:00009c84       __scrt_stub_for_acrt_initialize 000000018000ac84 f   MSVCRT:ucrt_stubs.obj
 0001:00009c84       __scrt_stub_for_acrt_thread_attach 000000018000ac84 f   MSVCRT:ucrt_stubs.obj
 0001:00009c84       __scrt_stub_for_acrt_thread_detach 000000018000ac84 f   MSVCRT:ucrt_stubs.obj
 0001:00009c84       __scrt_stub_for_acrt_uninitialize 000000018000ac84 f   MSVCRT:ucrt_stubs.obj
 0001:00009c84       __scrt_stub_for_acrt_uninitialize_critical 000000018000ac84 f   MSVCRT:ucrt_stubs.obj
 0001:00009c84       __vcrt_initialize          000000018000ac84 f   MSVCRT:ucrt_stubs.obj
 0001:00009c84       __vcrt_thread_attach       000000018000ac84 f   MSVCRT:ucrt_stubs.obj
 0001:00009c84       __vcrt_thread_detach       000000018000ac84 f   MSVCRT:ucrt_stubs.obj
 0001:00009c84       __vcrt_uninitialize        000000018000ac84 f   MSVCRT:ucrt_stubs.obj
 0001:00009c84       __vcrt_uninitialize_critical 000000018000ac84 f   MSVCRT:ucrt_stubs.obj
 0001:0000a6dc       bagAdd                     000000018000b6dc f   bag.obj
 0001:0000a784       bagCreateBag               000000018000b784 f   bag.obj
 0001:0000a7ec       bagDeleteAll               000000018000b7ec f   bag.obj
 0001:0000a7f4       bagDestroyBag              000000018000b7f4 f   bag.obj
 0001:0000a818       bagDup                     000000018000b818 f   bag.obj
 0001:0000a860       bagEnumerateOver           000000018000b860 f   bag.obj
 0001:0000a8cc       bagSize                    000000018000b8cc f   bag.obj
 0001:0000ab6c       cbTrackingClassPrepare     000000018000bb6c f   classTrack.obj
 0001:0000abc4       cbTrackingObjectFree       000000018000bbc4 f   classTrack.obj
 0001:0000ac18       classTrack_initialize      000000018000bc18 f   classTrack.obj
 0001:0000b020       commonRef_compact          000000018000c020 f   commonRef.obj
 0001:0000b124       commonRef_idToRef          000000018000c124 f   commonRef.obj
 0001:0000b290       commonRef_idToRef_delete   000000018000c290 f   commonRef.obj
 0001:0000b2b0       commonRef_initialize       000000018000c2b0 f   commonRef.obj
 0001:0000b2fc       commonRef_lock             000000018000c2fc f   commonRef.obj
 0001:0000b310       commonRef_pin              000000018000c310 f   commonRef.obj
 0001:0000b3cc       commonRef_pinAll           000000018000c3cc f   commonRef.obj
 0001:0000b4d4       commonRef_refToID          000000018000c4d4 f   commonRef.obj
 0001:0000b5b4       commonRef_release          000000018000c5b4 f   commonRef.obj
 0001:0000b608       commonRef_releaseMultiple  000000018000c608 f   commonRef.obj
 0001:0000b664       commonRef_reset            000000018000c664 f   commonRef.obj
 0001:0000b74c       commonRef_unlock           000000018000c74c f   commonRef.obj
 0001:0000b760       commonRef_unpin            000000018000c760 f   commonRef.obj
 0001:0000b7f4       commonRef_unpinAll         000000018000c7f4 f   commonRef.obj
 0001:0000c2a4       debugDispatch_getHandler   000000018000d2a4 f   debugDispatch.obj
 0001:0000c308       debugDispatch_initialize   000000018000d308 f   debugDispatch.obj
 0001:0000c484       _guard_check_icall_nop     000000018000d484 f   MSVCRT:guard_support.obj
 0001:0000c484       debugDispatch_reset        000000018000d484 f   debugDispatch.obj
 0001:0000c484       invoker_reset              000000018000d484 f   invoker.obj
 0001:0000c484       standardHandlers_onDisconnect 000000018000d484 f   standardHandlers.obj
 0001:0000c484       stepControl_reset          000000018000d484 f   stepControl.obj
 0001:0000c484       threadControl_onConnect    000000018000d484 f   threadControl.obj
 0001:0000c484       threadControl_onDisconnect 000000018000d484 f   threadControl.obj
 0001:0000c484       util_reset                 000000018000d484 f   util.obj
 0001:0000c488       Agent_OnLoad               000000018000d488 f   debugInit.obj
 0001:0000cabc       Agent_OnUnload             000000018000dabc f   debugInit.obj
 0001:0000d25c       debugInit_exit             000000018000e25c f   debugInit.obj
 0001:0000d378       debugInit_isInitComplete   000000018000e378 f   debugInit.obj
 0001:0000d380       debugInit_launchOnInit     000000018000e380 f   debugInit.obj
 0001:0000d388       debugInit_reset            000000018000e388 f   debugInit.obj
 0001:0000d48c       debugInit_suspendOnInit    000000018000e48c f   debugInit.obj
 0001:0000d494       debugInit_waitInitComplete 000000018000e494 f   debugInit.obj
 0001:0000d58c       forceExit                  000000018000e58c f   debugInit.obj
 0001:0000ebd8       debugLoop_initialize       000000018000fbd8 f   debugLoop.obj
 0001:0000ebf4       debugLoop_run              000000018000fbf4 f   debugLoop.obj
 0001:0000eeec       debugLoop_sync             000000018000feec f   debugLoop.obj
 0001:0000f1a0       do_pause                   00000001800101a0 f   error_messages.obj
 0001:0000f210       error_message              0000000180010210 f   error_messages.obj
 0001:0000f2d4       eventText                  00000001800102d4 f   error_messages.obj
 0001:0000f3c8       fprintf                    00000001800103c8 f i error_messages.obj
 0001:0000f40c       jdiAssertionFailed         000000018001040c f   error_messages.obj
 0001:0000f528       jdwpErrorText              0000000180010528 f   error_messages.obj
 0001:0000f860       jvmtiErrorText             0000000180010860 f   error_messages.obj
 0001:0000fc84       print_message              0000000180010c84 f   error_messages.obj
 0001:0000fca4       tty_message                0000000180010ca4 f   error_messages.obj
 0001:0000ffe8       eventFilterRestricted_alloc 0000000180010fe8 f   eventFilter.obj
 0001:0001004c       eventFilterRestricted_deinstall 000000018001104c f   eventFilter.obj
 0001:000101e4       eventFilterRestricted_install 00000001800111e4 f   eventFilter.obj
 0001:000102c0       eventFilterRestricted_isBreakpointInClass 00000001800112c0 f   eventFilter.obj
 0001:000102f0       eventFilterRestricted_passesFilter 00000001800112f0 f   eventFilter.obj
 0001:000107e0       eventFilterRestricted_passesUnloadFilter 00000001800117e0 f   eventFilter.obj
 0001:00010934       eventFilter_dumpHandlerFilters 0000000180011934 f   eventFilter.obj
 0001:00010b9c       eventFilter_predictFiltering 0000000180011b9c f   eventFilter.obj
 0001:00010cb8       eventFilter_setClassExcludeFilter 0000000180011cb8 f   eventFilter.obj
 0001:00010cec       eventFilter_setClassMatchFilter 0000000180011cec f   eventFilter.obj
 0001:00010d20       eventFilter_setClassOnlyFilter 0000000180011d20 f   eventFilter.obj
 0001:00010d90       eventFilter_setConditionalFilter 0000000180011d90 f   eventFilter.obj
 0001:00010dc0       eventFilter_setCountFilter 0000000180011dc0 f   eventFilter.obj
 0001:00010df8       eventFilter_setExceptionOnlyFilter 0000000180011df8 f   eventFilter.obj
 0001:00010e88       eventFilter_setFieldOnlyFilter 0000000180011e88 f   eventFilter.obj
 0001:00010f0c       eventFilter_setInstanceOnlyFilter 0000000180011f0c f   eventFilter.obj
 0001:00010f7c       eventFilter_setLocationOnlyFilter 0000000180011f7c f   eventFilter.obj
 0001:00011010       eventFilter_setPlatformThreadsOnlyFilter 0000000180012010 f   eventFilter.obj
 0001:00011038       eventFilter_setSourceNameMatchFilter 0000000180012038 f   eventFilter.obj
 0001:00011068       eventFilter_setStepFilter  0000000180012068 f   eventFilter.obj
 0001:00011130       eventFilter_setThreadOnlyFilter 0000000180012130 f   eventFilter.obj
 0001:000113a4       isBreakpointSet            00000001800123a4 f   eventFilter.obj
 0001:000117b4       callback_lock              00000001800127b4 f   eventHandler.obj
 0001:000117c0       callback_unlock            00000001800127c0 f   eventHandler.obj
 0001:00014608       eventHandlerRestricted_iterator 0000000180015608 f   eventHandler.obj
 0001:000146e8       eventHandler_alloc         00000001800156e8 f   eventHandler.obj
 0001:00014718       eventHandler_allocHandlerID 0000000180015718 f   eventHandler.obj
 0001:0001474c       eventHandler_createInternalThreadOnly 000000018001574c f   eventHandler.obj
 0001:00014770       eventHandler_createPermanentInternal 0000000180015770 f   eventHandler.obj
 0001:00014798       eventHandler_dumpAllHandlers 0000000180015798 f   eventHandler.obj
 0001:000147c8       eventHandler_dumpHandlers  00000001800157c8 f   eventHandler.obj
 0001:00014850       eventHandler_free          0000000180015850 f   eventHandler.obj
 0001:00014884       eventHandler_freeAll       0000000180015884 f   eventHandler.obj
 0001:000148e4       eventHandler_freeByID      00000001800158e4 f   eventHandler.obj
 0001:00014940       eventHandler_freeClassBreakpoints 0000000180015940 f   eventHandler.obj
 0001:000149c4       eventHandler_initialize    00000001800159c4 f   eventHandler.obj
 0001:00015178       eventHandler_installExternal 0000000180016178 f   eventHandler.obj
 0001:0001519c       eventHandler_lock          000000018001619c f   eventHandler.obj
 0001:000151a8       eventHandler_onConnect     00000001800161a8 f   eventHandler.obj
 0001:000152f4       eventHandler_reset         00000001800162f4 f   eventHandler.obj
 0001:000154bc       eventHandler_synthesizeUnloadEvent 00000001800164bc f   eventHandler.obj
 0001:00015648       eventHandler_unlock        0000000180016648 f   eventHandler.obj
 0001:00015654       eventHandler_waitForActiveCallbacks 0000000180016654 f   eventHandler.obj
 0001:00015b68       getMethodClass             0000000180016b68 f   eventHandler.obj
 0001:0001620c       commandLoop_exitVmDeathLockOnError 000000018001720c f   eventHelper.obj
 0001:0001637c       commandLoop_sync           000000018001737c f   eventHelper.obj
 0001:000165cc       eventHelper_createEventBag 00000001800175cc f   eventHelper.obj
 0001:000165dc       eventHelper_holdEvents     00000001800175dc f   eventHelper.obj
 0001:00016610       eventHelper_initialize     0000000180017610 f   eventHelper.obj
 0001:00016694       eventHelper_lock           0000000180017694 f   eventHelper.obj
 0001:000166b4       eventHelper_recordClassUnload 00000001800176b4 f   eventHelper.obj
 0001:00016778       eventHelper_recordEvent    0000000180017778 f   eventHelper.obj
 0001:00016870       eventHelper_recordFrameEvent 0000000180017870 f   eventHelper.obj
 0001:00016a4c       eventHelper_releaseEvents  0000000180017a4c f   eventHelper.obj
 0001:00016a80       eventHelper_reportEvents   0000000180017a80 f   eventHelper.obj
 0001:00016b64       eventHelper_reportInvokeDone 0000000180017b64 f   eventHelper.obj
 0001:00016c58       eventHelper_reportVMInit   0000000180017c58 f   eventHelper.obj
 0001:00016d58       eventHelper_reset          0000000180017d58 f   eventHelper.obj
 0001:00016d9c       eventHelper_suspendThread  0000000180017d9c f   eventHelper.obj
 0001:00016e90       eventHelper_unlock         0000000180017e90 f   eventHelper.obj
 0001:00017774       unblockCommandLoop         0000000180018774 f   eventHelper.obj
 0001:00017aa0       dbgsysExec                 0000000180018aa0 f   exec_md.obj
 0001:00017b3c       inStream_clearError        0000000180018b3c f   inStream.obj
 0001:00017b44       inStream_command           0000000180018b44 f   inStream.obj
 0001:00017b48       inStream_destroy           0000000180018b48 f   inStream.obj
 0001:00017b88       inStream_error             0000000180018b88 f   inStream.obj
 0001:00017b90       inStream_id                0000000180018b90 f   inStream.obj
 0001:00017b94       inStream_init              0000000180018b94 f   inStream.obj
 0001:00017bf0       inStream_readArrayRef      0000000180018bf0 f   inStream.obj
 0001:00017c34       inStream_readBoolean       0000000180018c34 f   inStream.obj
 0001:00017c6c       inStream_readByte          0000000180018c6c f   inStream.obj
 0001:00017c90       inStream_readBytes         0000000180018c90 f   inStream.obj
 0001:00017cb0       inStream_readChar          0000000180018cb0 f   inStream.obj
 0001:00017ce0       inStream_readClassLoaderRef 0000000180018ce0 f   inStream.obj
 0001:00017d24       inStream_readClassRef      0000000180018d24 f   inStream.obj
 0001:00017d68       inStream_readDouble        0000000180018d68 f   inStream.obj
 0001:00017d98       inStream_readFieldID       0000000180018d98 f   inStream.obj
 0001:00017d98       inStream_readFrameID       0000000180018d98 f   inStream.obj
 0001:00017d98       inStream_readLocation      0000000180018d98 f   inStream.obj
 0001:00017d98       inStream_readMethodID      0000000180018d98 f   inStream.obj
 0001:00017d98       inStream_readObjectID      0000000180018d98 f   inStream.obj
 0001:00017da0       inStream_readFloat         0000000180018da0 f   inStream.obj
 0001:00017dd0       inStream_readInt           0000000180018dd0 f   inStream.obj
 0001:00017e18       inStream_readLong          0000000180018e18 f   inStream.obj
 0001:00017eb0       inStream_readModuleRef     0000000180018eb0 f   inStream.obj
 0001:00017edc       inStream_readObjectRef     0000000180018edc f   inStream.obj
 0001:00017f60       inStream_readShort         0000000180018f60 f   inStream.obj
 0001:00017f94       inStream_readString        0000000180018f94 f   inStream.obj
 0001:00018028       inStream_readStringRef     0000000180019028 f   inStream.obj
 0001:0001806c       inStream_readThreadGroupRef 000000018001906c f   inStream.obj
 0001:000180b0       inStream_readThreadRef     00000001800190b0 f   inStream.obj
 0001:000180f4       inStream_readValue         00000001800190f4 f   inStream.obj
 0001:000197f0       invoker_completeInvokeRequest 000000018001a7f0 f   invoker.obj
 0001:00019c20       invoker_detach             000000018001ac20 f   invoker.obj
 0001:00019c7c       invoker_doInvoke           000000018001ac7c f   invoker.obj
 0001:00019f4c       invoker_enableInvokeRequests 000000018001af4c f   invoker.obj
 0001:0001a034       invoker_initialize         000000018001b034 f   invoker.obj
 0001:0001a050       invoker_isEnabled          000000018001b050 f   invoker.obj
 0001:0001a138       invoker_lock               000000018001b138 f   invoker.obj
 0001:0001a144       invoker_requestInvoke      000000018001b144 f   invoker.obj
 0001:0001a250       invoker_unlock             000000018001b250 f   invoker.obj
 0001:0001a380       dbgsysBuildLibName         000000018001b380 f   linker_md.obj
 0001:0001a47c       dbgsysFindLibraryEntry     000000018001b47c f   linker_md.obj
 0001:0001a484       dbgsysGetLastErrorString   000000018001b484 f   linker_md.obj
 0001:0001a568       dbgsysLoadLibrary          000000018001b568 f   linker_md.obj
 0001:0001a728       finish_logging             000000018001b728 f   log_messages.obj
 0001:0001a854       log_message_begin          000000018001b854 f   log_messages.obj
 0001:0001a8fc       log_message_end            000000018001b8fc f   log_messages.obj
 0001:0001aac4       setup_logging              000000018001bac4 f   log_messages.obj
 0001:0001aba0       outStream_destroy          000000018001bba0 f   outStream.obj
 0001:0001ac14       outStream_error            000000018001bc14 f   outStream.obj
 0001:0001ac1c       outStream_initCommand      000000018001bc1c f   outStream.obj
 0001:0001ac68       outStream_initReply        000000018001bc68 f   outStream.obj
 0001:0001ad5c       outStream_sendCommand      000000018001bd5c f   outStream.obj
 0001:0001ad80       outStream_sendReply        000000018001bd80 f   outStream.obj
 0001:0001adb0       outStream_setError         000000018001bdb0 f   outStream.obj
 0001:0001ae18       outStream_writeBoolean     000000018001be18 f   outStream.obj
 0001:0001ae38       outStream_writeByte        000000018001be38 f   outStream.obj
 0001:0001ae58       outStream_writeByteArray   000000018001be58 f   outStream.obj
 0001:0001ae94       outStream_writeChar        000000018001be94 f   outStream.obj
 0001:0001aeb8       outStream_writeDouble      000000018001beb8 f   outStream.obj
 0001:0001aef0       outStream_writeFieldID     000000018001bef0 f   outStream.obj
 0001:0001aef0       outStream_writeFrameID     000000018001bef0 f   outStream.obj
 0001:0001aef0       outStream_writeLocation    000000018001bef0 f   outStream.obj
 0001:0001aef0       outStream_writeMethodID    000000018001bef0 f   outStream.obj
 0001:0001aef8       outStream_writeFloat       000000018001bef8 f   outStream.obj
 0001:0001af30       outStream_writeInt         000000018001bf30 f   outStream.obj
 0001:0001af78       outStream_writeLong        000000018001bf78 f   outStream.obj
 0001:0001b010       outStream_writeModuleRef   000000018001c010 f   outStream.obj
 0001:0001b018       outStream_writeObjectRef   000000018001c018 f   outStream.obj
 0001:0001b1f4       outStream_writeObjectTag   000000018001c1f4 f   outStream.obj
 0001:0001b224       outStream_writeShort       000000018001c224 f   outStream.obj
 0001:0001b25c       outStream_writeString      000000018001c25c f   outStream.obj
 0001:0001b328       outStream_writeValue       000000018001c328 f   outStream.obj
 0001:0001b63c       componentTypeSignature     000000018001c63c f   signature.obj
 0001:0001b738       convertSignatureToClassname 000000018001c738 f   signature.obj
 0001:0001b770       methodSignature_init       000000018001c770 f   signature.obj
 0001:0001b7c4       methodSignature_nextArgumentExists 000000018001c7c4 f   signature.obj
 0001:0001b8ac       methodSignature_returnTag  000000018001c8ac f   signature.obj
 0001:0001bab0       standardHandlers_defaultHandler 000000018001cab0 f   standardHandlers.obj
 0001:0001bb28       standardHandlers_onConnect 000000018001cb28 f   standardHandlers.obj
 0001:0001cde4       stepControl_beginStep      000000018001dde4 f   stepControl.obj
 0001:0001cf88       stepControl_clearRequest   000000018001df88 f   stepControl.obj
 0001:0001cfe8       stepControl_endStep        000000018001dfe8 f   stepControl.obj
 0001:0001d06c       stepControl_handleStep     000000018001e06c f   stepControl.obj
 0001:0001d760       stepControl_initialize     000000018001e760 f   stepControl.obj
 0001:0001d77c       stepControl_lock           000000018001e77c f   stepControl.obj
 0001:0001d788       stepControl_resetRequest   000000018001e788 f   stepControl.obj
 0001:0001d8f4       stepControl_unlock         000000018001e8f4 f   stepControl.obj
 0001:0001d900       stream_encodeDouble        000000018001e900 f   stream.obj
 0001:0001d98c       stream_encodeFloat         000000018001e98c f   stream.obj
 0001:0001f76c       threadControl_addDebugThread 000000018002076c f   threadControl.obj
 0001:0001f7f4       threadControl_allVThreads  00000001800207f4 f   threadControl.obj
 0001:0001f8a4       threadControl_applicationThreadStatus 00000001800208a4 f   threadControl.obj
 0001:0001f948       threadControl_clearCLEInfo 0000000180020948 f   threadControl.obj
 0001:0001f9a4       threadControl_cmpCLEInfo   00000001800209a4 f   threadControl.obj
 0001:0001fa50       threadControl_currentThread 0000000180020a50 f   threadControl.obj
 0001:0001fac8       threadControl_detachInvokes 0000000180020ac8 f   threadControl.obj
 0001:0001fb18       threadControl_dumpAllThreads 0000000180020b18 f   threadControl.obj
 0001:0001fb7c       threadControl_getFrameGeneration 0000000180020b7c f   threadControl.obj
 0001:0001fbcc       threadControl_getInstructionStepMode 0000000180020bcc f   threadControl.obj
 0001:0001fc10       threadControl_getInvokeRequest 0000000180020c10 f   threadControl.obj
 0001:0001fc58       threadControl_getStepRequest 0000000180020c58 f   threadControl.obj
 0001:0001fca0       threadControl_initialize   0000000180020ca0 f   threadControl.obj
 0001:0001fce0       threadControl_interrupt    0000000180020ce0 f   threadControl.obj
 0001:0001fd54       threadControl_isDebugThread 0000000180020d54 f   threadControl.obj
 0001:0001fde4       threadControl_onEventHandlerEntry 0000000180020de4 f   threadControl.obj
 0001:000201a4       threadControl_onEventHandlerExit 00000001800211a4 f   threadControl.obj
 0001:00020420       threadControl_onHook       0000000180021420 f   threadControl.obj
 0001:00020574       threadControl_popFrames    0000000180021574 f   threadControl.obj
 0001:0002076c       threadControl_reset        000000018002176c f   threadControl.obj
 0001:000209c0       threadControl_resumeAll    00000001800219c0 f   threadControl.obj
 0001:00020c3c       threadControl_resumeThread 0000000180021c3c f   threadControl.obj
 0001:00020cd8       threadControl_saveCLEInfo  0000000180021cd8 f   threadControl.obj
 0001:00020d64       threadControl_setEventMode 0000000180021d64 f   threadControl.obj
 0001:00020eb0       threadControl_setPendingInterrupt 0000000180021eb0 f   threadControl.obj
 0001:00020f14       threadControl_stop         0000000180021f14 f   threadControl.obj
 0001:00020ffc       threadControl_suspendAll   0000000180021ffc f   threadControl.obj
 0001:00021284       threadControl_suspendCount 0000000180022284 f   threadControl.obj
 0001:000213a0       threadControl_suspendThread 00000001800223a0 f   threadControl.obj
 0001:00021ebc       transport_close            0000000180022ebc f   transport.obj
 0001:00021ed8       transport_initialize       0000000180022ed8 f   transport.obj
 0001:00021f10       transport_is_open          0000000180022f10 f   transport.obj
 0001:00021f30       transport_receivePacket    0000000180022f30 f   transport.obj
 0001:00021f88       transport_reset            0000000180022f88 f   transport.obj
 0001:00021fd0       transport_sendPacket       0000000180022fd0 f   transport.obj
 0001:00022054       transport_startTransport   0000000180023054 f   transport.obj
 0001:000223e4       transport_waitForConnection 00000001800233e4 f   transport.obj
 0001:0002256c       utf8FromPlatform           000000018002356c f   utf_util.obj
 0001:000226c0       utf8ToPlatform             00000001800236c0 f   utf_util.obj
 0001:000227fc       utf8mToUtf8s               00000001800237fc f   utf_util.obj
 0001:000229f4       utf8mToUtf8sLength         00000001800239f4 f   utf_util.obj
 0001:00022b18       utf8sToUtf8m               0000000180023b18 f   utf_util.obj
 0001:00022ce4       utf8sToUtf8mLength         0000000180023ce4 f   utf_util.obj
 0001:00022e1c       allClassLoaderClasses      0000000180023e1c f   util.obj
 0001:00022ea4       allInterfaces              0000000180023ea4 f   util.obj
 0001:00022f2c       allLoadedClasses           0000000180023f2c f   util.obj
 0001:00022fa4       allNestedClasses           0000000180023fa4 f   util.obj
 0001:00023428       allThreads                 0000000180024428 f   util.obj
 0001:00023670       classInstanceCounts        0000000180024670 f   util.obj
 0001:0002392c       classInstances             000000018002492c f   util.obj
 0001:00023b3c       classLoader                0000000180024b3c f   util.obj
 0001:00023bb0       classSignature             0000000180024bb0 f   util.obj
 0001:00023d1c       classStatus                0000000180024d1c f   util.obj
 0001:00023e00       createLocalRefSpace        0000000180024e00 f   util.obj
 0001:00023fc0       debugMonitorCreate         0000000180024fc0 f   util.obj
 0001:000240a8       debugMonitorEnter          00000001800250a8 f   util.obj
 0001:0002418c       debugMonitorExit           000000018002518c f   util.obj
 0001:00024270       debugMonitorNotify         0000000180025270 f   util.obj
 0001:00024354       debugMonitorNotifyAll      0000000180025354 f   util.obj
 0001:00024438       debugMonitorWait           0000000180025438 f   util.obj
 0001:00024548       eventIndex2EventName       0000000180025548 f   util.obj
 0001:000246fc       eventIndex2jdwp            00000001800256fc f   util.obj
 0001:000247ac       eventIndex2jvmti           00000001800257ac f   util.obj
 0001:00024858       eventIndexInit             0000000180025858 f   util.obj
 0001:00024924       fieldModifiers             0000000180025924 f   util.obj
 0001:000249a8       fieldSignature             00000001800259a8 f   util.obj
 0001:00024cd8       filterDebugThreads         0000000180025cd8 f   util.obj
 0001:00024d54       findClass                  0000000180025d54 f   util.obj
 0001:00024fe0       getClassname               0000000180025fe0 f   util.obj
 0001:0002501c       getEnv                     000000018002601c f   util.obj
 0001:00025114       getMethod                  0000000180026114 f   util.obj
 0001:000258ac       getSourceDebugExtension    00000001800268ac f   util.obj
 0001:0002591c       getSpecialJvmti            000000018002691c f   util.obj
 0001:00025dd8       isArray                    0000000180026dd8 f   util.obj
 0001:00025f98       isClass                    0000000180026f98 f   util.obj
 0001:00026010       isClassLoader              0000000180027010 f   util.obj
 0001:00026088       isFieldSynthetic           0000000180027088 f   util.obj
 0001:00026114       isMethodNative             0000000180027114 f   util.obj
 0001:00026200       isMethodObsolete           0000000180027200 f   util.obj
 0001:0002628c       isMethodSynthetic          000000018002728c f   util.obj
 0001:00026308       isObjectTag                0000000180027308 f   util.obj
 0001:00026328       isSameObject               0000000180027328 f   util.obj
 0001:0002633c       isString                   000000018002733c f   util.obj
 0001:000263b4       isThread                   00000001800273b4 f   util.obj
 0001:0002642c       isThreadGroup              000000018002742c f   util.obj
 0001:000264a4       isVThread                  00000001800274a4 f   util.obj
 0001:00026598       jdwp2EventIndex            0000000180027598 f   util.obj
 0001:00026688       jvmtiAllocate              0000000180027688 f   util.obj
 0001:00026778       jvmtiDeallocate            0000000180027778 f   util.obj
 0001:0002685c       jvmtiGetCapabilities       000000018002785c f   util.obj
 0001:00026908       jvmtiMajorVersion          0000000180027908 f   util.obj
 0001:00026920       jvmtiMicroVersion          0000000180027920 f   util.obj
 0001:00026934       jvmtiMinorVersion          0000000180027934 f   util.obj
 0001:00026a40       log_debugee_location       0000000180027a40 f   util.obj
 0001:00026e48       map2jdwpClassStatus        0000000180027e48 f   util.obj
 0001:00026e7c       map2jdwpError              0000000180027e7c f   util.obj
 0001:000271c4       map2jdwpSuspendStatus      00000001800281c4 f   util.obj
 0001:000271d0       map2jdwpThreadStatus       00000001800281d0 f   util.obj
 0001:00027210       map2jvmtiError             0000000180028210 f   util.obj
 0001:000274cc       methodClass                00000001800284cc f   util.obj
 0001:00027540       methodLocation             0000000180028540 f   util.obj
 0001:000275c0       methodModifiers            00000001800285c0 f   util.obj
 0001:00027634       methodReturnType           0000000180028634 f   util.obj
 0001:00027770       methodSignature            0000000180028770 f   util.obj
 0001:00027a8c       objectReferrers            0000000180028a8c f   util.obj
 0001:00027d4c       referenceTypeTag           0000000180028d4c f   util.obj
 0001:00027e58       saveGlobalRef              0000000180028e58 f   util.obj
 0001:000280f0       setAgentPropertyValue      00000001800290f0 f   util.obj
 0001:00028318       sharedGetFieldValues       0000000180029318 f   util.obj
 0001:00028440       sharedInvoke               0000000180029440 f   util.obj
 0001:00028640       spawnNewThread             0000000180029640 f   util.obj
 0001:000289f8       specificTypeKey            00000001800299f8 f   util.obj
 0001:00028c94       threadGroupInfo            0000000180029c94 f   util.obj
 0001:00028d74       tossGlobalRef              0000000180029d74 f   util.obj
 0001:00028f44       uniqueID                   0000000180029f44 f   util.obj
 0001:00028f54       util_initialize            0000000180029f54 f   util.obj
 0001:000296a8       writeCodeLocation          000000018002a6a8 f   util.obj
 0001:00029d30       writeGenericSignature      000000018002ad30 f   util.obj
 0001:0002a2ee       JVM_IsStaticallyLinked     000000018002b2ee f   jvm:jvm.dll
 0001:0002a2f4       __GSHandlerCheck           000000018002b2f4 f   MSVCRT:gshandler.obj
 0001:0002a314       __GSHandlerCheckCommon     000000018002b314 f   MSVCRT:gshandler.obj
 0001:0002a380       __security_check_cookie    000000018002b380 f   MSVCRT:amdsecgs.obj
 0001:0002a3a0       __scrt_acquire_startup_lock 000000018002b3a0 f   MSVCRT:utility.obj
 0001:0002a3dc       __scrt_dllmain_after_initialize_c 000000018002b3dc f   MSVCRT:utility.obj
 0001:0002a410       __scrt_dllmain_before_initialize_c 000000018002b410 f   MSVCRT:utility.obj
 0001:0002a428       __scrt_dllmain_crt_thread_attach 000000018002b428 f   MSVCRT:utility.obj
 0001:0002a450       __scrt_dllmain_crt_thread_detach 000000018002b450 f   MSVCRT:utility.obj
 0001:0002a468       __scrt_dllmain_exception_filter 000000018002b468 f   MSVCRT:utility.obj
 0001:0002a4c8       __scrt_dllmain_uninitialize_c 000000018002b4c8 f   MSVCRT:utility.obj
 0001:0002a4f8       __scrt_dllmain_uninitialize_critical 000000018002b4f8 f   MSVCRT:utility.obj
 0001:0002a50c       __scrt_initialize_crt      000000018002b50c f   MSVCRT:utility.obj
 0001:0002a558       __scrt_initialize_onexit_tables 000000018002b558 f   MSVCRT:utility.obj
 0001:0002a5e4       __scrt_is_nonwritable_in_current_image 000000018002b5e4 f   MSVCRT:utility.obj
 0001:0002a67c       __scrt_release_startup_lock 000000018002b67c f   MSVCRT:utility.obj
 0001:0002a6a0       __scrt_uninitialize_crt    000000018002b6a0 f   MSVCRT:utility.obj
 0001:0002a6cc       _onexit                    000000018002b6cc f   MSVCRT:utility.obj
 0001:0002a708       atexit                     000000018002b708 f   MSVCRT:utility.obj
 0001:0002aa40       _DllMainCRTStartup         000000018002ba40 f   MSVCRT:dll_dllmain.obj
 0001:0002aa80       __raise_securityfailure    000000018002ba80 f   MSVCRT:gs_report.obj
 0001:0002aab4       __report_gsfailure         000000018002bab4 f   MSVCRT:gs_report.obj
 0001:0002abfc       __isa_available_init       000000018002bbfc f   MSVCRT:cpu_disp.obj
 0001:0002ada8       _get_startup_argv_mode     000000018002bda8 f   MSVCRT:argv_mode.obj
 0001:0002adb0       __scrt_is_ucrt_dll_in_use  000000018002bdb0 f   MSVCRT:ucrt_detection.obj
 0001:0002adbc       __crt_debugger_hook        000000018002bdbc f   MSVCRT:utility_desktop.obj
 0001:0002adc4       __scrt_fastfail            000000018002bdc4 f   MSVCRT:utility_desktop.obj
 0001:0002af10       __security_init_cookie     000000018002bf10 f   MSVCRT:gs_support.obj
 0001:0002afbc       DllMain                    000000018002bfbc f   MSVCRT:dll_dllmain_stub.obj
 0001:0002afe0       ?__scrt_initialize_type_info@@YAXXZ 000000018002bfe0 f   MSVCRT:tncleanup.obj
 0001:0002aff0       ?__scrt_uninitialize_type_info@@YAXXZ 000000018002bff0 f   MSVCRT:tncleanup.obj
 0001:0002affc       __local_stdio_scanf_options 000000018002bffc f i MSVCRT:default_local_stdio_options.obj
 0001:0002b004       __scrt_initialize_default_local_stdio_options 000000018002c004 f   MSVCRT:default_local_stdio_options.obj
 0001:0002b020       __scrt_get_dyn_tls_init_callback 000000018002c020 f   MSVCRT:dyn_tls_init.obj
 0001:0002b028       _RTC_Initialize            000000018002c028 f   MSVCRT:initsect.obj
 0001:0002b064       _RTC_Terminate             000000018002c064 f   MSVCRT:initsect.obj
 0001:0002b0a0       memset                     000000018002c0a0 f   vcruntime:VCRUNTIME140.dll
 0001:0002b0a6       longjmp                    000000018002c0a6 f   vcruntime:VCRUNTIME140.dll
 0001:0002b0ac       memcpy                     000000018002c0ac f   vcruntime:VCRUNTIME140.dll
 0001:0002b0b2       strchr                     000000018002c0b2 f   vcruntime:VCRUNTIME140.dll
 0001:0002b0b8       strrchr                    000000018002c0b8 f   vcruntime:VCRUNTIME140.dll
 0001:0002b0be       __intrinsic_setjmp         000000018002c0be f   vcruntime:VCRUNTIME140.dll
 0001:0002b0be       _setjmp                    000000018002c0be f   vcruntime:VCRUNTIME140.dll
 0001:0002b0c4       __C_specific_handler       000000018002c0c4 f   vcruntime:VCRUNTIME140.dll
 0001:0002b0ca       __std_type_info_destroy_list 000000018002c0ca f   vcruntime:VCRUNTIME140.dll
 0001:0002b0d0       strcmp                     000000018002c0d0 f   ucrt:api-ms-win-crt-string-l1-1-0.dll
 0001:0002b0d6       strlen                     000000018002c0d6 f   ucrt:api-ms-win-crt-string-l1-1-0.dll
 0001:0002b0dc       strcat                     000000018002c0dc f   ucrt:api-ms-win-crt-string-l1-1-0.dll
 0001:0002b0e2       strcpy                     000000018002c0e2 f   ucrt:api-ms-win-crt-string-l1-1-0.dll
 0001:0002b0e8       _seh_filter_dll            000000018002c0e8 f   ucrt:api-ms-win-crt-runtime-l1-1-0.dll
 0001:0002b0ee       _configure_narrow_argv     000000018002c0ee f   ucrt:api-ms-win-crt-runtime-l1-1-0.dll
 0001:0002b0f4       _initialize_narrow_environment 000000018002c0f4 f   ucrt:api-ms-win-crt-runtime-l1-1-0.dll
 0001:0002b0fa       _initialize_onexit_table   000000018002c0fa f   ucrt:api-ms-win-crt-runtime-l1-1-0.dll
 0001:0002b100       _register_onexit_function  000000018002c100 f   ucrt:api-ms-win-crt-runtime-l1-1-0.dll
 0001:0002b106       _execute_onexit_table      000000018002c106 f   ucrt:api-ms-win-crt-runtime-l1-1-0.dll
 0001:0002b10c       _crt_atexit                000000018002c10c f   ucrt:api-ms-win-crt-runtime-l1-1-0.dll
 0001:0002b112       _cexit                     000000018002c112 f   ucrt:api-ms-win-crt-runtime-l1-1-0.dll
 0001:0002b118       _initterm                  000000018002c118 f   ucrt:api-ms-win-crt-runtime-l1-1-0.dll
 0001:0002b11e       _initterm_e                000000018002c11e f   ucrt:api-ms-win-crt-runtime-l1-1-0.dll
 0001:0002b124       __scrt_stub_for_is_c_termination_complete 000000018002c124 f   MSVCRT:ucrt_stubs.obj
 0001:0002b124       _is_c_termination_complete 000000018002c124 f   MSVCRT:ucrt_stubs.obj
 0001:0002b140       _guard_dispatch_icall_nop  000000018002c140 f   MSVCRT:guard_dispatch.obj
 0001:0002b160       _guard_xfg_dispatch_icall_nop 000000018002c160 f   MSVCRT:guard_xfg_dispatch.obj
 0002:00000000       __imp_QueryPerformanceCounter 000000018002d000     kernel32:KERNEL32.dll
 0002:00000008       __imp_InitializeSListHead  000000018002d008     kernel32:KERNEL32.dll
 0002:00000010       __imp_Sleep                000000018002d010     kernel32:KERNEL32.dll
 0002:00000018       __imp_GetCurrentThreadId   000000018002d018     kernel32:KERNEL32.dll
 0002:00000020       __imp_CreateProcessA       000000018002d020     kernel32:KERNEL32.dll
 0002:00000028       __imp_GetLastError         000000018002d028     kernel32:KERNEL32.dll
 0002:00000030       __imp_GetProcAddress       000000018002d030     kernel32:KERNEL32.dll
 0002:00000038       __imp_LoadLibraryA         000000018002d038     kernel32:KERNEL32.dll
 0002:00000040       __imp_FormatMessageA       000000018002d040     kernel32:KERNEL32.dll
 0002:00000048       __imp_MultiByteToWideChar  000000018002d048     kernel32:KERNEL32.dll
 0002:00000050       __imp_WideCharToMultiByte  000000018002d050     kernel32:KERNEL32.dll
 0002:00000058       __imp_GetACP               000000018002d058     kernel32:KERNEL32.dll
 0002:00000060       __imp_GetLocaleInfoA       000000018002d060     kernel32:KERNEL32.dll
 0002:00000068       __imp_GetUserDefaultLCID   000000018002d068     kernel32:KERNEL32.dll
 0002:00000070       __imp_RtlCaptureContext    000000018002d070     kernel32:KERNEL32.dll
 0002:00000078       __imp_RtlLookupFunctionEntry 000000018002d078     kernel32:KERNEL32.dll
 0002:00000080       __imp_RtlVirtualUnwind     000000018002d080     kernel32:KERNEL32.dll
 0002:00000088       __imp_UnhandledExceptionFilter 000000018002d088     kernel32:KERNEL32.dll
 0002:00000090       __imp_SetUnhandledExceptionFilter 000000018002d090     kernel32:KERNEL32.dll
 0002:00000098       __imp_GetCurrentProcess    000000018002d098     kernel32:KERNEL32.dll
 0002:000000a0       __imp_TerminateProcess     000000018002d0a0     kernel32:KERNEL32.dll
 0002:000000a8       __imp_IsProcessorFeaturePresent 000000018002d0a8     kernel32:KERNEL32.dll
 0002:000000b0       __imp_IsDebuggerPresent    000000018002d0b0     kernel32:KERNEL32.dll
 0002:000000b8       __imp_DisableThreadLibraryCalls 000000018002d0b8     kernel32:KERNEL32.dll
 0002:000000c0       __imp_GetCurrentProcessId  000000018002d0c0     kernel32:KERNEL32.dll
 0002:000000c8       __imp_GetSystemTimeAsFileTime 000000018002d0c8     kernel32:KERNEL32.dll
 0002:000000d0       \177KERNEL32_NULL_THUNK_DATA 000000018002d0d0     kernel32:KERNEL32.dll
 0002:000000d8       __imp___std_type_info_destroy_list 000000018002d0d8     vcruntime:VCRUNTIME140.dll
 0002:000000e0       __imp___C_specific_handler 000000018002d0e0     vcruntime:VCRUNTIME140.dll
 0002:000000e8       __imp_memset               000000018002d0e8     vcruntime:VCRUNTIME140.dll
 0002:000000f0       __imp_longjmp              000000018002d0f0     vcruntime:VCRUNTIME140.dll
 0002:000000f8       __imp_memcpy               000000018002d0f8     vcruntime:VCRUNTIME140.dll
 0002:00000100       __imp_strchr               000000018002d100     vcruntime:VCRUNTIME140.dll
 0002:00000108       __imp_strrchr              000000018002d108     vcruntime:VCRUNTIME140.dll
 0002:00000110       __imp___intrinsic_setjmp   000000018002d110     vcruntime:VCRUNTIME140.dll
 0002:00000118       \177VCRUNTIME140_NULL_THUNK_DATA 000000018002d118     vcruntime:VCRUNTIME140.dll
 0002:00000120       __imp_strtol               000000018002d120     ucrt:api-ms-win-crt-convert-l1-1-0.dll
 0002:00000128       __imp_atoi                 000000018002d128     ucrt:api-ms-win-crt-convert-l1-1-0.dll
 0002:00000130       __imp_atol                 000000018002d130     ucrt:api-ms-win-crt-convert-l1-1-0.dll
 0002:00000138       \177api-ms-win-crt-convert-l1-1-0_NULL_THUNK_DATA 000000018002d138     ucrt:api-ms-win-crt-convert-l1-1-0.dll
 0002:00000140       __imp_getenv               000000018002d140     ucrt:api-ms-win-crt-environment-l1-1-0.dll
 0002:00000148       \177api-ms-win-crt-environment-l1-1-0_NULL_THUNK_DATA 000000018002d148     ucrt:api-ms-win-crt-environment-l1-1-0.dll
 0002:00000150       __imp__access              000000018002d150     ucrt:api-ms-win-crt-filesystem-l1-1-0.dll
 0002:00000158       \177api-ms-win-crt-filesystem-l1-1-0_NULL_THUNK_DATA 000000018002d158     ucrt:api-ms-win-crt-filesystem-l1-1-0.dll
 0002:00000160       __imp_malloc               000000018002d160     ucrt:api-ms-win-crt-heap-l1-1-0.dll
 0002:00000168       __imp_free                 000000018002d168     ucrt:api-ms-win-crt-heap-l1-1-0.dll
 0002:00000170       \177api-ms-win-crt-heap-l1-1-0_NULL_THUNK_DATA 000000018002d170     ucrt:api-ms-win-crt-heap-l1-1-0.dll
 0002:00000178       __imp_abort                000000018002d178     ucrt:api-ms-win-crt-runtime-l1-1-0.dll
 0002:00000180       __imp_exit                 000000018002d180     ucrt:api-ms-win-crt-runtime-l1-1-0.dll
 0002:00000188       __imp__cexit               000000018002d188     ucrt:api-ms-win-crt-runtime-l1-1-0.dll
 0002:00000190       __imp__initialize_onexit_table 000000018002d190     ucrt:api-ms-win-crt-runtime-l1-1-0.dll
 0002:00000198       __imp__initialize_narrow_environment 000000018002d198     ucrt:api-ms-win-crt-runtime-l1-1-0.dll
 0002:000001a0       __imp__errno               000000018002d1a0     ucrt:api-ms-win-crt-runtime-l1-1-0.dll
 0002:000001a8       __imp_strerror             000000018002d1a8     ucrt:api-ms-win-crt-runtime-l1-1-0.dll
 0002:000001b0       __imp__crt_atexit          000000018002d1b0     ucrt:api-ms-win-crt-runtime-l1-1-0.dll
 0002:000001b8       __imp__initterm            000000018002d1b8     ucrt:api-ms-win-crt-runtime-l1-1-0.dll
 0002:000001c0       __imp__configure_narrow_argv 000000018002d1c0     ucrt:api-ms-win-crt-runtime-l1-1-0.dll
 0002:000001c8       __imp__seh_filter_dll      000000018002d1c8     ucrt:api-ms-win-crt-runtime-l1-1-0.dll
 0002:000001d0       __imp__register_onexit_function 000000018002d1d0     ucrt:api-ms-win-crt-runtime-l1-1-0.dll
 0002:000001d8       __imp__initterm_e          000000018002d1d8     ucrt:api-ms-win-crt-runtime-l1-1-0.dll
 0002:000001e0       __imp__execute_onexit_table 000000018002d1e0     ucrt:api-ms-win-crt-runtime-l1-1-0.dll
 0002:000001e8       __imp__getpid              000000018002d1e8     ucrt:api-ms-win-crt-runtime-l1-1-0.dll
 0002:000001e8       __imp_getpid               000000018002d1e8     ucrt:api-ms-win-crt-runtime-l1-1-0.dll
 0002:000001f0       \177api-ms-win-crt-runtime-l1-1-0_NULL_THUNK_DATA 000000018002d1f0     ucrt:api-ms-win-crt-runtime-l1-1-0.dll
 0002:000001f8       __imp___acrt_iob_func      000000018002d1f8     ucrt:api-ms-win-crt-stdio-l1-1-0.dll
 0002:00000200       __imp_fopen                000000018002d200     ucrt:api-ms-win-crt-stdio-l1-1-0.dll
 0002:00000208       __imp_fclose               000000018002d208     ucrt:api-ms-win-crt-stdio-l1-1-0.dll
 0002:00000210       __imp___stdio_common_vfprintf 000000018002d210     ucrt:api-ms-win-crt-stdio-l1-1-0.dll
 0002:00000218       __imp_fflush               000000018002d218     ucrt:api-ms-win-crt-stdio-l1-1-0.dll
 0002:00000220       __imp_setvbuf              000000018002d220     ucrt:api-ms-win-crt-stdio-l1-1-0.dll
 0002:00000228       __imp___stdio_common_vsprintf 000000018002d228     ucrt:api-ms-win-crt-stdio-l1-1-0.dll
 0002:00000230       \177api-ms-win-crt-stdio-l1-1-0_NULL_THUNK_DATA 000000018002d230     ucrt:api-ms-win-crt-stdio-l1-1-0.dll
 0002:00000238       __imp_strncpy              000000018002d238     ucrt:api-ms-win-crt-string-l1-1-0.dll
 0002:00000240       __imp_strtok_s             000000018002d240     ucrt:api-ms-win-crt-string-l1-1-0.dll
 0002:00000248       __imp_strcpy               000000018002d248     ucrt:api-ms-win-crt-string-l1-1-0.dll
 0002:00000250       __imp_strcat               000000018002d250     ucrt:api-ms-win-crt-string-l1-1-0.dll
 0002:00000258       __imp_strncmp              000000018002d258     ucrt:api-ms-win-crt-string-l1-1-0.dll
 0002:00000260       __imp_strlen               000000018002d260     ucrt:api-ms-win-crt-string-l1-1-0.dll
 0002:00000268       __imp_strcmp               000000018002d268     ucrt:api-ms-win-crt-string-l1-1-0.dll
 0002:00000270       __imp_isdigit              000000018002d270     ucrt:api-ms-win-crt-string-l1-1-0.dll
 0002:00000278       \177api-ms-win-crt-string-l1-1-0_NULL_THUNK_DATA 000000018002d278     ucrt:api-ms-win-crt-string-l1-1-0.dll
 0002:00000280       __imp_strftime             000000018002d280     ucrt:api-ms-win-crt-time-l1-1-0.dll
 0002:00000288       __imp__localtime64         000000018002d288     ucrt:api-ms-win-crt-time-l1-1-0.dll
 0002:00000290       __imp__time64              000000018002d290     ucrt:api-ms-win-crt-time-l1-1-0.dll
 0002:00000298       \177api-ms-win-crt-time-l1-1-0_NULL_THUNK_DATA 000000018002d298     ucrt:api-ms-win-crt-time-l1-1-0.dll
 0002:000002a0       __imp_JVM_IsStaticallyLinked 000000018002d2a0     jvm:jvm.dll
 0002:000002a8       \177jvm_NULL_THUNK_DATA    000000018002d2a8     jvm:jvm.dll
 0002:000002b0       __guard_check_icall_fptr   000000018002d2b0     MSVCRT:guard_support.obj
 0002:000002b8       __guard_xfg_check_icall_fptr 000000018002d2b8     MSVCRT:guard_support.obj
 0002:000002c0       __guard_dispatch_icall_fptr 000000018002d2c0     MSVCRT:guard_support.obj
 0002:000002c8       __guard_xfg_dispatch_icall_fptr 000000018002d2c8     MSVCRT:guard_support.obj
 0002:000002d0       __guard_xfg_table_dispatch_icall_fptr 000000018002d2d0     MSVCRT:guard_support.obj
 0002:000002d8       __castguard_check_failure_os_handled_fptr 000000018002d2d8     MSVCRT:guard_support.obj
 0002:000002e0       __guard_memcpy_fptr        000000018002d2e0     vcruntime:softmemtag.obj
 0002:000002e8       __xc_a                     000000018002d2e8     MSVCRT:initializers.obj
 0002:000002f0       __xc_z                     000000018002d2f0     MSVCRT:initializers.obj
 0002:000002f8       __xi_a                     000000018002d2f8     MSVCRT:initializers.obj
 0002:00000300       __xi_z                     000000018002d300     MSVCRT:initializers.obj
 0002:00000308       __xp_a                     000000018002d308     MSVCRT:initializers.obj
 0002:00000310       __xp_z                     000000018002d310     MSVCRT:initializers.obj
 0002:00000318       __xt_a                     000000018002d318     MSVCRT:initializers.obj
 0002:00000320       __xt_z                     000000018002d320     MSVCRT:initializers.obj
 0002:00000330       ??_C@_0BM@KIOODJOG@Tag?5is?5not?5a?5JVM?5basic?5type@ 000000018002d330     ArrayReferenceImpl.obj
 0002:00000350       ??_C@_0DG@KNIKPIPG@s?2src?2jdk?4jdwp?4agent?2share?2nati@ 000000018002d350     ArrayReferenceImpl.obj
 0002:00000388       ??_C@_0DP@KOAIFEMO@s?2src?2jdk?4jdwp?4agent?2share?2nati@ 000000018002d388     ArrayReferenceImpl.obj
 0002:000003c8       ??_C@_03HBKNMMDM@JNI@      000000018002d3c8     ArrayReferenceImpl.obj
 0002:000003d0       ??_C@_0P@KJGLIDCM@GetArrayLength@ 000000018002d3d0     ArrayReferenceImpl.obj
 0002:000003e0       ??_C@_04DLGOCPFH@?$CFs?$CI?$CJ@ 000000018002d3e0     ArrayReferenceImpl.obj
 0002:000003e8       ??_C@_0BG@DOJPBGJK@GetBooleanArrayRegion@ 000000018002d3e8     ArrayReferenceImpl.obj
 0002:00000400       ??_C@_0BD@DBCKLPHC@GetByteArrayRegion@ 000000018002d400     ArrayReferenceImpl.obj
 0002:00000418       ??_C@_0BD@EJLOJIMH@GetCharArrayRegion@ 000000018002d418     ArrayReferenceImpl.obj
 0002:00000430       ??_C@_0BE@LJPMIBLN@GetShortArrayRegion@ 000000018002d430     ArrayReferenceImpl.obj
 0002:00000448       ??_C@_0BC@PAFAELMA@GetIntArrayRegion@ 000000018002d448     ArrayReferenceImpl.obj
 0002:00000460       ??_C@_0BD@KDOJFBNI@GetLongArrayRegion@ 000000018002d460     ArrayReferenceImpl.obj
 0002:00000478       ??_C@_0BE@JEOBKBHM@GetFloatArrayRegion@ 000000018002d478     ArrayReferenceImpl.obj
 0002:00000490       ??_C@_0BF@HGGNLGEB@GetDoubleArrayRegion@ 000000018002d490     ArrayReferenceImpl.obj
 0002:000004a8       ??_C@_0BG@KEKOCCJB@GetObjectArrayElement@ 000000018002d4a8     ArrayReferenceImpl.obj
 0002:000004c0       ??_C@_0P@MIECHIDO@ExceptionCheck@ 000000018002d4c0     ArrayReferenceImpl.obj
 0002:000004d0       ??_C@_0O@EMINCBBD@PopLocalFrame@ 000000018002d4d0     ArrayReferenceImpl.obj
 0002:000004e0       ??_C@_0P@NDOJPFLH@GetObjectClass@ 000000018002d4e0     ArrayReferenceImpl.obj
 0002:000004f0       ??_C@_0P@KFEGKDII@ExceptionClear@ 000000018002d4f0     ArrayReferenceImpl.obj
 0002:00000500       ??_C@_0BG@MLMJMPNL@SetBooleanArrayRegion@ 000000018002d500     ArrayReferenceImpl.obj
 0002:00000518       ??_C@_0BD@MLAAIJJK@SetByteArrayRegion@ 000000018002d518     ArrayReferenceImpl.obj
 0002:00000530       ??_C@_0BD@LDJEKOCP@SetCharArrayRegion@ 000000018002d530     ArrayReferenceImpl.obj
 0002:00000548       ??_C@_0BE@BHNHMBMB@SetShortArrayRegion@ 000000018002d548     ArrayReferenceImpl.obj
 0002:00000560       ??_C@_0BC@NFFLMANO@SetIntArrayRegion@ 000000018002d560     ArrayReferenceImpl.obj
 0002:00000578       ??_C@_0BD@FJMDGHDA@SetLongArrayRegion@ 000000018002d578     ArrayReferenceImpl.obj
 0002:00000590       ??_C@_0BE@DKMKOBAA@SetFloatArrayRegion@ 000000018002d590     ArrayReferenceImpl.obj
 0002:000005a8       ??_C@_0BF@CPHAKABG@SetDoubleArrayRegion@ 000000018002d5a8     ArrayReferenceImpl.obj
 0002:000005c0       ??_C@_0BG@FBPIPLNA@SetObjectArrayElement@ 000000018002d5c0     ArrayReferenceImpl.obj
 0002:000005d8       ??_C@_05MBDEGLCK@ERROR@    000000018002d5d8     ArrayReferenceImpl.obj
 0002:000005e0       ??_C@_0CG@CDCBEMAB@Invalid?5array?5component?5signatu@ 000000018002d5e0     ArrayReferenceImpl.obj
 0002:00000606       ??_C@_00CNPNBAHC@@         000000018002d606     ArrayReferenceImpl.obj
 0002:00000608       ??_C@_0BD@HJCIAOFF@?$CFs?$CI?$CFd?$CJ?3?5?$CFs?5?$FL?$CFs?3?$CFd?$FN@ 000000018002d608     ArrayReferenceImpl.obj
 0002:0000061c       ??_C@_01EEMJAFIK@?6@       000000018002d61c     ArrayReferenceImpl.obj
 0002:00000620       ??_C@_0BB@BCMBBBKH@JDWP?5exit?5error?5@ 000000018002d620     ArrayReferenceImpl.obj
 0002:00000634       ??_C@_06MHCOIGNA@Length@   000000018002d634     ArrayReferenceImpl.obj
 0002:00000640       ??_C@_09JHHNDJLP@GetValues@ 000000018002d640     ArrayReferenceImpl.obj
 0002:00000650       ??_C@_09LJDIBICN@SetValues@ 000000018002d650     ArrayReferenceImpl.obj
 0002:00000660       ??_C@_0P@EGNIMIAH@ArrayReference@ 000000018002d660     ArrayReferenceImpl.obj
 0002:00000670       ??_C@_0DK@KCBNOHN@s?2src?2jdk?4jdwp?4agent?2share?2nati@ 000000018002d670     ArrayTypeImpl.obj
 0002:000006b0       ??_C@_0P@CNKIGBBL@NewObjectArray@ 000000018002d6b0     ArrayTypeImpl.obj
 0002:000006c0       ??_C@_0N@NGBLEHOM@NewByteArray@ 000000018002d6c0     ArrayTypeImpl.obj
 0002:000006d0       ??_C@_0N@BEEAOHOP@NewCharArray@ 000000018002d6d0     ArrayTypeImpl.obj
 0002:000006e0       ??_C@_0O@KEDKGJJM@NewFloatArray@ 000000018002d6e0     ArrayTypeImpl.obj
 0002:000006f0       ??_C@_0P@DNODLKGI@NewDoubleArray@ 000000018002d6f0     ArrayTypeImpl.obj
 0002:00000700       ??_C@_0M@PGNBGLNB@NewIntArray@ 000000018002d700     ArrayTypeImpl.obj
 0002:00000710       ??_C@_0N@GNOMHAGO@NewLongArray@ 000000018002d710     ArrayTypeImpl.obj
 0002:00000720       ??_C@_0O@IAEEJHKH@NewShortArray@ 000000018002d720     ArrayTypeImpl.obj
 0002:00000730       ??_C@_0BA@IMLHDFCA@NewBooleanArray@ 000000018002d730     ArrayTypeImpl.obj
 0002:00000740       ??_C@_0M@LPLNEPAH@NewInstance@ 000000018002d740     ArrayTypeImpl.obj
 0002:00000750       ??_C@_09MLBOOMFO@ArrayType@ 000000018002d750     ArrayTypeImpl.obj
 0002:00000760       ??_C@_0EF@FKFHKPAA@s?2src?2jdk?4jdwp?4agent?2share?2nati@ 000000018002d760     ClassLoaderReferenceImpl.obj
 0002:000007a8       ??_C@_0P@GEMMHMHN@VisibleClasses@ 000000018002d7a8     ClassLoaderReferenceImpl.obj
 0002:000007b8       ??_C@_0BF@MJJABFGE@ClassLoaderReference@ 000000018002d7b8     ClassLoaderReferenceImpl.obj
 0002:000007d0       ??_C@_0O@MBFCJPMM@ReflectedType@ 000000018002d7d0     ClassObjectReferenceImpl.obj
 0002:000007e0       ??_C@_0BF@IJHAFOFB@ClassObjectReference@ 000000018002d7e0     ClassObjectReferenceImpl.obj
 0002:000007f8       ??_C@_0DK@CPJOGD@s?2src?2jdk?4jdwp?4agent?2share?2nati@ 000000018002d7f8     ClassTypeImpl.obj
 0002:00000838       ??_C@_0O@NPFONKNM@GetSuperclass@ 000000018002d838     ClassTypeImpl.obj
 0002:00000848       ??_C@_0BF@NBNNHFAL@SetStaticObjectField@ 000000018002d848     ClassTypeImpl.obj
 0002:00000860       ??_C@_0BD@IANJADAE@SetStaticByteField@ 000000018002d860     ClassTypeImpl.obj
 0002:00000878       ??_C@_0BD@ECICKDAH@SetStaticCharField@ 000000018002d878     ClassTypeImpl.obj
 0002:00000890       ??_C@_0BE@KCBAKIGK@SetStaticFloatField@ 000000018002d890     ClassTypeImpl.obj
 0002:000008a8       ??_C@_0BF@MBJGKOHI@SetStaticDoubleField@ 000000018002d8a8     ClassTypeImpl.obj
 0002:000008c0       ??_C@_0BC@ENOHANEJ@SetStaticIntField@ 000000018002d8c0     ClassTypeImpl.obj
 0002:000008d8       ??_C@_0BD@DLCODEIG@SetStaticLongField@ 000000018002d8d8     ClassTypeImpl.obj
 0002:000008f0       ??_C@_0BE@IGGOFGFB@SetStaticShortField@ 000000018002d8f0     ClassTypeImpl.obj
 0002:00000908       ??_C@_0BG@DJFBDJKI@SetStaticBooleanField@ 000000018002d908     ClassTypeImpl.obj
 0002:00000920       ??_C@_0L@HFIGJMAA@Superclass@ 000000018002d920     ClassTypeImpl.obj
 0002:00000930       ??_C@_0N@LGIJNKMO@InvokeMethod@ 000000018002d930     ClassTypeImpl.obj
 0002:00000940       ??_C@_09IAHDNMJ@ClassType@ 000000018002d940     ClassTypeImpl.obj
 0002:00000950       ??_C@_0L@CAMDCGEO@SetCommand@ 000000018002d950     EventRequestImpl.obj
 0002:00000960       ??_C@_0N@NDABFFGD@ClearCommand@ 000000018002d960     EventRequestImpl.obj
 0002:00000970       ??_C@_0BE@IJFBELDD@ClearAllBreakpoints@ 000000018002d970     EventRequestImpl.obj
 0002:00000988       ??_C@_0N@PGGBGIFJ@EventRequest@ 000000018002d988     EventRequestImpl.obj
 0002:00000998       ??_C@_05EPLKDJMH@Field@    000000018002d998     FieldImpl.obj
 0002:000009a0       ??_C@_0O@IHENGMAG@InterfaceType@ 000000018002d9a0     InterfaceTypeImpl.obj
 0002:000009b0       ??_C@_0DH@BMAMHHMB@s?2src?2jdk?4jdwp?4agent?2share?2nati@ 000000018002d9b0     MethodImpl.obj
 0002:000009e8       ??_C@_05HENNLPPN@JVMTI@    000000018002d9e8     MethodImpl.obj
 0002:000009f0       ??_C@_0BD@MHLEIAPA@GetLineNumberTable@ 000000018002d9f0     MethodImpl.obj
 0002:00000a08       ??_C@_0BB@ELDBFBNO@GetArgumentsSize@ 000000018002da08     MethodImpl.obj
 0002:00000a20       ??_C@_0BG@JNJHMCNH@GetLocalVariableTable@ 000000018002da20     MethodImpl.obj
 0002:00000a38       ??_C@_0N@JCOMJEBO@GetBytecodes@ 000000018002da38     MethodImpl.obj
 0002:00000a48       ??_C@_09IPPJBAKB@LineTable@ 000000018002da48     MethodImpl.obj
 0002:00000a58       ??_C@_0O@CIFPCEPG@VariableTable@ 000000018002da58     MethodImpl.obj
 0002:00000a68       ??_C@_09EAOGBHHA@Bytecodes@ 000000018002da68     MethodImpl.obj
 0002:00000a78       ??_C@_0L@IIIMIJNI@IsObsolete@ 000000018002da78     MethodImpl.obj
 0002:00000a88       ??_C@_0BK@ILPNHFLA@VariableTableWithGenerics@ 000000018002da88     MethodImpl.obj
 0002:00000aa4       ??_C@_06KPKMBBIM@Method@   000000018002daa4     MethodImpl.obj
 0002:00000ab0       ??_C@_0BB@JPJICBFE@java?1lang?1Module@ 000000018002dab0     ModuleReferenceImpl.obj
 0002:00000ac8       ??_C@_0BF@FOHFOJOB@?$CI?$CJLjava?1lang?1String?$DL@ 000000018002dac8     ModuleReferenceImpl.obj
 0002:00000ae0       ??_C@_07DFBCBEHO@getName@  000000018002dae0     ModuleReferenceImpl.obj
 0002:00000af0       ??_C@_0EA@MKGDLANN@s?2src?2jdk?4jdwp?4agent?2share?2nati@ 000000018002daf0     ModuleReferenceImpl.obj
 0002:00000b30       ??_C@_0BB@FFOMHKKA@CallObjectMethod@ 000000018002db30     ModuleReferenceImpl.obj
 0002:00000b48       ??_C@_0DA@PDDOKJCN@JNI?5Exception?5occurred?5calling?5@ 000000018002db48     ModuleReferenceImpl.obj
 0002:00000b78       ??_C@_0BC@EDLHHKLL@GetStringUTFChars@ 000000018002db78     ModuleReferenceImpl.obj
 0002:00000b90       ??_C@_0BG@CNECBEKD@ReleaseStringUTFChars@ 000000018002db90     ModuleReferenceImpl.obj
 0002:00000ba8       ??_C@_0BK@JHGGPLEI@?$CI?$CJLjava?1lang?1ClassLoader?$DL@ 000000018002dba8     ModuleReferenceImpl.obj
 0002:00000bc8       ??_C@_0P@HCMNKIPB@getClassLoader@ 000000018002dbc8     ModuleReferenceImpl.obj
 0002:00000bd8       ??_C@_0DM@DHHMKOMK@JNI?5Exception?5occurred?5calling?5@ 000000018002dbd8     ModuleReferenceImpl.obj
 0002:00000c18       ??_C@_07MMGEHGCI@GetName@  000000018002dc18     ModuleReferenceImpl.obj
 0002:00000c20       ??_C@_0P@PKAIJGGP@GetClassLoader@ 000000018002dc20     ModuleReferenceImpl.obj
 0002:00000c30       ??_C@_0BA@OGHCDEJN@ModuleReference@ 000000018002dc30     ModuleReferenceImpl.obj
 0002:00000c40       ??_C@_0EA@CANAHBDF@s?2src?2jdk?4jdwp?4agent?2share?2nati@ 000000018002dc40     ObjectReferenceImpl.obj
 0002:00000c80       ??_C@_0P@BIEBOGNE@SetObjectField@ 000000018002dc80     ObjectReferenceImpl.obj
 0002:00000c90       ??_C@_0N@IMJNOBAL@SetByteField@ 000000018002dc90     ObjectReferenceImpl.obj
 0002:00000ca0       ??_C@_0N@EOMGEBAI@SetCharField@ 000000018002dca0     ObjectReferenceImpl.obj
 0002:00000cb0       ??_C@_0O@DCKDPBBJ@SetFloatField@ 000000018002dcb0     ObjectReferenceImpl.obj
 0002:00000cc0       ??_C@_0P@IAKDNKH@SetDoubleField@ 000000018002dcc0     ObjectReferenceImpl.obj
 0002:00000cd0       ??_C@_0M@LPBODKIC@SetIntField@ 000000018002dcd0     ObjectReferenceImpl.obj
 0002:00000ce0       ??_C@_0N@DHGKNGIJ@SetLongField@ 000000018002dce0     ObjectReferenceImpl.obj
 0002:00000cf0       ??_C@_0O@BGNNAPCC@SetShortField@ 000000018002dcf0     ObjectReferenceImpl.obj
 0002:00000d00       ??_C@_0BA@CPPEGKHO@SetBooleanField@ 000000018002dd00     ObjectReferenceImpl.obj
 0002:00000d10       ??_C@_0BG@LNEALOFM@GetObjectMonitorUsage@ 000000018002dd10     ObjectReferenceImpl.obj
 0002:00000d28       ??_C@_0O@EJIAIJCO@ReferenceType@ 000000018002dd28     ObjectReferenceImpl.obj
 0002:00000d38       ??_C@_08JLEAJAG@?$DMunused?$DO@ 000000018002dd38     ObjectReferenceImpl.obj
 0002:00000d48       ??_C@_0M@OFAPJLBC@MonitorInfo@ 000000018002dd48     ObjectReferenceImpl.obj
 0002:00000d58       ??_C@_0P@NMHCCJ@InvokeInstance@ 000000018002dd58     ObjectReferenceImpl.obj
 0002:00000d68       ??_C@_0BC@IIMACDIN@DisableCollection@ 000000018002dd68     ObjectReferenceImpl.obj
 0002:00000d80       ??_C@_0BB@MDMHJMHH@EnableCollection@ 000000018002dd80     ObjectReferenceImpl.obj
 0002:00000d98       ??_C@_0M@FOFOOCGH@IsCollected@ 000000018002dd98     ObjectReferenceImpl.obj
 0002:00000da8       ??_C@_0BB@CHKFAPKH@ReferringObjects@ 000000018002dda8     ObjectReferenceImpl.obj
 0002:00000dc0       ??_C@_0BA@PPKMBENC@ObjectReference@ 000000018002ddc0     ObjectReferenceImpl.obj
 0002:00000dd0       ??_C@_0DO@MDHPDAFB@s?2src?2jdk?4jdwp?4agent?2share?2nati@ 000000018002ddd0     ReferenceTypeImpl.obj
 0002:00000e10       ??_C@_09OLJHFFGC@GetModule@ 000000018002de10     ReferenceTypeImpl.obj
 0002:00000e20       ??_C@_0BC@GCIFGINE@GetClassModifiers@ 000000018002de20     ReferenceTypeImpl.obj
 0002:00000e38       ??_C@_0BA@FAMCEADF@GetClassMethods@ 000000018002de38     ReferenceTypeImpl.obj
 0002:00000e48       ??_C@_0BH@CNLIIJEM@GetClassVersionNumbers@ 000000018002de48     ReferenceTypeImpl.obj
 0002:00000e60       ??_C@_0BA@CMEFDKBB@GetConstantPool@ 000000018002de60     ReferenceTypeImpl.obj
 0002:00000e70       ??_C@_0P@KAMMPPGF@GetClassFields@ 000000018002de70     ReferenceTypeImpl.obj
 0002:00000e80       ??_C@_0BC@NBHLJMHF@GetSourceFileName@ 000000018002de80     ReferenceTypeImpl.obj
 0002:00000e98       ??_C@_09GDNFOKKF@Signature@ 000000018002de98     ReferenceTypeImpl.obj
 0002:00000ea8       ??_C@_09KLHEJKNK@Modifiers@ 000000018002dea8     ReferenceTypeImpl.obj
 0002:00000eb4       ??_C@_06BFNMHBP@Fields@    000000018002deb4     ReferenceTypeImpl.obj
 0002:00000ec0       ??_C@_07OALDEJCP@Methods@  000000018002dec0     ReferenceTypeImpl.obj
 0002:00000ec8       ??_C@_0L@CLDEMKOL@SourceFile@ 000000018002dec8     ReferenceTypeImpl.obj
 0002:00000ed8       ??_C@_0M@GJNEEGFC@NestedTypes@ 000000018002ded8     ReferenceTypeImpl.obj
 0002:00000ee8       ??_C@_0P@FHKLENLO@GetClassStatus@ 000000018002dee8     ReferenceTypeImpl.obj
 0002:00000ef8       ??_C@_0L@KBICGJBH@Interfaces@ 000000018002def8     ReferenceTypeImpl.obj
 0002:00000f08       ??_C@_0M@GFAKFENF@ClassObject@ 000000018002df08     ReferenceTypeImpl.obj
 0002:00000f18       ??_C@_0BF@JDJPNKHD@SourceDebugExtension@ 000000018002df18     ReferenceTypeImpl.obj
 0002:00000f30       ??_C@_0BF@IKGHKLIB@SignatureWithGeneric@ 000000018002df30     ReferenceTypeImpl.obj
 0002:00000f48       ??_C@_0BC@MCKDAAHH@FieldsWithGeneric@ 000000018002df48     ReferenceTypeImpl.obj
 0002:00000f60       ??_C@_0BD@KPILANFP@MethodsWithGeneric@ 000000018002df60     ReferenceTypeImpl.obj
 0002:00000f78       ??_C@_09FGLEONFO@Instances@ 000000018002df78     ReferenceTypeImpl.obj
 0002:00000f88       ??_C@_0BA@GGCIPEOH@GetClassVersion@ 000000018002df88     ReferenceTypeImpl.obj
 0002:00000f98       ??_C@_0DA@BMDMENKL@s?2src?2jdk?4jdwp?4agent?2share?2nati@ 000000018002df98     SDE.obj
 0002:00000fc8       ??_C@_04MKAMAPIC@MISC@     000000018002dfc8     SDE.obj
 0002:00000fd0       ??_C@_0CC@FDGBKJLJ@SDE?5is?5re?9ordering?5the?5line?5tab@ 000000018002dfd0     SDE.obj
 0002:00000ff8       ??_C@_0DE@CBOCIEPK@bad?5SourceDebugExtension?5syntax@ 000000018002dff8     SDE.obj
 0002:00001030       ??_C@_0P@BFDGOIGG@unexpected?5EOF@ 000000018002e030     SDE.obj
 0002:00001040       ??_C@_0P@BPOMJGMN@SDE?5line?5table@ 000000018002e040     SDE.obj
 0002:00001050       ??_C@_0P@NDLFOGMP@SDE?5file?5table@ 000000018002e050     SDE.obj
 0002:00001060       ??_C@_0BC@JMMEOMHE@SDE?5stratum?5table@ 000000018002e060     SDE.obj
 0002:00001078       ??_C@_0N@PPNMFI@expected?5?8?3?8@ 000000018002e078     SDE.obj
 0002:00001088       ??_C@_04IEJOJGGI@Java@     000000018002e088     SDE.obj
 0002:00001090       ??_C@_03EIMPEGPO@Aux@      000000018002e090     SDE.obj
 0002:00001098       ??_C@_0N@BMNJHPCI@expected?5?8?$CK?8@ 000000018002e098     SDE.obj
 0002:000010a8       ??_C@_0N@KAHJKGJC@?$CKterminator?$CK@ 000000018002e0a8     SDE.obj
 0002:000010b8       ??_C@_0DL@OGCCGFPD@s?2src?2jdk?4jdwp?4agent?2share?2nati@ 000000018002e0b8     StackFrameImpl.obj
 0002:000010f8       ??_C@_0P@CCOLHCFB@GetLocalObject@ 000000018002e0f8     StackFrameImpl.obj
 0002:00001108       ??_C@_0M@OFKPGHNH@GetLocalInt@ 000000018002e108     StackFrameImpl.obj
 0002:00001118       ??_C@_0O@BDGHGOEC@GetLocalFloat@ 000000018002e118     StackFrameImpl.obj
 0002:00001128       ??_C@_0P@LLJAGJLC@GetLocalDouble@ 000000018002e128     StackFrameImpl.obj
 0002:00001138       ??_C@_0N@FDADNLMD@GetLocalLong@ 000000018002e138     StackFrameImpl.obj
 0002:00001148       ??_C@_0P@OMPFIIHN@SetLocalObject@ 000000018002e148     StackFrameImpl.obj
 0002:00001158       ??_C@_0M@OKLBLBFE@SetLocalInt@ 000000018002e158     StackFrameImpl.obj
 0002:00001168       ??_C@_0O@GMHJNNDF@SetLocalFloat@ 000000018002e168     StackFrameImpl.obj
 0002:00001178       ??_C@_0P@HFIOJDJO@SetLocalDouble@ 000000018002e178     StackFrameImpl.obj
 0002:00001188       ??_C@_0N@CHLNBHIP@SetLocalLong@ 000000018002e188     StackFrameImpl.obj
 0002:00001198       ??_C@_0BB@ECEEEFHG@GetFrameLocation@ 000000018002e198     StackFrameImpl.obj
 0002:000011b0       ??_C@_0L@GFPHAPCK@ThisObject@ 000000018002e1b0     StackFrameImpl.obj
 0002:000011c0       ??_C@_09MMMKHAHA@PopFrames@ 000000018002e1c0     StackFrameImpl.obj
 0002:000011d0       ??_C@_0L@JHEHPHFN@StackFrame@ 000000018002e1d0     StackFrameImpl.obj
 0002:000011e0       ??_C@_0EA@PLKIPJLM@s?2src?2jdk?4jdwp?4agent?2share?2nati@ 000000018002e1e0     StringReferenceImpl.obj
 0002:00001220       ??_C@_05LPIJGKJ@Value@     000000018002e220     StringReferenceImpl.obj
 0002:00001228       ??_C@_0BA@LONLIKLM@StringReference@ 000000018002e228     StringReferenceImpl.obj
 0002:00001240       ??_C@_0EF@COMLBEIJ@s?2src?2jdk?4jdwp?4agent?2share?2nati@ 000000018002e240     ThreadGroupReferenceImpl.obj
 0002:00001288       ??_C@_0BH@GAOLNFJO@GetThreadGroupChildren@ 000000018002e288     ThreadGroupReferenceImpl.obj
 0002:000012a0       ??_C@_04FABLJDN@Name@      000000018002e2a0     ThreadGroupReferenceImpl.obj
 0002:000012a8       ??_C@_06EBOPLIP@Parent@    000000018002e2a8     ThreadGroupReferenceImpl.obj
 0002:000012b0       ??_C@_08IEBJFPPC@Children@ 000000018002e2b0     ThreadGroupReferenceImpl.obj
 0002:000012c0       ??_C@_0BF@HMNGNKAP@ThreadGroupReference@ 000000018002e2c0     ThreadGroupReferenceImpl.obj
 0002:000012e0       ??_C@_0EA@KHLCDHFG@s?2src?2jdk?4jdwp?4agent?2share?2nati@ 000000018002e2e0     ThreadReferenceImpl.obj
 0002:00001320       ??_C@_0O@OMCINHIO@GetThreadInfo@ 000000018002e320     ThreadReferenceImpl.obj
 0002:00001330       ??_C@_0O@OMMMFPCB@GetFrameCount@ 000000018002e330     ThreadReferenceImpl.obj
 0002:00001340       ??_C@_0O@HJBPDPBL@GetStackTrace@ 000000018002e340     ThreadReferenceImpl.obj
 0002:00001350       ??_C@_0BE@CFHIFOK@GetOwnedMonitorInfo@ 000000018002e350     ThreadReferenceImpl.obj
 0002:00001368       ??_C@_0BL@FKMDJLON@GetCurrentContendedMonitor@ 000000018002e368     ThreadReferenceImpl.obj
 0002:00001388       ??_C@_0BO@KJEKJMBJ@GetOwnedMonitorStackDepthInfo@ 000000018002e388     ThreadReferenceImpl.obj
 0002:000013a8       ??_C@_0BH@OGPJNGCM@ForceEarlyReturnObject@ 000000018002e3a8     ThreadReferenceImpl.obj
 0002:000013c0       ??_C@_0BF@GFOCGLCB@ForceEarlyReturnVoid@ 000000018002e3c0     ThreadReferenceImpl.obj
 0002:000013d8       ??_C@_0BE@OOLJADPL@ForceEarlyReturnInt@ 000000018002e3d8     ThreadReferenceImpl.obj
 0002:000013f0       ??_C@_0BG@GAIJKLLL@ForceEarlyReturnFloat@ 000000018002e3f0     ThreadReferenceImpl.obj
 0002:00001408       ??_C@_0BH@HPICMNMP@ForceEarlyReturnDouble@ 000000018002e408     ThreadReferenceImpl.obj
 0002:00001420       ??_C@_0BF@GBNAKBEE@ForceEarlyReturnLong@ 000000018002e420     ThreadReferenceImpl.obj
 0002:00001438       ??_C@_0BA@PCKAHKK@IsVirtualThread@ 000000018002e438     ThreadReferenceImpl.obj
 0002:00001448       ??_C@_07MEGAPLCH@Suspend@  000000018002e448     ThreadReferenceImpl.obj
 0002:00001450       ??_C@_06DEPGELNG@Resume@   000000018002e450     ThreadReferenceImpl.obj
 0002:00001458       ??_C@_06PGDKHFME@Status@   000000018002e458     ThreadReferenceImpl.obj
 0002:00001460       ??_C@_0M@FJLPMLGA@ThreadGroup@ 000000018002e460     ThreadReferenceImpl.obj
 0002:0000146c       ??_C@_06CELCJONF@Frames@   000000018002e46c     ThreadReferenceImpl.obj
 0002:00001478       ??_C@_0O@CIBGJGLJ@OwnedMonitors@ 000000018002e478     ThreadReferenceImpl.obj
 0002:00001488       ??_C@_0BI@LNCBLBIG@CurrentContendedMonitor@ 000000018002e488     ThreadReferenceImpl.obj
 0002:000014a0       ??_C@_04MOIHHPNJ@Stop@     000000018002e4a0     ThreadReferenceImpl.obj
 0002:000014a8       ??_C@_09JNFEIGJE@Interrupt@ 000000018002e4a8     ThreadReferenceImpl.obj
 0002:000014b8       ??_C@_0N@CJCCJPA@SuspendCount@ 000000018002e4b8     ThreadReferenceImpl.obj
 0002:000014c8       ??_C@_0BM@FMMKDMLC@OwnedMonitorsWithStackDepth@ 000000018002e4c8     ThreadReferenceImpl.obj
 0002:000014e8       ??_C@_0BB@OENGDAPG@ForceEarlyReturn@ 000000018002e4e8     ThreadReferenceImpl.obj
 0002:00001500       ??_C@_09KMJHIIFD@IsVirtual@ 000000018002e500     ThreadReferenceImpl.obj
 0002:00001510       ??_C@_0BA@DDHJAEOJ@ThreadReference@ 000000018002e510     ThreadReferenceImpl.obj
 0002:00001520       ??_C@_0DE@JKJKNCJP@Java?5Debug?5Wire?5Protocol?5?$CIRefer@ 000000018002e520     VirtualMachineImpl.obj
 0002:00001558       ??_C@_09EEKGDCPH@?$DMunknown?$DO@ 000000018002e558     VirtualMachineImpl.obj
 0002:00001570       ??_C@_0EL@OEBGOINI@?$CFs?5version?5?$CFd?4?$CFd?6JVM?5Debug?5Inte@ 000000018002e570     VirtualMachineImpl.obj
 0002:000015c0       ??_C@_0DP@KCADHKOO@s?2src?2jdk?4jdwp?4agent?2share?2nati@ 000000018002e5c0     VirtualMachineImpl.obj
 0002:00001600       ??_C@_0O@OCFPKCI@GetAllModules@ 000000018002e600     VirtualMachineImpl.obj
 0002:00001610       ??_C@_0BA@DLNPNDDE@RedefineClasses@ 000000018002e610     VirtualMachineImpl.obj
 0002:00001620       ??_C@_0BD@GPIPONPL@GetTopThreadGroups@ 000000018002e620     VirtualMachineImpl.obj
 0002:00001638       ??_C@_09OOFGMMEJ@JNI_FALSE@ 000000018002e638     VirtualMachineImpl.obj
 0002:00001648       ??_C@_0N@PHJGBMEP@NewStringUTF@ 000000018002e648     VirtualMachineImpl.obj
 0002:00001658       ??_C@_01ICJEACDI@?$DL@     000000018002e658     VirtualMachineImpl.obj
 0002:00001660       ??_C@_07NGFJPNPN@Version@  000000018002e660     VirtualMachineImpl.obj
 0002:00001668       ??_C@_0BE@FBNAKJLP@ClassesForSignature@ 000000018002e668     VirtualMachineImpl.obj
 0002:00001680       ??_C@_0L@FHGIJHIB@AllClasses@ 000000018002e680     VirtualMachineImpl.obj
 0002:00001690       ??_C@_0O@OOLBCKEI@GetAllThreads@ 000000018002e690     VirtualMachineImpl.obj
 0002:000016a0       ??_C@_0BF@PLHJIAHK@TopLevelThreadGroups@ 000000018002e6a0     VirtualMachineImpl.obj
 0002:000016b8       ??_C@_07HADINEKJ@Dispose@  000000018002e6b8     VirtualMachineImpl.obj
 0002:000016c0       ??_C@_07EMPPKEFJ@IDSizes@  000000018002e6c0     VirtualMachineImpl.obj
 0002:000016c8       ??_C@_06BJLINPHD@DoExit@   000000018002e6c8     VirtualMachineImpl.obj
 0002:000016d0       ??_C@_0N@DNBIJONA@CreateString@ 000000018002e6d0     VirtualMachineImpl.obj
 0002:000016e0       ??_C@_0N@FNJCOOAL@Capabilities@ 000000018002e6e0     VirtualMachineImpl.obj
 0002:000016f0       ??_C@_0L@KKBJMNEN@ClassPaths@ 000000018002e6f0     VirtualMachineImpl.obj
 0002:00001700       ??_C@_0P@MLKCHAIH@DisposeObjects@ 000000018002e700     VirtualMachineImpl.obj
 0002:00001710       ??_C@_0L@CAGABDAD@HoldEvents@ 000000018002e710     VirtualMachineImpl.obj
 0002:00001720       ??_C@_0O@IOKPODIB@ReleaseEvents@ 000000018002e720     VirtualMachineImpl.obj
 0002:00001730       ??_C@_0BA@IHAAAKEC@CapabilitiesNew@ 000000018002e730     VirtualMachineImpl.obj
 0002:00001740       ??_C@_0BC@JBKLKNCM@SetDefaultStratum@ 000000018002e740     VirtualMachineImpl.obj
 0002:00001758       ??_C@_0BG@HDJCDLB@AllClassesWithGeneric@ 000000018002e758     VirtualMachineImpl.obj
 0002:00001770       ??_C@_0P@GBGAFJLK@InstanceCounts@ 000000018002e770     VirtualMachineImpl.obj
 0002:00001780       ??_C@_0L@KEPNLMPE@AllModules@ 000000018002e780     VirtualMachineImpl.obj
 0002:00001790       ??_C@_0P@PELBDMOO@VirtualMachine@ 000000018002e790     VirtualMachineImpl.obj
 0002:000017a0       ??_C@_0BJ@MKFEFELD@jvmti_env?5?$DN?$DN?5trackingEnv@ 000000018002e7a0     classTrack.obj
 0002:000017c0       ??_C@_0DH@GANKBOKD@s?2src?2jdk?4jdwp?4agent?2share?2nati@ 000000018002e7c0     classTrack.obj
 0002:000017f8       ??_C@_0O@PLBDFGGD@gdata?9?$DOvmDead@ 000000018002e7f8     classTrack.obj
 0002:00001808       ??_C@_09CMIIOJHF@signature@ 000000018002e808     classTrack.obj
 0002:00001814       ??_C@_06JAJCHHBC@GetTag@   000000018002e814     classTrack.obj
 0002:00001820       ??_C@_0CI@IMNMNLEM@Unable?5to?5GetTag?5with?5class?5tra@ 000000018002e820     classTrack.obj
 0002:00001848       ??_C@_0CF@IACJLELA@strcmp?$CIsignature?0?5oldSignature?$CJ@ 000000018002e848     classTrack.obj
 0002:00001870       ??_C@_06DADMPMP@SetTag@    000000018002e870     classTrack.obj
 0002:00001878       ??_C@_0BA@GDHIKEAF@AddCapabilities@ 000000018002e878     classTrack.obj
 0002:00001888       ??_C@_0BC@GAGPFDAP@SetEventCallbacks@ 000000018002e888     classTrack.obj
 0002:000018a0       ??_C@_0BJ@MAECPKFO@SetEventNotificationMode@ 000000018002e8a0     classTrack.obj
 0002:000018c0       ??_C@_0CJ@MPKHDCCL@Failed?5to?5allocate?5tag?9tracking@ 000000018002e8c0     classTrack.obj
 0002:000018f0       ??_C@_0CE@GIKHACIF@Unable?5to?5setup?5ObjectFree?5trac@ 000000018002e8f0     classTrack.obj
 0002:00001918       ??_C@_0BF@GLPPHCDA@loaded?5classes?5array@ 000000018002e918     classTrack.obj
 0002:00001930       ??_C@_0DG@IIIEKKMO@s?2src?2jdk?4jdwp?4agent?2share?2nati@ 000000018002e930     commonRef.obj
 0002:00001968       ??_C@_0N@IAAOLNMM@NewGlobalRef@ 000000018002e968     commonRef.obj
 0002:00001978       ??_C@_0BB@DFCJOKMO@NewWeakGlobalRef@ 000000018002e978     commonRef.obj
 0002:00001990       ??_C@_0BA@HLIPMHMF@DeleteGlobalRef@ 000000018002e990     commonRef.obj
 0002:000019a0       ??_C@_0BE@BJLAMKFM@DeleteWeakGlobalRef@ 000000018002e9a0     commonRef.obj
 0002:000019b8       ??_C@_0BB@EBIINFKL@Freeing?5?$CFd?5?$CI?$CFx?$CJ?6@ 000000018002e9b8     commonRef.obj
 0002:000019d0       ??_C@_0BC@GLNEFKOL@RefNode?5count?5?$DM?50@ 000000018002e9d0     commonRef.obj
 0002:000019e8       ??_C@_0BN@ODBCKJDJ@JDWP?5Reference?5Table?5Monitor@ 000000018002e9e8     commonRef.obj
 0002:00001a08       ??_C@_0M@GAIIKJOJ@NewLocalRef@ 000000018002ea08     commonRef.obj
 0002:00001a18       ??_C@_0P@DFLOMFLG@DeleteLocalRef@ 000000018002ea18     commonRef.obj
 0002:00001a28       ??_C@_0DK@LLCGDOIF@s?2src?2jdk?4jdwp?4agent?2share?2nati@ 000000018002ea28     debugDispatch.obj
 0002:00001a68       ??_C@_0BC@DMLDOBBC@command?5set?5array@ 000000018002ea68     debugDispatch.obj
 0002:00001a80       ??_C@_0BF@OACBGPIG@?$DMInvalid?5CommandSet?$DO@ 000000018002ea80     debugDispatch.obj
 0002:00001a98       ??_C@_0BC@HOMPDMML@?$DMUnknown?5Command?$DO@ 000000018002ea98     debugDispatch.obj
 0002:00001ab0       ??_C@_0BC@KIDCJOPK@?$DMInvalid?5Command?$DO@ 000000018002eab0     debugDispatch.obj
 0002:00001ac8       ??_C@_0DG@GNAHAJEF@s?2src?2jdk?4jdwp?4agent?2share?2nati@ 000000018002eac8     debugInit.obj
 0002:00001b00       ??_C@_0DI@HJHBDLDN@JDWP?5unable?5to?5configure?5initia@ 000000018002eb00     debugInit.obj
 0002:00001b40       ??_C@_0FO@EFFMOFEA@Cannot?5load?5this?5JVM?5TI?5agent?5t@ 000000018002eb40     debugInit.obj
 0002:00001ba0       ??_C@_0BN@FIGCDEN@JDWP?5unable?5to?5load?0?5VM?5died@ 000000018002eba0     debugInit.obj
 0002:00001bc0       ??_C@_03HPEPLPA@JVM@       000000018002ebc0     debugInit.obj
 0002:00001bc4       ??_C@_06CALCCDMF@GetEnv@   000000018002ebc4     debugInit.obj
 0002:00001bd0       ??_C@_0FE@FNGBOPAF@JDWP?5unable?5to?5access?5JVMTI?5Ver@ 000000018002ebd0     debugInit.obj
 0002:00001c30       ??_C@_0GO@FFEFEJNO@This?5jdwp?5native?5library?5will?5n@ 000000018002ec30     debugInit.obj
 0002:00001ca0       ??_C@_0L@GCOJPMGE@Onload?3?5?$CFs@ 000000018002eca0     debugInit.obj
 0002:00001cb0       ??_C@_0BJ@DAFNBFMC@GetPotentialCapabilities@ 000000018002ecb0     debugInit.obj
 0002:00001cd0       ??_C@_0DI@HGBENBDB@JDWP?5unable?5to?5get?5potential?5JV@ 000000018002ecd0     debugInit.obj
 0002:00001d08       ??_C@_0DB@KIBJMMBD@JDWP?5unable?5to?5get?5necessary?5JV@ 000000018002ed08     debugInit.obj
 0002:00001d40       ??_C@_0DB@FLBLFKJC@JDWP?5unable?5to?5set?5JVMTI?5event?5@ 000000018002ed40     debugInit.obj
 0002:00001d78       ??_C@_0N@NKKDPPME@OnLoad?3?5DONE@ 000000018002ed78     debugInit.obj
 0002:00001d88       ??_C@_02LACNDIPD@CB@       000000018002ed88     debugInit.obj
 0002:00001d90       ??_C@_0O@DLFFEAD@cbEarlyVMInit@ 000000018002ed90     debugInit.obj
 0002:00001da0       ??_C@_0BI@BCONGKCA@VM?5dead?5at?5VM_INIT?5time@ 000000018002eda0     debugInit.obj
 0002:00001db8       ??_C@_0BC@IFIKOKIP@END?5cbEarlyVMInit@ 000000018002edb8     debugInit.obj
 0002:00001dd0       ??_C@_0BD@IBLDMNIE@DisposeEnvironment@ 000000018002edd0     debugInit.obj
 0002:00001de8       ??_C@_0DE@BOJEJHME@JDWP?5unable?5to?5dispose?5of?5JVMTI@ 000000018002ede8     debugInit.obj
 0002:00001e20       ??_C@_0P@DKNEAPGB@cbEarlyVMDeath@ 000000018002ee20     debugInit.obj
 0002:00001e30       ??_C@_0BH@MJOFBADO@VM?5died?5more?5than?5once@ 000000018002ee30     debugInit.obj
 0002:00001e48       ??_C@_0BD@NOFMPPNE@END?5cbEarlyVMDeath@ 000000018002ee48     debugInit.obj
 0002:00001e60       ??_C@_0BM@IEEFFE@cbEarlyException?3?5thread?$DN?$CFp@ 000000018002ee60     debugInit.obj
 0002:00001e80       ??_C@_0CD@LICFEBIC@VM?5dead?5at?5initial?5Exception?5ev@ 000000018002ee80     debugInit.obj
 0002:00001ea8       ??_C@_0BK@LELFCHPE@VM?5is?5not?5initialized?5yet@ 000000018002eea8     debugInit.obj
 0002:00001ec8       ??_C@_0BC@LPILBKGC@ExceptionOccurred@ 000000018002eec8     debugInit.obj
 0002:00001ee0       ??_C@_0CD@IFKJAMDD@Initializing?5on?5uncaught?5except@ 000000018002eee0     debugInit.obj
 0002:00001f08       ??_C@_0DE@NBANCLO@Checking?5specific?5exception?3?5lo@ 000000018002ef08     debugInit.obj
 0002:00001f40       ??_C@_0CD@DGOBNBPB@Initializing?5on?5specific?5except@ 000000018002ef40     debugInit.obj
 0002:00001f68       ??_C@_0CP@DAAMLOKM@No?5initialization?0?5didn?8t?5find?5@ 000000018002ef68     debugInit.obj
 0002:00001f98       ??_C@_05JCKDCDAK@Throw@    000000018002ef98     debugInit.obj
 0002:00001fa0       ??_C@_0BF@FLBJJJJM@END?5cbEarlyException@ 000000018002efa0     debugInit.obj
 0002:00001fb8       ??_C@_0BF@KCLMNAFK@Begin?5startTransport@ 000000018002efb8     debugInit.obj
 0002:00001fd0       ??_C@_0CP@GLCNJPPL@JDWP?5Transport?5?$CFs?5failed?5to?5ini@ 000000018002efd0     debugInit.obj
 0002:00002000       ??_C@_0BD@KMCJBFOI@End?5startTransport@ 000000018002f000     debugInit.obj
 0002:00002018       ??_C@_0BP@HFGABHKC@signal?5initialization?5complete@ 000000018002f018     debugInit.obj
 0002:00002038       ??_C@_0P@CPJAJOGP@UNKNOWN?5REASON@ 000000018002f038     debugInit.obj
 0002:00002048       ??_C@_0BL@EEDFKGOH@JDWP?5?$CFs?0?5jvmtiError?$DN?$CFs?$CI?$CFd?$CJ@ 000000018002f048     debugInit.obj
 0002:00002068       ??_C@_07CBPKFJFN@JDWP?5?$CFs@ 000000018002f068     debugInit.obj
 0002:00002070       ??_C@_0CG@MHFIMNKE@Can?8t?5call?5JNI?5FatalError?$CINULL?0@ 000000018002f070     debugInit.obj
 0002:00002098       ??_C@_0O@GBAEPAJL@ERROR?3?5JDWP?3?5@ 000000018002f098     debugInit.obj
 0002:000020a8       ??_C@_0BD@BEMOICGG@Begin?5initialize?$CI?$CJ@ 000000018002f0a8     debugInit.obj
 0002:000020c0       ??_C@_0BN@NHJNNMLF@VM?5dead?5at?5initialize?$CI?$CJ?5time@ 000000018002f0c0     debugInit.obj
 0002:000020e0       ??_C@_0CL@FOADKMNE@unable?5to?5disable?5JVMTI?5event?5n@ 000000018002f0e0     debugInit.obj
 0002:00002110       ??_C@_0CA@LEEFBLBH@unable?5to?5clear?5JVMTI?5callbacks@ 000000018002f110     debugInit.obj
 0002:00002130       ??_C@_0BM@GGAMJPIA@JDWP?5Initialization?5Monitor@ 000000018002f130     debugInit.obj
 0002:00002150       ??_C@_0BK@MDFDHGIG@No?5transports?5initialized@ 000000018002f150     debugInit.obj
 0002:00002170       ??_C@_0BM@IHKNNPNA@triggering_ei?5?$DN?$DN?5EI_VM_INIT@ 000000018002f170     debugInit.obj
 0002:00002190       ??_C@_0BO@EHMNOJNO@triggering_ei?5?$DN?$DN?5EI_EXCEPTION@ 000000018002f190     debugInit.obj
 0002:000021b0       ??_C@_0BB@DGEPDJNI@opt_info?5?$CB?$DN?5NULL@ 000000018002f1b0     debugInit.obj
 0002:000021c8       ??_C@_0CG@FBKKPEEO@VM?5dead?5before?5initialize?$CI?$CJ?5com@ 000000018002f1c8     debugInit.obj
 0002:000021f0       ??_C@_0BB@FNMNNOIE@End?5initialize?$CI?$CJ@ 000000018002f1f0     debugInit.obj
 0002:00002208       ??_C@_0BM@DDGJDKIN@debugInit_reset?$CI?$CJ?5beginning@ 000000018002f208     debugInit.obj
 0002:00002228       ??_C@_0BN@ICEPLJN@debugInit_reset?$CI?$CJ?5completed?4@ 000000018002f228     debugInit.obj
 0002:00002250       ??_C@_0GGE@OGKDMPPH@?5?5?5?5?5?5?5?5?5?5?5?5?5?5?5Java?5Debugger?5JD@ 000000018002f250     debugInit.obj
 0002:000028c0       ??_C@_0CEF@LOIFLEGE@Obsolete?5Options?6?9?9?9?9?9?9?9?9?9?9?9?9?9?9@ 000000018002f8c0     debugInit.obj
 0002:00002b10       ??_C@_0GE@PNCPNOJL@JDWP?5Non?9server?5transport?5?$CFs?5mu@ 000000018002fb10     debugInit.obj
 0002:00002b74       ??_C@_01IHBHIGKO@?0@       000000018002fb74     debugInit.obj
 0002:00002b78       ??_C@_01EANLCPLP@y@        000000018002fb78     debugInit.obj
 0002:00002b7c       ??_C@_01EFFIKLCJ@n@        000000018002fb7c     debugInit.obj
 0002:00002b80       ??_C@_04PCJFHION@help@     000000018002fb80     debugInit.obj
 0002:00002b88       ??_C@_0BD@BLCBAGAJ@_JAVA_JDWP_OPTIONS@ 000000018002fb88     debugInit.obj
 0002:00002ba0       ??_C@_07FOPBDDAL@options@  000000018002fba0     debugInit.obj
 0002:00002ba8       ??_C@_0L@PNFKLIOM@transports@ 000000018002fba8     debugInit.obj
 0002:00002bb8       ??_C@_09PBENLGJM@transport@ 000000018002fbb8     debugInit.obj
 0002:00002bc8       ??_C@_07LHEPONKL@address@  000000018002fbc8     debugInit.obj
 0002:00002bd0       ??_C@_0CE@KJBCDAKG@address?5specified?5without?5trans@ 000000018002fbd0     debugInit.obj
 0002:00002bf4       ??_C@_05IDFCDDHI@allow@    000000018002fbf4     debugInit.obj
 0002:00002c00       ??_C@_0CC@DKFOJBDD@allow?5specified?5without?5transpo@ 000000018002fc00     debugInit.obj
 0002:00002c28       ??_C@_07DDHNKDGP@timeout@  000000018002fc28     debugInit.obj
 0002:00002c30       ??_C@_0CE@KCGGPGKE@timeout?5specified?5without?5trans@ 000000018002fc30     debugInit.obj
 0002:00002c58       ??_C@_0BG@NBOGMFLN@includevirtualthreads@ 000000018002fc58     debugInit.obj
 0002:00002c70       ??_C@_06OAFDKBLG@launch@   000000018002fc70     debugInit.obj
 0002:00002c78       ??_C@_07JDKNNNFJ@onthrow@  000000018002fc78     debugInit.obj
 0002:00002c80       ??_C@_06GMEIIFFN@assert@   000000018002fc80     debugInit.obj
 0002:00002c88       ??_C@_05FAMCFOJB@fatal@    000000018002fc88     debugInit.obj
 0002:00002c90       ??_C@_05PDJBBECF@pause@    000000018002fc90     debugInit.obj
 0002:00002c98       ??_C@_08IANEBDLN@datadump@ 000000018002fc98     debugInit.obj
 0002:00002ca8       ??_C@_08JHOBLGK@coredump@  000000018002fca8     debugInit.obj
 0002:00002cb8       ??_C@_09NDIDIJNG@errorexit@ 000000018002fcb8     debugInit.obj
 0002:00002cc8       ??_C@_09KOPDMKB@exitpause@ 000000018002fcc8     debugInit.obj
 0002:00002cd8       ??_C@_0CO@FJOJNBJC@The?5exitpause?5option?5removed?0?5u@ 000000018002fcd8     debugInit.obj
 0002:00002d08       ??_C@_08KLNFLELA@precrash@ 000000018002fd08     debugInit.obj
 0002:00002d18       ??_C@_0CN@FJOGMEJD@The?5precrash?5option?5removed?0?5us@ 000000018002fd18     debugInit.obj
 0002:00002d48       ??_C@_07HMINABEO@logfile@  000000018002fd48     debugInit.obj
 0002:00002d50       ??_C@_08KMAEEIGA@logflags@ 000000018002fd50     debugInit.obj
 0002:00002d60       ??_C@_0L@NDPADBNN@debugflags@ 000000018002fd60     debugInit.obj
 0002:00002d70       ??_C@_07DNBGJJHB@suspend@  000000018002fd70     debugInit.obj
 0002:00002d78       ??_C@_06HJHJCKIO@server@   000000018002fd78     debugInit.obj
 0002:00002d80       ??_C@_06OLFOGHEN@strict@   000000018002fd80     debugInit.obj
 0002:00002d88       ??_C@_05PMBAOCDH@quiet@    000000018002fd88     debugInit.obj
 0002:00002d90       ??_C@_0L@EINCANF@onuncaught@ 000000018002fd90     debugInit.obj
 0002:00002d9c       ??_C@_05HEPNBBMF@mutf8@    000000018002fd9c     debugInit.obj
 0002:00002da8       ??_C@_08GEPKFJKM@stdalloc@ 000000018002fda8     debugInit.obj
 0002:00002db8       ??_C@_0BH@HHOMGJCA@no?5transport?5specified@ 000000018002fdb8     debugInit.obj
 0002:00002dd0       ??_C@_0DG@LFMJLIEN@multiple?5transports?5are?5not?5sup@ 000000018002fdd0     debugInit.obj
 0002:00002e10       ??_C@_0EJ@JJILEHOC@Specify?5launch?$DN?$DMcommand?5line?$DO?5w@ 000000018002fe10     debugInit.obj
 0002:00002e60       ??_C@_0P@KGDIDJKL@?9agentlib?3jdwp@ 000000018002fe60     debugInit.obj
 0002:00002e70       ??_C@_0CA@PBEIFGCB@JDWP?5option?5syntax?5error?3?5?$CFs?$DN?$CFs@ 000000018002fe70     debugInit.obj
 0002:00002e90       ??_C@_0P@HJPPKHBO@JDWP?5?$CFs?3?5?$CFs?$DN?$CFs@ 000000018002fe90     debugInit.obj
 0002:00002ea0       ??_C@_0P@PJFAGLMH@invalid?5option@ 000000018002fea0     debugInit.obj
 0002:00002eb0       ??_C@_0BO@EGHMLMKO@Exiting?5with?5error?5?$CFs?$CI?$CFd?$CJ?3?5?$CFs@ 000000018002feb0     debugInit.obj
 0002:00002ed0       ??_C@_0CK@CLPEKKDE@Dumping?5core?5as?5requested?5by?5co@ 000000018002fed0     debugInit.obj
 0002:00002f00       ??_C@_0BD@KBEAEDMA@JDWP?5VM_DEATH?5Lock@ 000000018002ff00     debugLoop.obj
 0002:00002f18       ??_C@_0BI@KEHBCJBK@JDWP?5Command?5Queue?5Lock@ 000000018002ff18     debugLoop.obj
 0002:00002f30       ??_C@_0BE@OJJPFMMB@JDWP?5Command?5Reader@ 000000018002ff30     debugLoop.obj
 0002:00002f48       ??_C@_0DG@PEEBJHLA@s?2src?2jdk?4jdwp?4agent?2share?2nati@ 000000018002ff48     debugLoop.obj
 0002:00002f80       ??_C@_0CD@BCFANGIM@Command?5set?5?$CFs?$CI?$CFd?$CJ?0?5command?5?$CFs?$CI@ 000000018002ff80     debugLoop.obj
 0002:00002fa8       ??_C@_0BE@LPIOKOFH@Begin?5reader?5thread@ 000000018002ffa8     debugLoop.obj
 0002:00002fc0       ??_C@_0FI@EMFENIBI@Received?5jdwpPacket?5with?5flags?5@ 000000018002ffc0     debugLoop.obj
 0002:00003018       ??_C@_0BC@PBMDCOFP@End?5reader?5thread@ 0000000180030018     debugLoop.obj
 0002:00003030       ??_C@_0M@FFFEEGHJ@packet?5list@ 0000000180030030     debugLoop.obj
 0002:0000303c       ??_C@_06DIJPEION@?$CFs?$CFs?$CFs@ 000000018003003c     error_messages.obj
 0002:00003048       ??_C@_07JHDPBCI@ERROR?3?5@ 0000000180030048     error_messages.obj
 0002:00003050       ??_C@_0DL@OBDMDFEC@s?2src?2jdk?4jdwp?4agent?2share?2nati@ 0000000180030050     error_messages.obj
 0002:00003090       ??_C@_0BN@HFAPOECE@Requested?5errorexit?$DNy?5exit?$CI?$CJ@ 0000000180030090     error_messages.obj
 0002:000030b0       ??_C@_0BN@BNMAOKIE@ASSERT?5FAILED?3?5?$CFs?5?3?5?$CFd?5?9?5?$CFs?6@ 00000001800300b0     error_messages.obj
 0002:000030d0       ??_C@_0N@BMIGOGFN@?$CFs?5?3?5?$CFd?5?9?5?$CFs@ 00000001800300d0     error_messages.obj
 0002:000030e0       ??_C@_0BA@HJKPOGGF@ASSERT?5FAILED?3?5@ 00000001800300e0     error_messages.obj
 0002:000030f0       ??_C@_0BB@NAGLCMLI@Assertion?5Failed@ 00000001800300f0     error_messages.obj
 0002:00003108       ??_C@_0BB@JCNMKLLK@JVMTI_ERROR_NONE@ 0000000180030108     error_messages.obj
 0002:00003120       ??_C@_0BL@LDIMKLPH@JVMTI_ERROR_INVALID_THREAD@ 0000000180030120     error_messages.obj
 0002:00003140       ??_C@_0CB@PJFPAIKJ@JVMTI_ERROR_INVALID_THREAD_GROU@ 0000000180030140     error_messages.obj
 0002:00003168       ??_C@_0BN@LLMKHMNF@JVMTI_ERROR_INVALID_PRIORITY@ 0000000180030168     error_messages.obj
 0002:00003188       ??_C@_0CB@MBOFKAGB@JVMTI_ERROR_THREAD_NOT_SUSPENDE@ 0000000180030188     error_messages.obj
 0002:000031b0       ??_C@_0BN@FABOLPBI@JVMTI_ERROR_THREAD_SUSPENDED@ 00000001800301b0     error_messages.obj
 0002:000031d0       ??_C@_0BN@FDGNOBJM@JVMTI_ERROR_THREAD_NOT_ALIVE@ 00000001800301d0     error_messages.obj
 0002:000031f0       ??_C@_0BL@GOBIFKNJ@JVMTI_ERROR_INVALID_OBJECT@ 00000001800301f0     error_messages.obj
 0002:00003210       ??_C@_0BK@FCMAJPPC@JVMTI_ERROR_INVALID_CLASS@ 0000000180030210     error_messages.obj
 0002:00003230       ??_C@_0BP@IKLLBKEB@JVMTI_ERROR_CLASS_NOT_PREPARED@ 0000000180030230     error_messages.obj
 0002:00003250       ??_C@_0BN@KLPPLKG@JVMTI_ERROR_INVALID_METHODID@ 0000000180030250     error_messages.obj
 0002:00003270       ??_C@_0BN@BCEKOKND@JVMTI_ERROR_INVALID_LOCATION@ 0000000180030270     error_messages.obj
 0002:00003290       ??_C@_0BM@DFDGPME@JVMTI_ERROR_INVALID_FIELDID@ 0000000180030290     error_messages.obj
 0002:000032b0       ??_C@_0BL@NELIEPEC@JVMTI_ERROR_NO_MORE_FRAMES@ 00000001800302b0     error_messages.obj
 0002:000032d0       ??_C@_0BJ@BDBECFDM@JVMTI_ERROR_OPAQUE_FRAME@ 00000001800302d0     error_messages.obj
 0002:000032f0       ??_C@_0BK@MIIFNLOB@JVMTI_ERROR_TYPE_MISMATCH@ 00000001800302f0     error_messages.obj
 0002:00003310       ??_C@_0BJ@HPCAOILC@JVMTI_ERROR_INVALID_SLOT@ 0000000180030310     error_messages.obj
 0002:00003330       ??_C@_0BG@CHILOPNI@JVMTI_ERROR_DUPLICATE@ 0000000180030330     error_messages.obj
 0002:00003348       ??_C@_0BG@DIEMLHKM@JVMTI_ERROR_NOT_FOUND@ 0000000180030348     error_messages.obj
 0002:00003360       ??_C@_0BM@NHMCKHOB@JVMTI_ERROR_INVALID_MONITOR@ 0000000180030360     error_messages.obj
 0002:00003380       ??_C@_0BO@PPEDAJGL@JVMTI_ERROR_NOT_MONITOR_OWNER@ 0000000180030380     error_messages.obj
 0002:000033a0       ??_C@_0BG@FCAIPEID@JVMTI_ERROR_INTERRUPT@ 00000001800303a0     error_messages.obj
 0002:000033b8       ??_C@_0CB@EGDBNKOI@JVMTI_ERROR_INVALID_CLASS_FORMA@ 00000001800303b8     error_messages.obj
 0002:000033e0       ??_C@_0CG@DGKOGIAL@JVMTI_ERROR_CIRCULAR_CLASS_DEFI@ 00000001800303e0     error_messages.obj
 0002:00003408       ??_C@_0BP@ICEALPKC@JVMTI_ERROR_FAILS_VERIFICATION@ 0000000180030408     error_messages.obj
 0002:00003428       ??_C@_0DC@JDACLMIO@JVMTI_ERROR_UNSUPPORTED_REDEFIN@ 0000000180030428     error_messages.obj
 0002:00003460       ??_C@_0DE@GKDKNOMJ@JVMTI_ERROR_UNSUPPORTED_REDEFIN@ 0000000180030460     error_messages.obj
 0002:00003498       ??_C@_0BO@LAFKIOG@JVMTI_ERROR_INVALID_TYPESTATE@ 0000000180030498     error_messages.obj
 0002:000034b8       ??_C@_0DH@INDGCLLB@JVMTI_ERROR_UNSUPPORTED_REDEFIN@ 00000001800304b8     error_messages.obj
 0002:000034f0       ??_C@_0DE@NHEOMMGI@JVMTI_ERROR_UNSUPPORTED_REDEFIN@ 00000001800304f0     error_messages.obj
 0002:00003528       ??_C@_0CA@EKPNJOEP@JVMTI_ERROR_UNSUPPORTED_VERSION@ 0000000180030528     error_messages.obj
 0002:00003548       ??_C@_0BN@OFFMAHHL@JVMTI_ERROR_NAMES_DONT_MATCH@ 0000000180030548     error_messages.obj
 0002:00003568       ??_C@_0DN@HHBBLAKE@JVMTI_ERROR_UNSUPPORTED_REDEFIN@ 0000000180030568     error_messages.obj
 0002:000035a8       ??_C@_0DO@HMBGBGNA@JVMTI_ERROR_UNSUPPORTED_REDEFIN@ 00000001800305a8     error_messages.obj
 0002:000035e8       ??_C@_0DN@MKMCJOKD@JVMTI_ERROR_UNSUPPORTED_REDEFIN@ 00000001800305e8     error_messages.obj
 0002:00003628       ??_C@_0CC@PODLINNP@JVMTI_ERROR_UNSUPPORTED_OPERATI@ 0000000180030628     error_messages.obj
 0002:00003650       ??_C@_0BK@CANILEHF@JVMTI_ERROR_NOT_AVAILABLE@ 0000000180030650     error_messages.obj
 0002:00003670       ??_C@_0CE@INJKMEFK@JVMTI_ERROR_MUST_POSSESS_CAPABI@ 0000000180030670     error_messages.obj
 0002:00003698       ??_C@_0BJ@LBFPFPDM@JVMTI_ERROR_NULL_POINTER@ 0000000180030698     error_messages.obj
 0002:000036b8       ??_C@_0BP@CHJPNNEM@JVMTI_ERROR_ABSENT_INFORMATION@ 00000001800306b8     error_messages.obj
 0002:000036d8       ??_C@_0BP@OMFMNLC@JVMTI_ERROR_INVALID_EVENT_TYPE@ 00000001800306d8     error_messages.obj
 0002:000036f8       ??_C@_0BN@BIBNPHHO@JVMTI_ERROR_ILLEGAL_ARGUMENT@ 00000001800306f8     error_messages.obj
 0002:00003718       ??_C@_0BK@PMKCFHAE@JVMTI_ERROR_OUT_OF_MEMORY@ 0000000180030718     error_messages.obj
 0002:00003738       ??_C@_0BK@NNJBDMNB@JVMTI_ERROR_ACCESS_DENIED@ 0000000180030738     error_messages.obj
 0002:00003758       ??_C@_0BI@GHECLMNC@JVMTI_ERROR_WRONG_PHASE@ 0000000180030758     error_messages.obj
 0002:00003770       ??_C@_0BF@OLIHJOII@JVMTI_ERROR_INTERNAL@ 0000000180030770     error_messages.obj
 0002:00003788       ??_C@_0BO@EOHGKJHI@JVMTI_ERROR_UNATTACHED_THREAD@ 0000000180030788     error_messages.obj
 0002:000037a8       ??_C@_0CA@LKHFDACL@JVMTI_ERROR_INVALID_ENVIRONMENT@ 00000001800307a8     error_messages.obj
 0002:000037c8       ??_C@_0BF@KCDLAD@AGENT_ERROR_INTERNAL@ 00000001800307c8     error_messages.obj
 0002:000037e0       ??_C@_0BE@KFGADCIM@AGENT_ERROR_VM_DEAD@ 00000001800307e0     error_messages.obj
 0002:000037f8       ??_C@_0BH@IOOMLCPK@AGENT_ERROR_NO_JNI_ENV@ 00000001800307f8     error_messages.obj
 0002:00003810       ??_C@_0BK@OHNBOEAB@AGENT_ERROR_JNI_EXCEPTION@ 0000000180030810     error_messages.obj
 0002:00003830       ??_C@_0BL@HHHLGBCJ@AGENT_ERROR_JVMTI_INTERNAL@ 0000000180030830     error_messages.obj
 0002:00003850       ??_C@_0BK@DOAJMAC@AGENT_ERROR_JDWP_INTERNAL@ 0000000180030850     error_messages.obj
 0002:00003870       ??_C@_0BO@HMIKBJDH@AGENT_ERROR_NOT_CURRENT_FRAME@ 0000000180030870     error_messages.obj
 0002:00003890       ??_C@_0BK@MDCNJBJM@AGENT_ERROR_OUT_OF_MEMORY@ 0000000180030890     error_messages.obj
 0002:000038b0       ??_C@_0BI@OCBNFCC@AGENT_ERROR_INVALID_TAG@ 00000001800308b0     error_messages.obj
 0002:000038c8       ??_C@_0BN@PEANMDOB@AGENT_ERROR_ALREADY_INVOKING@ 00000001800308c8     error_messages.obj
 0002:000038e8       ??_C@_0BK@HKJFNPFH@AGENT_ERROR_INVALID_INDEX@ 00000001800308e8     error_messages.obj
 0002:00003908       ??_C@_0BL@BMIJGCKP@AGENT_ERROR_INVALID_LENGTH@ 0000000180030908     error_messages.obj
 0002:00003928       ??_C@_0BL@JGHDGIGP@AGENT_ERROR_INVALID_STRING@ 0000000180030928     error_messages.obj
 0002:00003948       ??_C@_0CB@GJDCCCGC@AGENT_ERROR_INVALID_CLASS_LOADE@ 0000000180030948     error_messages.obj
 0002:00003970       ??_C@_0BK@FILGLGGH@AGENT_ERROR_INVALID_ARRAY@ 0000000180030970     error_messages.obj
 0002:00003990       ??_C@_0BL@FDPHKKDB@AGENT_ERROR_TRANSPORT_LOAD@ 0000000180030990     error_messages.obj
 0002:000039b0       ??_C@_0BL@GHHKABMN@AGENT_ERROR_TRANSPORT_INIT@ 00000001800309b0     error_messages.obj
 0002:000039d0       ??_C@_0BK@JFFMLFLM@AGENT_ERROR_NATIVE_METHOD@ 00000001800309d0     error_messages.obj
 0002:000039f0       ??_C@_0BK@KOCLEFJG@AGENT_ERROR_INVALID_COUNT@ 00000001800309f0     error_messages.obj
 0002:00003a10       ??_C@_0BM@LDFIPDCL@AGENT_ERROR_INVALID_FRAMEID@ 0000000180030a10     error_messages.obj
 0002:00003a30       ??_C@_0BJ@ILJPBKJK@AGENT_ERROR_NULL_POINTER@ 0000000180030a30     error_messages.obj
 0002:00003a50       ??_C@_0BN@LLKPAHA@AGENT_ERROR_ILLEGAL_ARGUMENT@ 0000000180030a50     error_messages.obj
 0002:00003a70       ??_C@_0BL@ENGHDPEH@AGENT_ERROR_INVALID_THREAD@ 0000000180030a70     error_messages.obj
 0002:00003a90       ??_C@_0BP@OCCGGDI@AGENT_ERROR_INVALID_EVENT_TYPE@ 0000000180030a90     error_messages.obj
 0002:00003ab0       ??_C@_0BL@JAPDMOGJ@AGENT_ERROR_INVALID_OBJECT@ 0000000180030ab0     error_messages.obj
 0002:00003ad0       ??_C@_0BL@CKFDNLPC@AGENT_ERROR_NO_MORE_FRAMES@ 0000000180030ad0     error_messages.obj
 0002:00003af0       ??_C@_0O@LFPPCNKG@ERROR_unknown@ 0000000180030af0     error_messages.obj
 0002:00003b00       ??_C@_0P@KOMKCNJP@EI_SINGLE_STEP@ 0000000180030b00     error_messages.obj
 0002:00003b10       ??_C@_0O@PLAPKDL@EI_BREAKPOINT@ 0000000180030b10     error_messages.obj
 0002:00003b20       ??_C@_0N@PGOIKMFF@EI_FRAME_POP@ 0000000180030b20     error_messages.obj
 0002:00003b30       ??_C@_0N@CEKAFBCB@EI_EXCEPTION@ 0000000180030b30     error_messages.obj
 0002:00003b40       ??_C@_0BA@EJAFLEFO@EI_THREAD_START@ 0000000180030b40     error_messages.obj
 0002:00003b50       ??_C@_0O@GJFHOBHI@EI_THREAD_END@ 0000000180030b50     error_messages.obj
 0002:00003b60       ??_C@_0BB@FOCFHABH@EI_CLASS_PREPARE@ 0000000180030b60     error_messages.obj
 0002:00003b78       ??_C@_0BA@MCOBNBEP@EI_CLASS_UNLOAD@ 0000000180030b78     error_messages.obj
 0002:00003b88       ??_C@_0O@BCBJODOG@EI_CLASS_LOAD@ 0000000180030b88     error_messages.obj
 0002:00003b98       ??_C@_0BA@DBHDLMCN@EI_FIELD_ACCESS@ 0000000180030b98     error_messages.obj
 0002:00003ba8       ??_C@_0BG@BKOJDIGF@EI_FIELD_MODIFICATION@ 0000000180030ba8     error_messages.obj
 0002:00003bc0       ??_C@_0BD@IMHNDJNF@EI_EXCEPTION_CATCH@ 0000000180030bc0     error_messages.obj
 0002:00003bd8       ??_C@_0BA@BMAHDEKG@EI_METHOD_ENTRY@ 0000000180030bd8     error_messages.obj
 0002:00003be8       ??_C@_0P@EODELCOH@EI_METHOD_EXIT@ 0000000180030be8     error_messages.obj
 0002:00003bf8       ??_C@_0L@DINKDGIA@EI_VM_INIT@ 0000000180030bf8     error_messages.obj
 0002:00003c08       ??_C@_0M@NLNKJGDL@EI_VM_DEATH@ 0000000180030c08     error_messages.obj
 0002:00003c18       ??_C@_0BI@IBKICKHP@EI_VIRTUAL_THREAD_START@ 0000000180030c18     error_messages.obj
 0002:00003c30       ??_C@_0BG@MMKMHLPD@EI_VIRTUAL_THREAD_END@ 0000000180030c30     error_messages.obj
 0002:00003c48       ??_C@_0O@MBFGOMME@EVENT_unknown@ 0000000180030c48     error_messages.obj
 0002:00003c58       ??_C@_04OKGDLNCL@NONE@     0000000180030c58     error_messages.obj
 0002:00003c60       ??_C@_0P@JCGOCJJM@INVALID_THREAD@ 0000000180030c60     error_messages.obj
 0002:00003c70       ??_C@_0BF@BFLDLBKG@INVALID_THREAD_GROUP@ 0000000180030c70     error_messages.obj
 0002:00003c88       ??_C@_0BB@DOHFANFH@INVALID_PRIORITY@ 0000000180030c88     error_messages.obj
 0002:00003ca0       ??_C@_0BF@CNAJBJGO@THREAD_NOT_SUSPENDED@ 0000000180030ca0     error_messages.obj
 0002:00003cb8       ??_C@_0BB@NFKBMOJK@THREAD_SUSPENDED@ 0000000180030cb8     error_messages.obj
 0002:00003cd0       ??_C@_0P@EPPKNILC@INVALID_OBJECT@ 0000000180030cd0     error_messages.obj
 0002:00003ce0       ??_C@_0O@ELGEBMG@INVALID_CLASS@ 0000000180030ce0     error_messages.obj
 0002:00003cf0       ??_C@_0BD@KEAMCEJN@CLASS_NOT_PREPARED@ 0000000180030cf0     error_messages.obj
 0002:00003d08       ??_C@_0BB@IPAAIKCE@INVALID_METHODID@ 0000000180030d08     error_messages.obj
 0002:00003d20       ??_C@_0BB@JHPFJLFB@INVALID_LOCATION@ 0000000180030d20     error_messages.obj
 0002:00003d38       ??_C@_0BA@NJBCDFJG@INVALID_FIELDID@ 0000000180030d38     error_messages.obj
 0002:00003d48       ??_C@_0BA@KCIGPBGB@INVALID_FRAMEID@ 0000000180030d48     error_messages.obj
 0002:00003d58       ??_C@_0P@PFFKMNCJ@NO_MORE_FRAMES@ 0000000180030d58     error_messages.obj
 0002:00003d68       ??_C@_0N@NGAODCAJ@OPAQUE_FRAME@ 0000000180030d68     error_messages.obj
 0002:00003d78       ??_C@_0BC@JIBCMOEK@NOT_CURRENT_FRAME@ 0000000180030d78     error_messages.obj
 0002:00003d90       ??_C@_0O@JOPDAFNF@TYPE_MISMATCH@ 0000000180030d90     error_messages.obj
 0002:00003da0       ??_C@_0N@LKDKPPIH@INVALID_SLOT@ 0000000180030da0     error_messages.obj
 0002:00003db0       ??_C@_09JHHLKDOI@DUPLICATE@ 0000000180030db0     error_messages.obj
 0002:00003dc0       ??_C@_09IILMPLJM@NOT_FOUND@ 0000000180030dc0     error_messages.obj
 0002:00003dd0       ??_C@_0BA@NIDPNLD@INVALID_MONITOR@ 0000000180030dd0     error_messages.obj
 0002:00003de0       ??_C@_0BC@PMHAFEBG@NOT_MONITOR_OWNER@ 0000000180030de0     error_messages.obj
 0002:00003df8       ??_C@_09OCPILILD@INTERRUPT@ 0000000180030df8     error_messages.obj
 0002:00003e08       ??_C@_0BF@KKNNGDOH@INVALID_CLASS_FORMAT@ 0000000180030e08     error_messages.obj
 0002:00003e20       ??_C@_0BK@IGLHGLOO@CIRCULAR_CLASS_DEFINITION@ 0000000180030e20     error_messages.obj
 0002:00003e40       ??_C@_0BD@KMPHIBHO@FAILS_VERIFICATION@ 0000000180030e40     error_messages.obj
 0002:00003e58       ??_C@_0BL@PPBPAAJH@ADD_METHOD_NOT_IMPLEMENTED@ 0000000180030e58     error_messages.obj
 0002:00003e78       ??_C@_0BO@EMGJAAKO@SCHEMA_CHANGE_NOT_IMPLEMENTED@ 0000000180030e78     error_messages.obj
 0002:00003e98       ??_C@_0BC@IDGPFJL@INVALID_TYPESTATE@ 0000000180030e98     error_messages.obj
 0002:00003eb0       ??_C@_0CB@DMMJDFBN@HIERARCHY_CHANGE_NOT_IMPLEMENTE@ 0000000180030eb0     error_messages.obj
 0002:00003ed8       ??_C@_0BO@EGGEGIDF@DELETE_METHOD_NOT_IMPLEMENTED@ 0000000180030ed8     error_messages.obj
 0002:00003ef8       ??_C@_0BE@MFLGLHIO@UNSUPPORTED_VERSION@ 0000000180030ef8     error_messages.obj
 0002:00003f10       ??_C@_0BB@GAODHGPJ@NAMES_DONT_MATCH@ 0000000180030f10     error_messages.obj
 0002:00003f28       ??_C@_0CH@NAGMIHMO@CLASS_MODIFIERS_CHANGE_NOT_IMPL@ 0000000180030f28     error_messages.obj
 0002:00003f50       ??_C@_0CI@BOHKDDHK@METHOD_MODIFIERS_CHANGE_NOT_IMP@ 0000000180030f50     error_messages.obj
 0002:00003f78       ??_C@_0CH@LDPJIDCO@CLASS_ATTRIBUTE_CHANGE_NOT_IMPL@ 0000000180030f78     error_messages.obj
 0002:00003fa0       ??_C@_0BA@PIOOPNBD@NOT_IMPLEMENTED@ 0000000180030fa0     error_messages.obj
 0002:00003fb0       ??_C@_0N@HEEFEIAJ@NULL_POINTER@ 0000000180030fb0     error_messages.obj
 0002:00003fc0       ??_C@_0BD@JCIODJA@ABSENT_INFORMATION@ 0000000180030fc0     error_messages.obj
 0002:00003fd8       ??_C@_0BD@CAHCPDGO@INVALID_EVENT_TYPE@ 0000000180030fd8     error_messages.obj
 0002:00003ff0       ??_C@_0BB@JNKCIGPM@ILLEGAL_ARGUMENT@ 0000000180030ff0     error_messages.obj
 0002:00004008       ??_C@_0O@KKNEIJDA@OUT_OF_MEMORY@ 0000000180031008     error_messages.obj
 0002:00004018       ??_C@_0O@ILOHOCOF@ACCESS_DENIED@ 0000000180031018     error_messages.obj
 0002:00004028       ??_C@_07DFGEEPDM@VM_DEAD@  0000000180031028     error_messages.obj
 0002:00004030       ??_C@_08MLFDIMPC@INTERNAL@ 0000000180031030     error_messages.obj
 0002:00004040       ??_C@_0BC@ENEFPEAF@UNATTACHED_THREAD@ 0000000180031040     error_messages.obj
 0002:00004058       ??_C@_0M@NLBJDGPL@INVALID_TAG@ 0000000180031058     error_messages.obj
 0002:00004068       ??_C@_0BB@GCBFLFGN@ALREADY_INVOKING@ 0000000180031068     error_messages.obj
 0002:00004080       ??_C@_0O@BDGMMHPL@INVALID_INDEX@ 0000000180031080     error_messages.obj
 0002:00004090       ??_C@_0P@MDIAHEHE@INVALID_LENGTH@ 0000000180031090     error_messages.obj
 0002:000040a0       ??_C@_0P@EJHKHOLE@INVALID_STRING@ 00000001800310a0     error_messages.obj
 0002:000040b0       ??_C@_0BF@FLGJBCL@INVALID_CLASS_LOADER@ 00000001800310b0     error_messages.obj
 0002:000040c8       ??_C@_0O@DBEPKOML@INVALID_ARRAY@ 00000001800310c8     error_messages.obj
 0002:000040d8       ??_C@_0P@IMPOLMOK@TRANSPORT_LOAD@ 00000001800310d8     error_messages.obj
 0002:000040e8       ??_C@_0P@LIHDBHBG@TRANSPORT_INIT@ 00000001800310e8     error_messages.obj
 0002:000040f8       ??_C@_0O@PMKFKNBA@NATIVE_METHOD@ 00000001800310f8     error_messages.obj
 0002:00004108       ??_C@_0O@MHNCFNDK@INVALID_COUNT@ 0000000180031108     error_messages.obj
 0002:00004118       ??_C@_0BD@EHLJKCDN@JDWP_ERROR_unknown@ 0000000180031118     error_messages.obj
 0002:00004130       ??_C@_0DD@FOCDBFMB@DEBUGGING?3?5JDWP?5pause?5for?5PID?5?$CF@ 0000000180031130     error_messages.obj
 0002:00004168       ??_C@_0DI@FMKFEDPB@DEBUGGING?3?5JDWP?5pause?5got?5tired@ 0000000180031168     error_messages.obj
 0002:000041a0       ??_C@_0DI@GJAHDGCJ@s?2src?2jdk?4jdwp?4agent?2share?2nati@ 00000001800311a0     eventFilter.obj
 0002:000041d8       ??_C@_0BB@GAFCOFIH@GetVersionNumber@ 00000001800311d8     eventFilter.obj
 0002:000041f0       ??_C@_0BB@BEKNDEAI@GetLocalInstance@ 00000001800311f0     eventFilter.obj
 0002:00004208       ??_C@_0BB@FFOAPJHA@IsAssignableFrom@ 0000000180031208     eventFilter.obj
 0002:00004220       ??_C@_0N@JPGMCHOC@IsInstanceOf@ 0000000180031220     eventFilter.obj
 0002:00004230       ??_C@_0BK@BBNCBBEI@filter?9?$DOu?4Count?4count?5?$DO?50@ 0000000180031230     eventFilter.obj
 0002:00004250       ??_C@_0BI@BDIJIJG@Invalid?5filter?5modifier@ 0000000180031250     eventFilter.obj
 0002:00004268       ??_C@_03KPOLBBFN@LOC@      0000000180031268     eventFilter.obj
 0002:00004270       ??_C@_0DB@GIOMMMKK@SetBreakpoint?5at?5location?3?5meth@ 0000000180031270     eventFilter.obj
 0002:000042a8       ??_C@_0O@OBFGDNOO@SetBreakpoint@ 00000001800312a8     eventFilter.obj
 0002:000042b8       ??_C@_0DD@BOLIJEFD@ClearBreakpoint?5at?5location?3?5me@ 00000001800312b8     eventFilter.obj
 0002:000042f0       ??_C@_0BA@KALLGBAH@ClearBreakpoint@ 00000001800312f0     eventFilter.obj
 0002:00004300       ??_C@_0BE@BNFCJLBG@SetFieldAccessWatch@ 0000000180031300     eventFilter.obj
 0002:00004318       ??_C@_0BK@LOHLKOFB@SetFieldModificationWatch@ 0000000180031318     eventFilter.obj
 0002:00004338       ??_C@_0BG@IELHINIE@ClearFieldAccessWatch@ 0000000180031338     eventFilter.obj
 0002:00004350       ??_C@_0BM@BCBGEJEO@ClearFieldModificationWatch@ 0000000180031350     eventFilter.obj
 0002:00004370       ??_C@_0CF@PAONPLA@ThreadOnly?3?5thread?$CI?$CFp?$CJ?5isVThrea@ 0000000180031370     eventFilter.obj
 0002:00004398       ??_C@_0BF@IDEBLFKK@ClassOnly?3?5clazz?$CI?$CFs?$CJ@ 0000000180031398     eventFilter.obj
 0002:000043b0       ??_C@_0DB@HPCLAJFC@LocationOnly?3?5clazz?$CI?$CFs?$CJ?0?5method@ 00000001800313b0     eventFilter.obj
 0002:000043e8       ??_C@_0CA@PJNPBAB@FieldOnly?3?5clazz?$CI?$CFp?$CJ?0?5field?$CI?$CFd?$CJ@ 00000001800313e8     eventFilter.obj
 0002:00004408       ??_C@_0DC@MMBOEIIC@ExceptionOnly?3?5clazz?$CI?$CFp?$CJ?0?5caugh@ 0000000180031408     eventFilter.obj
 0002:00004440       ??_C@_0BL@NDAGGOAN@InstanceOnly?3?5instance?$CI?$CFp?$CJ@ 0000000180031440     eventFilter.obj
 0002:00004460       ??_C@_0BB@IEHAPCOC@Count?3?5count?$CI?$CFd?$CJ@ 0000000180031460     eventFilter.obj
 0002:00004478       ??_C@_0BI@NELMLCNN@Conditional?3?5exprID?$CI?$CFd?$CJ@ 0000000180031478     eventFilter.obj
 0002:00004490       ??_C@_0BN@HEEAEBJG@ClassMatch?3?5classPattern?$CI?$CFs?$CJ@ 0000000180031490     eventFilter.obj
 0002:000044b0       ??_C@_0BP@HHOKKDDO@ClassExclude?3?5classPattern?$CI?$CFs?$CJ@ 00000001800314b0     eventFilter.obj
 0002:000044d0       ??_C@_0DC@HDCDDCI@Step?3?5size?$CI?$CFd?$CJ?5depth?$CI?$CFd?$CJ?5thread@ 00000001800314d0     eventFilter.obj
 0002:00004508       ??_C@_0CH@BDELFMMK@SourceNameMatch?3?5sourceNamePatt@ 0000000180031508     eventFilter.obj
 0002:00004530       ??_C@_0BN@BKICEDDC@PlatformThreadsOnly?3?5enabled@ 0000000180031530     eventFilter.obj
 0002:00004550       ??_C@_0DJ@IALHBKPF@s?2src?2jdk?4jdwp?4agent?2share?2nati@ 0000000180031550     eventHandler.obj
 0002:00004590       ??_C@_0BG@HNCJHGFL@bad?5index?5for?5handler@ 0000000180031590     eventHandler.obj
 0002:000045a8       ??_C@_0BH@GJLAODLP@iterator?5function?5NULL@ 00000001800315a8     eventHandler.obj
 0002:000045c0       ??_C@_0EP@MEMOEFKL@Co?9located?5breakpoint?5event?5fou@ 00000001800315c0     eventHandler.obj
 0002:00004610       ??_C@_0EL@CHJDLPBE@event?5report?5being?5skipped?3?5ei?$DN@ 0000000180031610     eventHandler.obj
 0002:00004660       ??_C@_0BB@EIEOGLKK@eventBag?5?$CB?$DN?5NULL@ 0000000180031660     eventHandler.obj
 0002:00004678       ??_C@_0BG@HHJEAHIC@handler?5function?5NULL@ 0000000180031678     eventHandler.obj
 0002:00004690       ??_C@_0BI@NCLCAKI@event_callback?$CI?$CJ?3?5ei?$DN?$CFs@ 0000000180031690     eventHandler.obj
 0002:000046a8       ??_C@_0BB@GKNNLBLP@event_callback?$CI?$CJ@ 00000001800316a8     eventHandler.obj
 0002:000046c0       ??_C@_0CK@GFKKNCOE@Can?8t?5get?5jclass?5for?5a?5methodID@ 00000001800316c0     eventHandler.obj
 0002:000046f0       ??_C@_0BI@OKNNPEIC@cbSingleStep?3?5thread?$DN?$CFp@ 00000001800316f0     eventHandler.obj
 0002:00004708       ??_C@_0CD@FPLFBNDA@Problems?5tracking?5active?5callba@ 0000000180031708     eventHandler.obj
 0002:00004730       ??_C@_0BB@HHEIIDE@END?5cbSingleStep@ 0000000180031730     eventHandler.obj
 0002:00004748       ??_C@_0BI@INKCIGJH@cbBreakpoint?3?5thread?$DN?$CFp@ 0000000180031748     eventHandler.obj
 0002:00004760       ??_C@_0BB@MLFPCDPM@END?5cbBreakpoint@ 0000000180031760     eventHandler.obj
 0002:00004778       ??_C@_0BG@DJEPKKOO@cbFramePop?3?5thread?$DN?$CFp@ 0000000180031778     eventHandler.obj
 0002:00004790       ??_C@_0P@OGOCKOP@END?5cbFramePop@ 0000000180031790     eventHandler.obj
 0002:000047a0       ??_C@_0BH@OOFFIBDG@cbException?3?5thread?$DN?$CFp@ 00000001800317a0     eventHandler.obj
 0002:000047b8       ??_C@_0BA@JBFNAOBA@END?5cbException@ 00000001800317b8     eventHandler.obj
 0002:000047c8       ??_C@_0BJ@DNMCHIHH@cbThreadStart?3?5thread?$DN?$CFp@ 00000001800317c8     eventHandler.obj
 0002:000047e8       ??_C@_0BC@HNAGBODM@END?5cbThreadStart@ 00000001800317e8     eventHandler.obj
 0002:00004800       ??_C@_0BH@CLNHMLJ@cbThreadEnd?3?5thread?$DN?$CFp@ 0000000180031800     eventHandler.obj
 0002:00004818       ??_C@_0BA@PMEDEDIF@END?5cbThreadEnd@ 0000000180031818     eventHandler.obj
 0002:00004828       ??_C@_0BL@EJIHEFHJ@cbVThreadStart?3?5vthread?$DN?$CFp@ 0000000180031828     eventHandler.obj
 0002:00004848       ??_C@_0BJ@GCLBGOLK@gdata?9?$DOvthreadsSupported@ 0000000180031848     eventHandler.obj
 0002:00004868       ??_C@_0BD@BAFFGDHA@END?5cbVThreadStart@ 0000000180031868     eventHandler.obj
 0002:00004880       ??_C@_0BJ@CPLLIFFA@cbVThreadEnd?3?5vthread?$DN?$CFp@ 0000000180031880     eventHandler.obj
 0002:000048a0       ??_C@_0BB@NLALKPBI@END?5cbVThreadEnd@ 00000001800318a0     eventHandler.obj
 0002:000048b8       ??_C@_0BK@KPCGMFCD@cbClassPrepare?3?5thread?$DN?$CFp@ 00000001800318b8     eventHandler.obj
 0002:000048d8       ??_C@_0BD@NJBOMDHE@END?5cbClassPrepare@ 00000001800318d8     eventHandler.obj
 0002:000048f0       ??_C@_0BK@DBGEMJPF@cbGarbageCollectionFinish@ 00000001800318f0     eventHandler.obj
 0002:00004910       ??_C@_0BO@NFODBOGB@END?5cbGarbageCollectionFinish@ 0000000180031910     eventHandler.obj
 0002:00004930       ??_C@_0BH@OAIHEEJM@cbClassLoad?3?5thread?$DN?$CFp@ 0000000180031930     eventHandler.obj
 0002:00004948       ??_C@_0BA@OJJLNIBG@END?5cbClassLoad@ 0000000180031948     eventHandler.obj
 0002:00004958       ??_C@_0BJ@NDKLILBO@cbFieldAccess?3?5thread?$DN?$CFp@ 0000000180031958     eventHandler.obj
 0002:00004978       ??_C@_0BC@PHEEKBJC@END?5cbFieldAccess@ 0000000180031978     eventHandler.obj
 0002:00004990       ??_C@_0BP@NOJMIFFP@cbFieldModification?3?5thread?$DN?$CFp@ 0000000180031990     eventHandler.obj
 0002:000049b0       ??_C@_0BI@JFPADOMO@END?5cbFieldModification@ 00000001800319b0     eventHandler.obj
 0002:000049c8       ??_C@_0BM@FNPGHFD@cbExceptionCatch?3?5thread?$DN?$CFp@ 00000001800319c8     eventHandler.obj
 0002:000049e8       ??_C@_0BF@KCHHGDCL@END?5cbExceptionCatch@ 00000001800319e8     eventHandler.obj
 0002:00004a00       ??_C@_0BJ@BDJJHIIJ@cbMethodEntry?3?5thread?$DN?$CFp@ 0000000180031a00     eventHandler.obj
 0002:00004a20       ??_C@_0BC@ODEOLGDB@END?5cbMethodEntry@ 0000000180031a20     eventHandler.obj
 0002:00004a38       ??_C@_0BI@DMPAEBFP@cbMethodExit?3?5thread?$DN?$CFp@ 0000000180031a38     eventHandler.obj
 0002:00004a50       ??_C@_0BB@DDLCHFPG@END?5cbMethodExit@ 0000000180031a50     eventHandler.obj
 0002:00004a68       ??_C@_0CD@MLINJBLL@cbMonitorContendedEnter?3?5thread@ 0000000180031a68     eventHandler.obj
 0002:00004a90       ??_C@_0BM@FCFEADJF@END?5cbMonitorContendedEnter@ 0000000180031a90     eventHandler.obj
 0002:00004ab0       ??_C@_0CF@PHEBGJDK@cbMonitorContendedEntered?3?5thre@ 0000000180031ab0     eventHandler.obj
 0002:00004ad8       ??_C@_0BO@NKLCNKNJ@END?5cbMonitorContendedEntered@ 0000000180031ad8     eventHandler.obj
 0002:00004af8       ??_C@_0BJ@DBNLPCK@cbMonitorWait?3?5thread?$DN?$CFp@ 0000000180031af8     eventHandler.obj
 0002:00004b18       ??_C@_0BC@HCJEOKMD@END?5cbMonitorWait@ 0000000180031b18     eventHandler.obj
 0002:00004b30       ??_C@_0BL@EDMNBHDO@cbMonitorWaited?3?5thread?$DN?$CFp@ 0000000180031b30     eventHandler.obj
 0002:00004b50       ??_C@_0BE@OPIFFKBH@END?5cbMonitorWaited@ 0000000180031b50     eventHandler.obj
 0002:00004b68       ??_C@_08JPFKMCJM@cbVMInit@ 0000000180031b68     eventHandler.obj
 0002:00004b78       ??_C@_0N@CGBLLPFL@END?5cbVMInit@ 0000000180031b78     eventHandler.obj
 0002:00004b88       ??_C@_09FKPIGOCC@cbVMDeath@ 0000000180031b88     eventHandler.obj
 0002:00004b98       ??_C@_0CI@BDMPOPOL@Can?8t?5clear?5event?5callbacks?5on?5@ 0000000180031b98     eventHandler.obj
 0002:00004bc0       ??_C@_0O@FPEBHIEM@END?5cbVMDeath@ 0000000180031bc0     eventHandler.obj
 0002:00004bd0       ??_C@_0BG@OAPFAEPB@Debug?5Agent?5Data?5Dump@ 0000000180031bd0     eventHandler.obj
 0002:00004be8       ??_C@_0BD@DPDENKHO@?$DN?$DN?$DN?5START?5DUMP?5?$DN?$DN?$DN@ 0000000180031be8     eventHandler.obj
 0002:00004c00       ??_C@_0BB@HKMOAHGB@?$DN?$DN?$DN?5END?5DUMP?5?$DN?$DN?$DN@ 0000000180031c00     eventHandler.obj
 0002:00004c18       ??_C@_0BD@GLFAIKMG@JDWP?5Callback?5Lock@ 0000000180031c18     eventHandler.obj
 0002:00004c30       ??_C@_0BE@MNAKHAMD@JDWP?5Callback?5Block@ 0000000180031c30     eventHandler.obj
 0002:00004c48       ??_C@_0BI@FOIPGHII@JDWP?5Event?5Handler?5Lock@ 0000000180031c48     eventHandler.obj
 0002:00004c60       ??_C@_0BM@MPBGMHFO@Can?8t?5enable?5vm?5init?5events@ 0000000180031c60     eventHandler.obj
 0002:00004c80       ??_C@_0BN@JOALGOKL@Can?8t?5enable?5vm?5death?5events@ 0000000180031c80     eventHandler.obj
 0002:00004ca0       ??_C@_0CB@JOBGHMA@Can?8t?5enable?5thread?5start?5event@ 0000000180031ca0     eventHandler.obj
 0002:00004cc8       ??_C@_0BP@FDDGJEME@Can?8t?5enable?5thread?5end?5events@ 0000000180031cc8     eventHandler.obj
 0002:00004ce8       ??_C@_0CO@BHGAKFIC@Can?8t?5enable?5garbage?5collection@ 0000000180031ce8     eventHandler.obj
 0002:00004d18       ??_C@_0CG@JBBCEOMI@Can?8t?5enable?5data?5dump?5request?5@ 0000000180031d18     eventHandler.obj
 0002:00004d40       ??_C@_0CC@PIGDBGBB@Can?8t?5enable?5vthread?5start?5even@ 0000000180031d40     eventHandler.obj
 0002:00004d68       ??_C@_0CA@HDGBGGPB@Can?8t?5enable?5vthread?5end?5events@ 0000000180031d68     eventHandler.obj
 0002:00004d88       ??_C@_0BK@PHMDAOAK@Can?8t?5set?5event?5callbacks@ 0000000180031d88     eventHandler.obj
 0002:00004da8       ??_C@_0CD@IECGOLID@Can?8t?5disable?5vthread?5start?5eve@ 0000000180031da8     eventHandler.obj
 0002:00004dd0       ??_C@_0CB@GIBFBCPC@Can?8t?5disable?5vthread?5end?5event@ 0000000180031dd0     eventHandler.obj
 0002:00004df8       ??_C@_0BF@KMAHMJND@?6Handlers?5for?5?$CFs?$CI?$CFd?$CJ@ 0000000180031df8     eventHandler.obj
 0002:00004e10       ??_C@_0DH@KJCOMJPA@node?$CI?$CFp?$CJ?5handlerID?$CI?$CFd?$CJ?5suspendP@ 0000000180031e10     eventHandler.obj
 0002:00004e48       ??_C@_0DA@KKIKEDIE@enqueueCommand?$CI?$CJ?3?5HelperCommand@ 0000000180031e48     eventHelper.obj
 0002:00004e78       ??_C@_0CF@LMNBMKHE@enqueueCommand?$CI?$CJ?3?5HelperCommand@ 0000000180031e78     eventHelper.obj
 0002:00004ea0       ??_C@_0CO@HANEHINJ@completeCommand?$CI?$CJ?3?5HelperComman@ 0000000180031ea0     eventHelper.obj
 0002:00004ed0       ??_C@_0DI@GNPLLKOC@s?2src?2jdk?4jdwp?4agent?2share?2nati@ 0000000180031ed0     eventHelper.obj
 0002:00004f08       ??_C@_0CJ@KNNNNIJI@dequeueCommand?$CI?$CJ?3?5command?5being@ 0000000180031f08     eventHelper.obj
 0002:00004f38       ??_C@_0CK@HMEDCJBG@dequeueCommand?$CI?$CJ?3?5command?5sessi@ 0000000180031f38     eventHelper.obj
 0002:00004f68       ??_C@_0CF@PABMCNLB@should?5be?5THREAD_START?5or?5THREA@ 0000000180031f68     eventHelper.obj
 0002:00004f90       ??_C@_0BE@OLGJGEIN@unknown?5event?5index@ 0000000180031f90     eventHelper.obj
 0002:00004fa8       ??_C@_0BF@EBMLONF@Event?5Helper?5Command@ 0000000180031fa8     eventHelper.obj
 0002:00004fc0       ??_C@_0BK@IAKHDCAG@Begin?5command?5loop?5thread@ 0000000180031fc0     eventHelper.obj
 0002:00004fe0       ??_C@_0CF@IHKNBMKL@commandLoop?$CI?$CJ?3?5command?5being?5ha@ 0000000180031fe0     eventHelper.obj
 0002:00005008       ??_C@_0CA@PBIKJLAJ@JDWP?5Event?5Helper?5Queue?5Monitor@ 0000000180032008     eventHelper.obj
 0002:00005028       ??_C@_0CF@DAMBCHBM@JDWP?5Event?5Helper?5Completion?5Mo@ 0000000180032028     eventHelper.obj
 0002:00005050       ??_C@_0CF@PDAKBDPJ@JDWP?5Event?5Block?5CommandLoop?5Mo@ 0000000180032050     eventHelper.obj
 0002:00005078       ??_C@_0CC@JBOJCKEK@JDWP?5VM_DEATH?5CommandLoop?5Monit@ 0000000180032078     eventHelper.obj
 0002:000050a0       ??_C@_0BJ@MHCAKDHO@JDWP?5Event?5Helper?5Thread@ 00000001800320a0     eventHelper.obj
 0002:000050c0       ??_C@_0CP@KONMJMJG@exitVmDeathLockOnError?3?5error?5i@ 00000001800320c0     eventHelper.obj
 0002:000050f0       ??_C@_0BB@POGOAJG@GetCurrentThread@ 00000001800320f0     eventHelper.obj
 0002:00005108       ??_C@_0BB@BFBJHKBE@bagAdd?$CIeventBag?$CJ@ 0000000180032108     eventHelper.obj
 0002:00005120       ??_C@_0BI@GCGOKABC@err?5?$DN?$DN?5JVMTI_ERROR_NONE@ 0000000180032120     eventHelper.obj
 0002:00005138       ??_C@_0O@LKPPNPDK@HelperCommand@ 0000000180032138     eventHelper.obj
 0002:00005148       ??_C@_0P@FHCDPAEP@HelperCommmand@ 0000000180032148     eventHelper.obj
 0002:00005158       ??_C@_0BF@BPGCNEIM@JDWP?5Invocation?5Lock@ 0000000180032158     invoker.obj
 0002:00005170       ??_C@_0CB@NAOIBAAB@Request?5methodSignature?5not?5nul@ 0000000180032170     invoker.obj
 0002:00005198       ??_C@_0DE@EFONEHB@s?2src?2jdk?4jdwp?4agent?2share?2nati@ 0000000180032198     invoker.obj
 0002:000051cc       ??_C@_06FJHNOCKE@thread@   00000001800321cc     invoker.obj
 0002:000051d8       ??_C@_0BO@ICHBCBGF@getting?5thread?5invoke?5request@ 00000001800321d8     invoker.obj
 0002:000051f8       ??_C@_0BI@MLBHEPJD@GetMethodDeclaringClass@ 00000001800321f8     invoker.obj
 0002:00005210       ??_C@_0N@FKNOGHOK@IsSameObject@ 0000000180032210     invoker.obj
 0002:00005220       ??_C@_0BD@GGJIMJB@Request?5clazz?5null@ 0000000180032220     invoker.obj
 0002:00005238       ??_C@_0L@DEGKKCHL@NewObjectA@ 0000000180032238     invoker.obj
 0002:00005248       ??_C@_0BI@JEDJKLFO@CallStaticObjectMethodA@ 0000000180032248     invoker.obj
 0002:00005260       ??_C@_0BG@OLLEIINM@CallStaticByteMethodA@ 0000000180032260     invoker.obj
 0002:00005278       ??_C@_0BG@BGEPLKKM@CallStaticCharMethodA@ 0000000180032278     invoker.obj
 0002:00005290       ??_C@_0BH@PAMJMCFG@CallStaticFloatMethodA@ 0000000180032290     invoker.obj
 0002:000052a8       ??_C@_0BI@IBCKJKHM@CallStaticDoubleMethodA@ 00000001800322a8     invoker.obj
 0002:000052c0       ??_C@_0BF@JPBMCNAM@CallStaticIntMethodA@ 00000001800322c0     invoker.obj
 0002:000052d8       ??_C@_0BG@FKLMGMON@CallStaticLongMethodA@ 00000001800322d8     invoker.obj
 0002:000052f0       ??_C@_0BH@JGHONGAL@CallStaticShortMethodA@ 00000001800322f0     invoker.obj
 0002:00005308       ??_C@_0BJ@PIJAHNCD@CallStaticBooleanMethodA@ 0000000180032308     invoker.obj
 0002:00005328       ??_C@_0BG@GHMCEOMM@CallStaticVoidMethodA@ 0000000180032328     invoker.obj
 0002:00005340       ??_C@_0BJ@NJKAEDMC@Invalid?5method?5signature@ 0000000180032340     invoker.obj
 0002:00005360       ??_C@_0BG@LMEMBPGM@Request?5instance?5null@ 0000000180032360     invoker.obj
 0002:00005378       ??_C@_0BC@DPOBDBNG@CallObjectMethodA@ 0000000180032378     invoker.obj
 0002:00005390       ??_C@_0BA@PKCJIMNA@CallByteMethodA@ 0000000180032390     invoker.obj
 0002:000053a0       ??_C@_0BA@HNCLOKA@CallCharMethodA@ 00000001800323a0     invoker.obj
 0002:000053b0       ??_C@_0BB@PJGOBDHJ@CallFloatMethodA@ 00000001800323b0     invoker.obj
 0002:000053c8       ??_C@_0BC@CKPCAAPE@CallDoubleMethodA@ 00000001800323c8     invoker.obj
 0002:000053e0       ??_C@_0P@DBDHNNH@CallIntMethodA@ 00000001800323e0     invoker.obj
 0002:000053f0       ??_C@_0BA@ELCBGIOB@CallLongMethodA@ 00000001800323f0     invoker.obj
 0002:00005400       ??_C@_0BB@JPNJAHCE@CallShortMethodA@ 0000000180032400     invoker.obj
 0002:00005418       ??_C@_0BD@BLFIKOKL@CallBooleanMethodA@ 0000000180032418     invoker.obj
 0002:00005430       ??_C@_0BA@HGFPEKMA@CallVoidMethodA@ 0000000180032430     invoker.obj
 0002:00005440       ??_C@_0BM@GJKAAPAH@CallNonvirtualObjectMethodA@ 0000000180032440     invoker.obj
 0002:00005460       ??_C@_0BK@GCNLPHID@CallNonvirtualByteMethodA@ 0000000180032460     invoker.obj
 0002:00005480       ??_C@_0BK@JPCAMFPD@CallNonvirtualCharMethodA@ 0000000180032480     invoker.obj
 0002:000054a0       ??_C@_0BL@LJEOBEM@CallNonvirtualFloatMethodA@ 00000001800324a0     invoker.obj
 0002:000054c0       ??_C@_0BM@HMLDDOCF@CallNonvirtualDoubleMethodA@ 00000001800324c0     invoker.obj
 0002:000054e0       ??_C@_0BJ@CDEIJCJF@CallNonvirtualIntMethodA@ 00000001800324e0     invoker.obj
 0002:00005500       ??_C@_0BK@NDNDBDLC@CallNonvirtualLongMethodA@ 0000000180032500     invoker.obj
 0002:00005520       ??_C@_0BL@GNCDPFBB@CallNonvirtualShortMethodA@ 0000000180032520     invoker.obj
 0002:00005540       ??_C@_0BN@OKNKANNH@CallNonvirtualBooleanMethodA@ 0000000180032540     invoker.obj
 0002:00005560       ??_C@_0BK@OOKNDBJD@CallNonvirtualVoidMethodA@ 0000000180032560     invoker.obj
 0002:00005580       ??_C@_0BB@EDABLKKF@request?9?$DOpending@ 0000000180032580     invoker.obj
 0002:00005598       ??_C@_0BB@JHNKMJKL@request?9?$DOstarted@ 0000000180032598     invoker.obj
 0002:000055b0       ??_C@_0BI@OKOEINGF@methodSignature?5is?5NULL@ 00000001800325b0     invoker.obj
 0002:000055c8       ??_C@_07ENHGAJCI@request@  00000001800325c8     invoker.obj
 0002:000055d0       ??_C@_09CMKFMIAO@?$CFs?2?$CFs?4dll@ 00000001800325d0     linker_md.obj
 0002:000055e0       ??_C@_0DI@JPDHMHMH@s?2src?2jdk?4jdwp?4agent?2windows?2na@ 00000001800325e0     linker_md.obj
 0002:00005620       ??_C@_0GB@EFLPCEDF@One?5or?5more?5of?5the?5library?5path@ 0000000180032620     linker_md.obj
 0002:00005684       ??_C@_06DAJAKOAL@?$CFs?4dll@ 0000000180032684     linker_md.obj
 0002:00005690       ??_C@_0BP@KMBPCJLM@Can?8t?5find?5dependent?5libraries@ 0000000180032690     linker_md.obj
 0002:000056b0       ??_C@_0M@ILCKPJLM@?$CFd?4?$CFm?4?$CFY?5?$CFT@ 00000001800326b0     log_messages.obj
 0002:000056bc       ??_C@_02HOGMBHDI@?$CFZ@    00000001800326bc     log_messages.obj
 0002:000056c0       ??_C@_04FHKNIFPB@?$CF?43d@ 00000001800326c0     log_messages.obj
 0002:000056c8       ??_C@_0L@LMNAMKMD@?$CFs?4?$CF?43s?5?$CFs@ 00000001800326c8     log_messages.obj
 0002:000056d8       ??_C@_07CIFAGBMG@unknown@  00000001800326d8     log_messages.obj
 0002:000056e0       ??_C@_0M@JJMNGIAI@?$CFs?3?$CC?$CFs?$CC?3?$CFd?$DL@ 00000001800326e0     log_messages.obj
 0002:000056f0       ??_C@_0BM@BMLHDEI@?$FL?$CD?$HM?$CFs?$HM?$CFs?$HM?$CFs?$HM?$CFs?$HM?$CFs?$HM?$CFs?3?$CFs?$HM?$CD?$FN?6@ 00000001800326f0     log_messages.obj
 0002:0000570c       ??_C@_01NOFIACDB@w@        000000018003270c     log_messages.obj
 0002:00005710       ??_C@_06JGDLHNPI@FINEST@   0000000180032710     log_messages.obj
 0002:00005718       ??_C@_07NPAANBDA@J2SE1?45@ 0000000180032718     log_messages.obj
 0002:00005720       ??_C@_04CAJKAAHJ@jdwp@     0000000180032720     log_messages.obj
 0002:00005728       ??_C@_0BH@HINFEDE@LOC?$DN?$CFs?$DLPID?$DN?$CFd?$DLTHR?$DNt?$EA?$CFd@ 0000000180032728     log_messages.obj
 0002:00005740       ??_C@_05NINEKCGD@?$CFs?4?$CFd@ 0000000180032740     log_messages.obj
 0002:00005748       ??_C@_0DG@EGMOAHHB@s?2src?2jdk?4jdwp?4agent?2share?2nati@ 0000000180032748     outStream.obj
 0002:00005780       ??_C@_0BB@JPLDOFMC@Invalid?5type?5key@ 0000000180032780     outStream.obj
 0002:00005798       ??_C@_0CA@OJHGJLHC@outStream_setError?5error?$DN?$CFs?$CI?$CFd?$CJ@ 0000000180032798     outStream.obj
 0002:000057b8       ??_C@_0BE@DHHKMLKH@isArrayTag?$CItypeKey?$CJ@ 00000001800327b8     signature.obj
 0002:000057d0       ??_C@_0DG@EOHOCBDN@s?2src?2jdk?4jdwp?4agent?2share?2nati@ 00000001800327d0     signature.obj
 0002:00005808       ??_C@_06BHPCHHEB@tagPtr@   0000000180032808     signature.obj
 0002:00005810       ??_C@_0CF@NLOPLAKC@signature?$FL0?$FN?5?$DN?$DN?5SIGNATURE_BEGIN@ 0000000180032810     signature.obj
 0002:00005838       ??_C@_0CE@HPMJLGGG@Should?5never?5call?5handleClassUn@ 0000000180032838     standardHandlers.obj
 0002:00005860       ??_C@_0DN@BIHCGFFE@s?2src?2jdk?4jdwp?4agent?2share?2nati@ 0000000180032860     standardHandlers.obj
 0002:000058a0       ??_C@_0CJ@EJBINECN@Unable?5to?5install?5VM?5Death?5even@ 00000001800328a0     standardHandlers.obj
 0002:000058d0       ??_C@_0DI@LNANLGGM@s?2src?2jdk?4jdwp?4agent?2share?2nati@ 00000001800328d0     stepControl.obj
 0002:00005908       ??_C@_0BE@MKGOBEGB@getting?5frame?5count@ 0000000180032908     stepControl.obj
 0002:0000591c       ??_C@_04MOOLDHHD@STEP@     000000018003291c     stepControl.obj
 0002:00005928       ??_C@_0BK@NIDDNIOA@enableStepping?3?5thread?$DN?$CFp@ 0000000180032928     stepControl.obj
 0002:00005948       ??_C@_0BF@CCJDHFEH@enabling?5single?5step@ 0000000180032948     stepControl.obj
 0002:00005960       ??_C@_0BL@EHDJHHNF@disableStepping?3?5thread?$DN?$CFp@ 0000000180032960     stepControl.obj
 0002:00005980       ??_C@_0BG@LEFCIDGN@disabling?5single?5step@ 0000000180032980     stepControl.obj
 0002:00005998       ??_C@_0P@IEFLKDKM@NotifyFramePop@ 0000000180032998     stepControl.obj
 0002:000059a8       ??_C@_0BG@OKKJJMAC@initState?$CI?$CJ?3?5frame?$DN?$CFd@ 00000001800329a8     stepControl.obj
 0002:000059c0       ??_C@_0BN@LKIHPCMO@initState?$CI?$CJ?3?5Begin?5line?5step@ 00000001800329c0     stepControl.obj
 0002:000059e0       ??_C@_0BF@FOPEDPHN@getting?5step?5request@ 00000001800329e0     stepControl.obj
 0002:000059f8       ??_C@_0DJ@BEIBIGEH@handleFramePopEvent?3?5BEGIN?5from@ 00000001800329f8     stepControl.obj
 0002:00005a38       ??_C@_0DG@IPJGEBF@handleFramePopEvent?3?5starting?5s@ 0000000180032a38     stepControl.obj
 0002:00005a70       ??_C@_0FK@PCMGCGNB@handleFramePopEvent?3?5starting?5s@ 0000000180032a70     stepControl.obj
 0002:00005ad0       ??_C@_0CF@MGOMDHJC@step?9?$DOdepth?5?$DN?$DN?5JDWP_STEP_DEPTH?$CI@ 0000000180032ad0     stepControl.obj
 0002:00005b00       ??_C@_0HJ@MEDPAGIL@handleFramePopEvent?3?5starting?5s@ 0000000180032b00     stepControl.obj
 0002:00005b80       ??_C@_0HH@NFEOAAP@handleFramePopEvent?3?5starting?5s@ 0000000180032b80     stepControl.obj
 0002:00005bf8       ??_C@_0BO@EJIOKDML@handleFramePopEvent?3?5finished@ 0000000180032bf8     stepControl.obj
 0002:00005c18       ??_C@_0DJ@FFHBGECC@handleExceptionCatchEvent?3?5from@ 0000000180032c18     stepControl.obj
 0002:00005c58       ??_C@_0CC@GMNCKPDI@handleMethodEnterEvent?3?5thread?$DN@ 0000000180032c58     stepControl.obj
 0002:00005c80       ??_C@_0BI@ONNFECIM@completeStep?3?5thread?$DN?$CFp@ 0000000180032c80     stepControl.obj
 0002:00005c98       ??_C@_0BI@POGAKJLC@initializing?5step?5state@ 0000000180032c98     stepControl.obj
 0002:00005cb0       ??_C@_0CC@JMCHFEAK@stepControl_handleStep?3?5thread?$DN@ 0000000180032cb0     stepControl.obj
 0002:00005cd8       ??_C@_0CM@NNBPEOLN@stepControl_handleStep?3?5complet@ 0000000180032cd8     stepControl.obj
 0002:00005d08       ??_C@_0DA@FOFCMEJP@stepControl_handleStep?3?5complet@ 0000000180032d08     stepControl.obj
 0002:00005d40       ??_C@_0EB@JJDJIOHA@stepControl_handleStep?3?5complet@ 0000000180032d40     stepControl.obj
 0002:00005d90       ??_C@_0FM@PAKAGCBL@stepControl_handleStep?3?5complet@ 0000000180032d90     stepControl.obj
 0002:00005df0       ??_C@_0CG@MFJECOCG@installing?5event?5method?5enter?5h@ 0000000180032df0     stepControl.obj
 0002:00005e20       ??_C@_0EG@INCGEIIO@stepControl_handleStep?3?5NotifyF@ 0000000180032e20     stepControl.obj
 0002:00005e68       ??_C@_0BM@IPAAJJGN@setting?5up?5notify?5frame?5pop@ 0000000180032e68     stepControl.obj
 0002:00005e90       ??_C@_0EH@PDNBFMBE@stepControl_handleStep?3?5complet@ 0000000180032e90     stepControl.obj
 0002:00005ed8       ??_C@_0BH@BJILJMJK@getting?5frame?5location@ 0000000180032ed8     stepControl.obj
 0002:00005ef0       ??_C@_0CP@KIJNJAEA@stepControl_handleStep?3?5checkin@ 0000000180032ef0     stepControl.obj
 0002:00005f20       ??_C@_0CK@BMELMNFO@stepControl_handleStep?3?5checkin@ 0000000180032f20     stepControl.obj
 0002:00005f50       ??_C@_0FC@HLIPCJAI@stepControl_handleStep?3?5complet@ 0000000180032f50     stepControl.obj
 0002:00005fb0       ??_C@_0EL@JOGIECCM@stepControl_handleStep?3?5complet@ 0000000180032fb0     stepControl.obj
 0002:00006000       ??_C@_0CB@DMEMPEEG@stepControl_handleStep?3?5finishe@ 0000000180033000     stepControl.obj
 0002:00006028       ??_C@_0BH@NFDHFKGE@JDWP?5Step?5Handler?5Lock@ 0000000180033028     stepControl.obj
 0002:00006040       ??_C@_0CE@GBBAGAOP@stepControl_resetRequest?3?5threa@ 0000000180033040     stepControl.obj
 0002:00006068       ??_C@_0CC@POHINOEB@step?9?$DOframePopHandlerNode?5?$DN?$DN?5NU@ 0000000180033068     stepControl.obj
 0002:00006090       ??_C@_0BP@KCAAPAME@installing?5step?5event?5handlers@ 0000000180033090     stepControl.obj
 0002:000060b0       ??_C@_0DC@LKPPLDLN@stepControl_beginStep?3?5thread?$DN?$CF@ 00000001800330b0     stepControl.obj
 0002:000060e8       ??_C@_0CN@MHELALJG@stepControl_beginStep?3?5cannot?5s@ 00000001800330e8     stepControl.obj
 0002:00006118       ??_C@_0P@BHNPMDOE@GetThreadState@ 0000000180033118     stepControl.obj
 0002:00006128       ??_C@_0BF@KAINFNPD@getting?5thread?5state@ 0000000180033128     stepControl.obj
 0002:00006140       ??_C@_0O@HMJOGGOE@SuspendThread@ 0000000180033140     stepControl.obj
 0002:00006150       ??_C@_0BC@BCPADGJN@suspending?5thread@ 0000000180033150     stepControl.obj
 0002:00006168       ??_C@_0BC@GCBOJDGD@ClearAllFramePops@ 0000000180033168     stepControl.obj
 0002:00006180       ??_C@_0BI@KLMOFAGI@clearing?5all?5frame?5pops@ 0000000180033180     stepControl.obj
 0002:00006198       ??_C@_0N@JPHIGJOE@ResumeThread@ 0000000180033198     stepControl.obj
 0002:000061a8       ??_C@_0BA@KDDODNDH@resuming?5thread@ 00000001800331a8     stepControl.obj
 0002:000061b8       ??_C@_0BP@INDEPPPG@stepControl_endStep?3?5thread?$DN?$CFp@ 00000001800331b8     stepControl.obj
 0002:000061d8       ??_C@_0CE@EJEIFKKI@stepControl_clearRequest?3?5threa@ 00000001800331d8     stepControl.obj
 0002:00006200       ??_C@_0DK@MIIMOJNB@s?2src?2jdk?4jdwp?4agent?2share?2nati@ 0000000180033200     threadControl.obj
 0002:00006240       ??_C@_0BG@OHKNBDMG@SetThreadLocalStorage@ 0000000180033240     threadControl.obj
 0002:00006258       ??_C@_0CA@BNIMIHGG@cannot?5set?5thread?5local?5storage@ 0000000180033258     threadControl.obj
 0002:00006278       ??_C@_0BG@BCPLMKIH@GetThreadLocalStorage@ 0000000180033278     threadControl.obj
 0002:00006290       ??_C@_0CA@LOCGOKPD@cannot?5get?5thread?5local?5storage@ 0000000180033290     threadControl.obj
 0002:000062b0       ??_C@_0DB@ONEDOJMK@?$CBnonTlsSearch?$CIgetEnv?$CI?$CJ?0?5?$CGrunnin@ 00000001800332b0     threadControl.obj
 0002:000062e8       ??_C@_0DC@LFGBDHNF@?$CBnonTlsSearch?$CIgetEnv?$CI?$CJ?0?5?$CGrunnin@ 00000001800332e8     threadControl.obj
 0002:00006320       ??_C@_0BD@NHJKPLLD@thread?5table?5entry@ 0000000180033320     threadControl.obj
 0002:00006338       ??_C@_0BG@KBBPCCOI@getting?5vthread?5state@ 0000000180033338     threadControl.obj
 0002:00006350       ??_C@_0N@MOPCPKLO@node?5?$CB?$DN?5NULL@ 0000000180033350     threadControl.obj
 0002:00006360       ??_C@_0CH@CFIIJJMO@findThread?$CIdest?0?5node?9?$DOthread?$CJ?5@ 0000000180033360     threadControl.obj
 0002:00006390       ??_C@_0ED@OAECAMKM@cannot?5process?5deferred?5thread?5@ 0000000180033390     threadControl.obj
 0002:000063d8       ??_C@_0BB@EFDALKHP@JDWP?5Thread?5Lock@ 00000001800333d8     threadControl.obj
 0002:000063f0       ??_C@_0N@BJJFBAKB@thread?5table@ 00000001800333f0     threadControl.obj
 0002:00006400       ??_C@_0BE@PLBAIHPP@thread?$DN?$CFp?5suspended@ 0000000180033400     threadControl.obj
 0002:00006418       ??_C@_0CG@OBNDHFIM@error?5?$CB?$DN?5JVMTI_ERROR_THREAD_SUS@ 0000000180033418     threadControl.obj
 0002:00006440       ??_C@_0BG@MADFCJCH@?$CBnode?9?$DOsuspendOnStart@ 0000000180033440     threadControl.obj
 0002:00006458       ??_C@_0BC@DNHNKGGE@thread?$DN?$CFp?5resumed@ 0000000180033458     threadControl.obj
 0002:00006470       ??_C@_0BD@BIMLGJDG@?$CBnode?9?$DOtoBeResumed@ 0000000180033470     threadControl.obj
 0002:00006488       ??_C@_0BE@PGDPIDGL@resume?5request?5list@ 0000000180033488     threadControl.obj
 0002:000064a0       ??_C@_0M@FIFGDPKA@resume?5list@ 00000001800334a0     threadControl.obj
 0002:000064b0       ??_C@_0BB@FPIEDMNB@ResumeThreadList@ 00000001800334b0     threadControl.obj
 0002:000064c8       ??_C@_0CG@OGGIDGFO@missing?5entry?5in?5running?5thread@ 00000001800334c8     threadControl.obj
 0002:000064f0       ??_C@_0CC@EENAOFCJ@thread?$DN?$CFp?5resumed?5as?5part?5of?5li@ 00000001800334f0     threadControl.obj
 0002:00006518       ??_C@_0N@JJLGEDON@request?5list@ 0000000180033518     threadControl.obj
 0002:00006528       ??_C@_0BF@BGHKIDKG@suspend?5list?5results@ 0000000180033528     threadControl.obj
 0002:00006540       ??_C@_0BC@GFPPJMEE@SuspendThreadList@ 0000000180033540     threadControl.obj
 0002:00006558       ??_C@_0BP@JBJIEHDD@missing?5entry?5in?5thread?5tables@ 0000000180033558     threadControl.obj
 0002:00006578       ??_C@_0CE@BDMKGMJL@thread?$DN?$CFp?5suspended?5as?5part?5of?5@ 0000000180033578     threadControl.obj
 0002:000065a0       ??_C@_0BO@IJHNAMAJ@threadControl_suspendThread?$CI?$CJ@ 00000001800335a0     threadControl.obj
 0002:000065c0       ??_C@_0BN@GKLHJPIH@threadControl_resumeThread?$CI?$CJ@ 00000001800335c0     threadControl.obj
 0002:000065e0       ??_C@_0BL@CGJFPBGG@threadControl_suspendAll?$CI?$CJ@ 00000001800335e0     threadControl.obj
 0002:00006600       ??_C@_0BJ@KNDIOMNP@SuspendAllVirtualThreads@ 0000000180033600     threadControl.obj
 0002:00006620       ??_C@_0CD@GIPOMLIK@cannot?5suspend?5all?5virtual?5thre@ 0000000180033620     threadControl.obj
 0002:00006648       ??_C@_0BK@PPCACBKK@error?5?$DN?$DN?5JVMTI_ERROR_NONE@ 0000000180033648     threadControl.obj
 0002:00006668       ??_C@_0BB@LANBAGIB@node?9?$DOis_vthread@ 0000000180033668     threadControl.obj
 0002:00006680       ??_C@_0BK@KAONLLJF@threadControl_resumeAll?$CI?$CJ@ 0000000180033680     threadControl.obj
 0002:000066a0       ??_C@_0N@PEEDDFGM@exclude?5list@ 00000001800336a0     threadControl.obj
 0002:000066b0       ??_C@_0BI@BIEAGNLB@ResumeAllVirtualThreads@ 00000001800336b0     threadControl.obj
 0002:000066c8       ??_C@_0CC@MINDHLLL@cannot?5resume?5all?5virtual?5threa@ 00000001800336c8     threadControl.obj
 0002:000066f0       ??_C@_0BJ@CHKMKGNA@JDWP?5PopFrame?5Event?5Lock@ 00000001800336f0     threadControl.obj
 0002:00006710       ??_C@_0BL@NLADKEIC@JDWP?5PopFrame?5Proceed?5Lock@ 0000000180033710     threadControl.obj
 0002:00006730       ??_C@_0BG@BDPIMKHA@entry?5in?5thread?5table@ 0000000180033730     threadControl.obj
 0002:00006748       ??_C@_08PALMFDC@PopFrame@  0000000180033748     threadControl.obj
 0002:00006758       ??_C@_0CB@FDGFBJBH@thread?$DN?$CFp?5resumed?5in?5popOneFram@ 0000000180033758     threadControl.obj
 0002:00006780       ??_C@_0CD@CBFJIOGD@thread?$DN?$CFp?5suspended?5in?5popOneFr@ 0000000180033780     threadControl.obj
 0002:000067a8       ??_C@_0BK@HGCCNNPL@threadControl_popFrames?$CI?$CJ@ 00000001800337a8     threadControl.obj
 0002:000067c8       ??_C@_0BO@BMDHOIKK@thread?5start?5during?5pop?5frame@ 00000001800337c8     threadControl.obj
 0002:000067e8       ??_C@_0CE@DLABLPCM@threadControl_onEventHandlerEnt@ 00000001800337e8     threadControl.obj
 0002:00006810       ??_C@_0BO@JCMOFHDO@ei?5?$CB?$DN?5EI_VIRTUAL_THREAD_START@ 0000000180033810     threadControl.obj
 0002:00006830       ??_C@_0BM@CJBFEEHN@ei?5?$CB?$DN?5EI_VIRTUAL_THREAD_END@ 0000000180033830     threadControl.obj
 0002:00006850       ??_C@_0BA@PNKGFJII@InterruptThread@ 0000000180033850     threadControl.obj
 0002:00006860       ??_C@_0L@FBFPPEII@StopThread@ 0000000180033860     threadControl.obj
 0002:00006870       ??_C@_0CD@DBNMOEOD@threadControl_onEventHandlerExi@ 0000000180033870     threadControl.obj
 0002:00006898       ??_C@_0BG@EPAAPLLF@thread?5list?5corrupted@ 0000000180033898     threadControl.obj
 0002:000068b0       ??_C@_0CI@GCOAEGE@threadControl_applicationThread@ 00000001800338b0     threadControl.obj
 0002:000068d8       ??_C@_0BK@BIOOONKE@threadControl_interrupt?$CI?$CJ@ 00000001800338d8     threadControl.obj
 0002:000068f8       ??_C@_0BF@NHLBNOB@threadControl_stop?$CI?$CJ@ 00000001800338f8     threadControl.obj
 0002:00006910       ??_C@_0BL@KPAJNPJE@otherThreads?4first?5?$DN?$DN?5NULL@ 0000000180033910     threadControl.obj
 0002:00006930       ??_C@_0CG@BCMJEBGB@countedVThreads?5?$DN?$DN?5numRunningVT@ 0000000180033930     threadControl.obj
 0002:00006958       ??_C@_0BE@NCJPIJME@suspendAllCount?3?5?$CFd@ 0000000180033958     threadControl.obj
 0002:00006970       ??_C@_0BI@CABFDKOI@Dumping?5runningThreads?3@ 0000000180033970     threadControl.obj
 0002:00006988       ??_C@_0BK@OPBOAPDA@?6Dumping?5runningVThreads?3@ 0000000180033988     threadControl.obj
 0002:000069a8       ??_C@_0BH@OCINPPDO@?6Dumping?5otherThreads?3@ 00000001800339a8     threadControl.obj
 0002:000069c0       ??_C@_0CA@PPMGHLOG@Thread?3?5node?5?$DN?5?$CFp?0?5jthread?5?$DN?5?$CFp@ 00000001800339c0     threadControl.obj
 0002:000069e0       ??_C@_0BC@BAGDNDCK@?7suspendCount?3?5?$CFd@ 00000001800339e0     threadControl.obj
 0002:000069f8       ??_C@_0DG@DKBGPIDI@s?2src?2jdk?4jdwp?4agent?2share?2nati@ 00000001800339f8     transport.obj
 0002:00006a30       ??_C@_0BH@DPMJLMBJ@transport?5error?5?$CFd?3?5?$CFs@ 0000000180033a30     transport.obj
 0002:00006a48       ??_C@_07NFANNNEC@UNKNOWN@  0000000180033a48     transport.obj
 0002:00006a50       ??_C@_0BF@FOBNBFPM@jdwpTransport_OnLoad@ 0000000180033a50     transport.obj
 0002:00006a68       ??_C@_0BG@FMJOLAEE@library?5name?5is?5empty@ 0000000180033a68     transport.obj
 0002:00006a80       ??_C@_0CI@LAKGPIH@internal?5error?3?5info?5should?5not@ 0000000180033a80     transport.obj
 0002:00006aa8       ??_C@_0CP@KHDMANEH@Java?5property?5sun?4boot?4library?4@ 0000000180033aa8     transport.obj
 0002:00006ad8       ??_C@_0CA@EHDNLIPG@transport?5library?5not?5found?3?5?$CFs@ 0000000180033ad8     transport.obj
 0002:00006af8       ??_C@_0CL@KNFBHFGD@transport?5library?5missing?5onLoa@ 0000000180033af8     transport.obj
 0002:00006b28       ??_C@_09KFMAMAFK@GetJavaVM@ 0000000180033b28     transport.obj
 0002:00006b38       ??_C@_0CP@JIHKFCKD@insufficient?5memory?5to?5complete@ 0000000180033b38     transport.obj
 0002:00006b70       ??_C@_0EB@ONKBAHBP@transport?5doesn?8t?5recognize?5all@ 0000000180033b70     transport.obj
 0002:00006bb8       ??_C@_0DA@LIDKNCMN@transport?5doesn?8t?5support?5multi@ 0000000180033bb8     transport.obj
 0002:00006be8       ??_C@_0CF@BGANCHCG@unrecognized?5error?5?$CFd?5from?5tran@ 0000000180033be8     transport.obj
 0002:00006c10       ??_C@_0BJ@IFDFBAP@sun?4jdwp?4listenerAddress@ 0000000180033c10     transport.obj
 0002:00006c30       ??_C@_0BE@JKJABKEE@Begin?5accept?5thread@ 0000000180033c30     transport.obj
 0002:00006c48       ??_C@_0CK@GLGDCAJA@could?5not?5connect?0?5timeout?5or?5f@ 0000000180033c48     transport.obj
 0002:00006c78       ??_C@_0BC@NENNJKEM@End?5accept?5thread@ 0000000180033c78     transport.obj
 0002:00006c90       ??_C@_0BE@BNNAEGLJ@Begin?5attach?5thread@ 0000000180033c90     transport.obj
 0002:00006ca8       ??_C@_0BC@FDJNMGLB@End?5attach?5thread@ 0000000180033ca8     transport.obj
 0002:00006cc0       ??_C@_0CA@PPOAMFKF@JDWP?5Transport?5Listener?5Monitor@ 0000000180033cc0     transport.obj
 0002:00006ce0       ??_C@_0BM@EOHCCJHG@JDWP?5Transport?5Send?5Monitor@ 0000000180033ce0     transport.obj
 0002:00006cfc       ??_C@_01CLKCMJKC@?5@       0000000180033cfc     transport.obj
 0002:00006d00       ??_C@_0DO@LDLIIPAI@Allow?5parameter?5is?5specified?5bu@ 0000000180033d00     transport.obj
 0002:00006d40       ??_C@_01JLIPDDHJ@?3@       0000000180033d40     transport.obj
 0002:00006d48       ??_C@_0BK@NKDBJPAM@JDWP?5Transport?5Listener?3?5@ 0000000180033d48     transport.obj
 0002:00006d68       ??_C@_0CK@NABHANCN@Listening?5for?5transport?5?$CFs?5at?5a@ 0000000180033d68     transport.obj
 0002:00006d98       ??_C@_0BJ@NDKKCKOJ@UTF?5ERROR?5?$FL?$CC?$CFs?$CC?3?$CFd?$FN?3?5?$CFs?6@ 0000000180033d98     utf_util.obj
 0002:00006db8       ??_C@_0BH@PGKNPGMC@ASSERT?5ERROR?5i?$DN?$DNlength@ 0000000180033db8     utf_util.obj
 0002:00006dd0       ??_C@_0DF@HFLPGPCA@s?2src?2jdk?4jdwp?4agent?2share?2nati@ 0000000180033dd0     utf_util.obj
 0002:00006e08       ??_C@_0BK@HADMOKCE@ASSERT?5ERROR?5j?$DN?$DNnewLength@ 0000000180033e08     utf_util.obj
 0002:00006e28       ??_C@_0BN@ILDOBJEF@Can?8t?5get?5WIDE?5string?5length@ 0000000180033e28     utf_util.obj
 0002:00006e48       ??_C@_0BJ@LFBNLHDK@Can?8t?5malloc?$CI?$CJ?5any?5space@ 0000000180033e48     utf_util.obj
 0002:00006e68       ??_C@_0BG@OELEGHKP@Can?8t?5get?5WIDE?5string@ 0000000180033e68     utf_util.obj
 0002:00006e80       ??_C@_0BC@FAJHJFKN@ASSERT?5ERROR?5utf8@ 0000000180033e80     utf_util.obj
 0002:00006e98       ??_C@_0BE@MONHEHKE@ASSERT?5ERROR?5output@ 0000000180033e98     utf_util.obj
 0002:00006eb0       ??_C@_0BG@IGPBKLGM@ASSERT?5ERROR?5len?5?$DO?$DN?50@ 0000000180033eb0     utf_util.obj
 0002:00006ec8       ??_C@_0CB@NCJBKIBF@ASSERT?5ERROR?5outputBufSize?5?$DO?5le@ 0000000180033ec8     utf_util.obj
 0002:00006ef0       ??_C@_0BB@LBCDKBGH@ASSERT?5ERROR?5str@ 0000000180033ef0     utf_util.obj
 0002:00006f08       ??_C@_0CI@EJHCPIBO@Can?8t?5convert?5WIDE?5string?5to?5mu@ 0000000180033f08     utf_util.obj
 0002:00006f30       ??_C@_0DB@OKLBDJGC@s?2src?2jdk?4jdwp?4agent?2share?2nati@ 0000000180033f30     util.obj
 0002:00006f68       ??_C@_0BD@FDGEFMPC@saveGlobalRef?5pobj@ 0000000180033f68     util.obj
 0002:00006f80       ??_C@_0BE@HPCONGOG@saveGlobalRef?5?$CKpobj@ 0000000180033f80     util.obj
 0002:00006f98       ??_C@_0BC@DCADFAHL@saveGlobalRef?5env@ 0000000180033f98     util.obj
 0002:00006fb0       ??_C@_0BC@LCNDBECG@saveGlobalRef?5obj@ 0000000180033fb0     util.obj
 0002:00006fc8       ??_C@_0BD@EBGPHOMG@tossGlobalRef?5pobj@ 0000000180033fc8     util.obj
 0002:00006fe0       ??_C@_0BC@IOMIDECC@tossGlobalRef?5env@ 0000000180033fe0     util.obj
 0002:00006ff8       ??_C@_0BC@OBIHAHP@tossGlobalRef?5obj@ 0000000180033ff8     util.obj
 0002:00007010       ??_C@_0O@IHOLADDN@findClass?5env@ 0000000180034010     util.obj
 0002:00007020       ??_C@_0P@HPKFFFCG@findClass?5name@ 0000000180034020     util.obj
 0002:00007030       ??_C@_09MBLIIDDK@FindClass@ 0000000180034030     util.obj
 0002:00007040       ??_C@_0CI@KCCMKKPA@JNI?5Exception?5occurred?5finding?5@ 0000000180034040     util.obj
 0002:00007068       ??_C@_0O@GPBJKDDD@getMethod?5env@ 0000000180034068     util.obj
 0002:00007078       ??_C@_0BA@FGFFFLNK@getMethod?5clazz@ 0000000180034078     util.obj
 0002:00007088       ??_C@_0P@JIPFIKIB@getMethod?5name@ 0000000180034088     util.obj
 0002:00007098       ??_C@_0BE@CCFOHHKE@getMethod?5signature@ 0000000180034098     util.obj
 0002:000070b0       ??_C@_0M@BBNOPHHB@GetMethodID@ 00000001800340b0     util.obj
 0002:000070c0       ??_C@_0DL@FGGIPDMN@JNI?5Exception?5occurred?5finding?5@ 00000001800340c0     util.obj
 0002:00007100       ??_C@_0BE@PJAHCBJI@getStaticMethod?5env@ 0000000180034100     util.obj
 0002:00007118       ??_C@_0BG@BIBAEKOK@getStaticMethod?5clazz@ 0000000180034118     util.obj
 0002:00007130       ??_C@_0BF@NJGHOOGD@getStaticMethod?5name@ 0000000180034130     util.obj
 0002:00007148       ??_C@_0BK@NDPLJBJF@getStaticMethod?5signature@ 0000000180034148     util.obj
 0002:00007168       ??_C@_0BC@MJDCJNCH@GetStaticMethodID@ 0000000180034168     util.obj
 0002:00007180       ??_C@_0DM@IMIOOKLN@JDWP?5Exception?5occurred?5finding@ 0000000180034180     util.obj
 0002:000071c0       ??_C@_0BA@JJLOPNCP@java?1lang?1Class@ 00000001800341c0     util.obj
 0002:000071d0       ??_C@_0BB@NOKBFPFO@java?1lang?1Thread@ 00000001800341d0     util.obj
 0002:000071e8       ??_C@_0BG@FMEDAMPL@java?1lang?1ThreadGroup@ 00000001800341e8     util.obj
 0002:00007200       ??_C@_0BG@HADLBHEN@java?1lang?1ClassLoader@ 0000000180034200     util.obj
 0002:00007218       ??_C@_0BB@FLFAIHG@java?1lang?1String@ 0000000180034218     util.obj
 0002:00007230       ??_C@_0BB@NAICLKDB@java?1lang?1System@ 0000000180034230     util.obj
 0002:00007248       ??_C@_0BF@JMMLIHKH@java?1util?1Properties@ 0000000180034248     util.obj
 0002:00007260       ??_C@_0CN@EFABAIOP@?$CILjava?1lang?1ThreadGroup?$DLLjava?1l@ 0000000180034260     util.obj
 0002:00007290       ??_C@_06FALKBLGB@?$DMinit?$DO@ 0000000180034290     util.obj
 0002:00007298       ??_C@_04LHKBAEFM@?$CIZ?$CJV@ 0000000180034298     util.obj
 0002:000072a0       ??_C@_09GMGCGCNB@setDaemon@ 00000001800342a0     util.obj
 0002:000072b0       ??_C@_0CH@NCPCFFHJ@?$CILjava?1lang?1String?$DL?$CJLjava?1lang?1@ 00000001800342b0     util.obj
 0002:000072d8       ??_C@_0M@NBNLNHMA@getProperty@ 00000001800342d8     util.obj
 0002:000072e8       ??_C@_0DJ@BABOCAJP@?$CILjava?1lang?1String?$DLLjava?1lang?1S@ 00000001800342e8     util.obj
 0002:00007328       ??_C@_0M@NOMFABED@setProperty@ 0000000180034328     util.obj
 0002:00007338       ??_C@_0BO@CMFEIIEP@Can?8t?5get?5system?5thread?5group@ 0000000180034338     util.obj
 0002:00007358       ??_C@_0N@KAKDDEJA@java?4version@ 0000000180034358     util.obj
 0002:00007368       ??_C@_0N@FFLEMEAC@java?4vm?4name@ 0000000180034368     util.obj
 0002:00007378       ??_C@_0N@EJENAPCP@java?4vm?4info@ 0000000180034378     util.obj
 0002:00007388       ??_C@_0BA@BKCDAGON@java?4class?4path@ 0000000180034388     util.obj
 0002:00007398       ??_C@_0BG@HAHGGNHO@sun?4boot?4library?4path@ 0000000180034398     util.obj
 0002:000073b0       ??_C@_0P@GNCHJOPK@path?4separator@ 00000001800343b0     util.obj
 0002:000073c0       ??_C@_08IOMDCONK@user?4dir@ 00000001800343c0     util.obj
 0002:000073d0       ??_C@_0BK@DKBCNDAC@jdk?1internal?1vm?1VMSupport@ 00000001800343d0     util.obj
 0002:000073f0       ??_C@_0BJ@BIOCMJG@?$CI?$CJLjava?1util?1Properties?$DL@ 00000001800343f0     util.obj
 0002:00007410       ??_C@_0BD@KIFIICML@getAgentProperties@ 0000000180034410     util.obj
 0002:00007428       ??_C@_0BH@FMELKLIP@CallStaticObjectMethod@ 0000000180034428     util.obj
 0002:00007440       ??_C@_0DI@CNPAJEKH@Exception?5occurred?5calling?5VMSu@ 0000000180034440     util.obj
 0002:00007478       ??_C@_0P@NGFPBMPI@GetObjectField@ 0000000180034478     util.obj
 0002:00007488       ??_C@_0N@PICDCNEH@GetByteField@ 0000000180034488     util.obj
 0002:00007498       ??_C@_0N@DKHIINEE@GetCharField@ 0000000180034498     util.obj
 0002:000074a8       ??_C@_0O@ENLNECGO@GetFloatField@ 00000001800344a8     util.obj
 0002:000074b8       ??_C@_0P@MGBEMHIL@GetDoubleField@ 00000001800344b8     util.obj
 0002:000074c8       ??_C@_0M@LAAAOMAB@GetIntField@ 00000001800344c8     util.obj
 0002:000074d8       ??_C@_0N@EDNEBKMF@GetLongField@ 00000001800344d8     util.obj
 0002:000074e8       ??_C@_0O@GJMDLMFF@GetShortField@ 00000001800344e8     util.obj
 0002:000074f8       ??_C@_0BA@BNOCBIGH@GetBooleanField@ 00000001800344f8     util.obj
 0002:00007508       ??_C@_0BF@IIMAGDFM@GetStaticObjectField@ 0000000180034508     util.obj
 0002:00007520       ??_C@_0BD@HKPDDFOM@GetStaticByteField@ 0000000180034520     util.obj
 0002:00007538       ??_C@_0BD@LIKIJFOP@GetStaticCharField@ 0000000180034538     util.obj
 0002:00007550       ??_C@_0BE@MDLOIBG@GetStaticFloatField@ 0000000180034550     util.obj
 0002:00007568       ??_C@_0BF@JIILLICP@GetStaticDoubleField@ 0000000180034568     util.obj
 0002:00007580       ??_C@_0BC@GIOMIGFH@GetStaticIntField@ 0000000180034580     util.obj
 0002:00007598       ??_C@_0BD@MBAEACGO@GetStaticLongField@ 0000000180034598     util.obj
 0002:000075b0       ??_C@_0BE@CIEFBGCN@GetStaticShortField@ 00000001800345b0     util.obj
 0002:000075c8       ??_C@_0BG@MMAHOAOJ@GetStaticBooleanField@ 00000001800345c8     util.obj
 0002:000075e0       ??_C@_0BC@OMFJHBGB@GetFieldModifiers@ 00000001800345e0     util.obj
 0002:000075f8       ??_C@_0BD@MKDIHAMO@GetMethodModifiers@ 00000001800345f8     util.obj
 0002:00007610       ??_C@_0BC@IEPBNALO@GetMethodLocation@ 0000000180034610     util.obj
 0002:00007628       ??_C@_0O@GILEHKFL@GetMethodName@ 0000000180034628     util.obj
 0002:00007638       ??_C@_0N@NGLPCACC@GetFieldName@ 0000000180034638     util.obj
 0002:00007650       ??_C@_0EH@KPFCNOHP@JDWP?5Unable?5to?5get?5JNI?51?42?5envi@ 0000000180034650     util.obj
 0002:00007698       ??_C@_0BI@LAHADAN@Spawning?5new?5thread?3?5?$CFs@ 0000000180034698     util.obj
 0002:000076b0       ??_C@_09FKAPGGP@NewObject@ 00000001800346b0     util.obj
 0002:000076c0       ??_C@_0P@ICNACBEG@CallVoidMethod@ 00000001800346c0     util.obj
 0002:000076d0       ??_C@_0P@DJOFCLII@RunAgentThread@ 00000001800346d0     util.obj
 0002:000076e0       ??_C@_0BA@OPKACKGF@GetCapabilities@ 00000001800346e0     util.obj
 0002:000076f0       ??_C@_0CE@HHNFGJJN@on?5getting?5the?5JVMTI?5version?5nu@ 00000001800346f0     util.obj
 0002:00007718       ??_C@_0BI@ENBJCOLA@GetSourceDebugExtension@ 0000000180034718     util.obj
 0002:00007730       ??_C@_0BN@EMLFDJOM@VM_DEAD?0?5in?5debugMonitor?$CK?$CI?$CJ?$DP@ 0000000180034730     util.obj
 0002:00007750       ??_C@_0BA@LGEBNIEA@RawMonitorEnter@ 0000000180034750     util.obj
 0002:00007760       ??_C@_0BF@HPIHFHIM@on?5raw?5monitor?5enter@ 0000000180034760     util.obj
 0002:00007778       ??_C@_0P@KLKLHGFP@RawMonitorExit@ 0000000180034778     util.obj
 0002:00007788       ??_C@_0BE@GBAEDMCM@on?5raw?5monitor?5exit@ 0000000180034788     util.obj
 0002:000077a0       ??_C@_0P@JMJKKKKI@RawMonitorWait@ 00000001800347a0     util.obj
 0002:000077b0       ??_C@_0BE@FGDFOANL@on?5raw?5monitor?5wait@ 00000001800347b0     util.obj
 0002:000077c8       ??_C@_0BB@BADFPBLM@RawMonitorNotify@ 00000001800347c8     util.obj
 0002:000077e0       ??_C@_0BG@ICCOLJKI@on?5raw?5monitor?5notify@ 00000001800347e0     util.obj
 0002:000077f8       ??_C@_0BE@DMHNDKAM@RawMonitorNotifyAll@ 00000001800347f8     util.obj
 0002:00007810       ??_C@_0BK@IADPLGNI@on?5raw?5monitor?5notify?5all@ 0000000180034810     util.obj
 0002:00007830       ??_C@_0BB@JDINKLEG@CreateRawMonitor@ 0000000180034830     util.obj
 0002:00007848       ??_C@_0BN@LOANNDKM@on?5creation?5of?5a?5raw?5monitor@ 0000000180034848     util.obj
 0002:00007868       ??_C@_0BE@EADHGNCO@getting?5all?5threads@ 0000000180034868     util.obj
 0002:00007880       ??_C@_0BD@NCBLAKCF@GetThreadGroupInfo@ 0000000180034880     util.obj
 0002:00007898       ??_C@_0BN@CIHPHBI@on?5getting?5thread?5group?5info@ 0000000180034898     util.obj
 0002:000078b8       ??_C@_0BC@KKCEBIKL@GetClassSignature@ 00000001800348b8     util.obj
 0002:000078d0       ??_C@_0BI@DOAGCGDM@on?5getting?5class?5status@ 00000001800348d0     util.obj
 0002:000078e8       ??_C@_0N@MDOILCOK@IsArrayClass@ 00000001800348e8     util.obj
 0002:000078f8       ??_C@_0BP@KJLIJLJN@on?5checking?5for?5an?5array?5class@ 00000001800348f8     util.obj
 0002:00007918       ??_C@_0M@MIKDFOKN@IsInterface@ 0000000180034918     util.obj
 0002:00007928       ??_C@_0BN@DEKKBCOO@on?5checking?5for?5an?5interface@ 0000000180034928     util.obj
 0002:00007948       ??_C@_0BB@GDNGBOGG@IsFieldSynthetic@ 0000000180034948     util.obj
 0002:00007960       ??_C@_0BC@CNKKCFND@IsMethodSynthetic@ 0000000180034960     util.obj
 0002:00007978       ??_C@_0P@MGFNMOMF@IsMethodNative@ 0000000180034978     util.obj
 0002:00007988       ??_C@_0CD@EMIAHINC@on?5checking?5for?5a?5native?5interf@ 0000000180034988     util.obj
 0002:000079b0       ??_C@_0BJ@MOLBHIDD@GetImplementedInterfaces@ 00000001800349b0     util.obj
 0002:000079d0       ??_C@_0BB@GNCMCKG@GetLoadedClasses@ 00000001800349d0     util.obj
 0002:000079e8       ??_C@_0BG@MKDAPNKD@GetClassLoaderClasses@ 00000001800349e8     util.obj
 0002:00007a00       ??_C@_0P@KJBCCNJH@PushLocalFrame@ 0000000180034a00     util.obj
 0002:00007a10       ??_C@_0CJ@GCEOKHEO@PushLocalFrame?3?5Unable?5to?5push?5@ 0000000180034a10     util.obj
 0002:00007a40       ??_C@_0BC@GGHEKHNA@GetSystemProperty@ 0000000180034a40     util.obj
 0002:00007a58       ??_C@_0CF@NNJAIEKP@JDWP?5Can?8t?5get?5property?5value?5f@ 0000000180034a58     util.obj
 0002:00007a80       ??_C@_0BB@CBHJBEJP@IsMethodObsolete@ 0000000180034a80     util.obj
 0002:00007a98       ??_C@_08PEJFBAGK@Allocate@ 0000000180034a98     util.obj
 0002:00007aa8       ??_C@_0BM@ODCKHMNI@Can?8t?5allocate?5jvmti?5memory@ 0000000180034aa8     util.obj
 0002:00007ac8       ??_C@_0L@KKLFJCNC@Deallocate@ 0000000180034ac8     util.obj
 0002:00007ad8       ??_C@_0BO@BLAPEFNH@Can?8t?5deallocate?5jvmti?5memory@ 0000000180034ad8     util.obj
 0002:00007af8       ??_C@_0P@IBCMMHME@bad?5EventIndex@ 0000000180034af8     util.obj
 0002:00007b08       ??_C@_0BL@BIJDOKDA@EI_MONITOR_CONTENDED_ENTER@ 0000000180034b08     util.obj
 0002:00007b28       ??_C@_0BN@HNNNOACM@EI_MONITOR_CONTENDED_ENTERED@ 0000000180034b28     util.obj
 0002:00007b48       ??_C@_0BA@EKCEMLPD@EI_MONITOR_WAIT@ 0000000180034b48     util.obj
 0002:00007b58       ??_C@_0BC@NBGDCGEI@EI_MONITOR_WAITED@ 0000000180034b58     util.obj
 0002:00007b6c       ??_C@_06OJMFFNPK@Bad?5EI@  0000000180034b6c     util.obj
 0002:00007b74       ??_C@_01OGPIMHDM@?$DP@     0000000180034b74     util.obj
 0002:00007b78       ??_C@_0DF@KKCEPIGI@?$CFs?3?5debuggee?3?5thread?$DN?$CFp?$CI?$CFs?30x?$CFx@ 0000000180034b78     util.obj
 0002:00007bb0       ??_C@_0BB@GFEELDOE@FollowReferences@ 0000000180034bb0     util.obj
 0002:00007bc8       ??_C@_0BD@BPILAJHK@GetObjectsWithTags@ 0000000180034bc8     util.obj
 0002:00007be0       ??_C@_0BH@NKLJCIAP@ForceGarbageCollection@ 0000000180034be0     util.obj
 0002:00007bf8       ??_C@_0BD@FIHAEDOF@IterateThroughHeap@ 0000000180034bf8     util.obj
 0002:00007c10       __xmm@00000000000000380000003500000034 0000000180034c10     util.obj
 0002:00007c20       __xmm@00000033000000320000004a00000049 0000000180034c20     util.obj
 0002:00007c30       __xmm@0000003a0000003d0000003e0000003c 0000000180034c30     util.obj
 0002:00007c40       __xmm@0000003b000000400000003f00000037 0000000180034c40     util.obj
 0002:00007c50       __xmm@0000004c0000004b0000004200000041 0000000180034c50     util.obj
 0002:00007c60       __xmm@ffffffffffffffffffffffffffffffff 0000000180034c60     MSVCRT:utility.obj
 0002:00007c70       _pDefaultRawDllMain        0000000180034c70     MSVCRT:dll_dllmain.obj
 0002:00007c70       _pRawDllMain               0000000180034c70     MSVCRT:dll_dllmain.obj
 0002:00007c90       _load_config_used          0000000180034c90     MSVCRT:loadcfg.obj
 0002:00007e80       __volatile_metadata        0000000180034e80     <linker-defined>
 0002:00008250       __rtc_iaa                  0000000180035250     MSVCRT:initsect.obj
 0002:00008258       __rtc_izz                  0000000180035258     MSVCRT:initsect.obj
 0002:00008260       __rtc_taa                  0000000180035260     MSVCRT:initsect.obj
 0002:00008268       __rtc_tzz                  0000000180035268     MSVCRT:initsect.obj
 0002:00009244       __IMPORT_DESCRIPTOR_jvm    0000000180036244     jvm:jvm.dll
 0002:00009258       __IMPORT_DESCRIPTOR_KERNEL32 0000000180036258     kernel32:KERNEL32.dll
 0002:0000926c       __IMPORT_DESCRIPTOR_VCRUNTIME140 000000018003626c     vcruntime:VCRUNTIME140.dll
 0002:00009280       __IMPORT_DESCRIPTOR_api-ms-win-crt-stdio-l1-1-0 0000000180036280     ucrt:api-ms-win-crt-stdio-l1-1-0.dll
 0002:00009294       __IMPORT_DESCRIPTOR_api-ms-win-crt-string-l1-1-0 0000000180036294     ucrt:api-ms-win-crt-string-l1-1-0.dll
 0002:000092a8       __IMPORT_DESCRIPTOR_api-ms-win-crt-runtime-l1-1-0 00000001800362a8     ucrt:api-ms-win-crt-runtime-l1-1-0.dll
 0002:000092bc       __IMPORT_DESCRIPTOR_api-ms-win-crt-convert-l1-1-0 00000001800362bc     ucrt:api-ms-win-crt-convert-l1-1-0.dll
 0002:000092d0       __IMPORT_DESCRIPTOR_api-ms-win-crt-environment-l1-1-0 00000001800362d0     ucrt:api-ms-win-crt-environment-l1-1-0.dll
 0002:000092e4       __IMPORT_DESCRIPTOR_api-ms-win-crt-filesystem-l1-1-0 00000001800362e4     ucrt:api-ms-win-crt-filesystem-l1-1-0.dll
 0002:000092f8       __IMPORT_DESCRIPTOR_api-ms-win-crt-time-l1-1-0 00000001800362f8     ucrt:api-ms-win-crt-time-l1-1-0.dll
 0002:0000930c       __IMPORT_DESCRIPTOR_api-ms-win-crt-heap-l1-1-0 000000018003630c     ucrt:api-ms-win-crt-heap-l1-1-0.dll
 0002:00009320       __NULL_IMPORT_DESCRIPTOR   0000000180036320     jvm:jvm.dll
 0003:00000000       ArrayReference_CmdSet      0000000180037000     ArrayReferenceImpl.obj
 0003:00000018       ArrayReference_Commands    0000000180037018     ArrayReferenceImpl.obj
 0003:00000048       ArrayType_CmdSet           0000000180037048     ArrayTypeImpl.obj
 0003:00000060       ArrayType_Commands         0000000180037060     ArrayTypeImpl.obj
 0003:00000070       ClassLoaderReference_CmdSet 0000000180037070     ClassLoaderReferenceImpl.obj
 0003:00000088       ClassLoaderReference_Commands 0000000180037088     ClassLoaderReferenceImpl.obj
 0003:00000098       ClassObjectReference_CmdSet 0000000180037098     ClassObjectReferenceImpl.obj
 0003:000000b0       ClassObjectReference_Commands 00000001800370b0     ClassObjectReferenceImpl.obj
 0003:000000c0       ClassType_CmdSet           00000001800370c0     ClassTypeImpl.obj
 0003:000000e0       ClassType_Commands         00000001800370e0     ClassTypeImpl.obj
 0003:00000120       EventRequest_CmdSet        0000000180037120     EventRequestImpl.obj
 0003:00000138       EventRequest_Commands      0000000180037138     EventRequestImpl.obj
 0003:00000168       Field_CmdSet               0000000180037168     FieldImpl.obj
 0003:00000180       InterfaceType_CmdSet       0000000180037180     InterfaceTypeImpl.obj
 0003:00000198       InterfaceType_Commands     0000000180037198     InterfaceTypeImpl.obj
 0003:000001b0       Method_CmdSet              00000001800371b0     MethodImpl.obj
 0003:000001d0       Method_Commands            00000001800371d0     MethodImpl.obj
 0003:00000220       ModuleReference_CmdSet     0000000180037220     ModuleReferenceImpl.obj
 0003:00000238       ModuleReference_Commands   0000000180037238     ModuleReferenceImpl.obj
 0003:00000260       ObjectReference_CmdSet     0000000180037260     ObjectReferenceImpl.obj
 0003:00000280       ObjectReference_Commands   0000000180037280     ObjectReferenceImpl.obj
 0003:00000320       ReferenceType_CmdSet       0000000180037320     ReferenceTypeImpl.obj
 0003:00000340       ReferenceType_Commands     0000000180037340     ReferenceTypeImpl.obj
 0003:00000470       StackFrame_CmdSet          0000000180037470     StackFrameImpl.obj
 0003:00000490       StackFrame_Commands        0000000180037490     StackFrameImpl.obj
 0003:000004d0       StringReference_CmdSet     00000001800374d0     StringReferenceImpl.obj
 0003:000004e8       StringReference_Commands   00000001800374e8     StringReferenceImpl.obj
 0003:000004f8       ThreadGroupReference_CmdSet 00000001800374f8     ThreadGroupReferenceImpl.obj
 0003:00000510       ThreadGroupReference_Commands 0000000180037510     ThreadGroupReferenceImpl.obj
 0003:00000540       ThreadReference_CmdSet     0000000180037540     ThreadReferenceImpl.obj
 0003:00000560       ThreadReference_Commands   0000000180037560     ThreadReferenceImpl.obj
 0003:00000650       VirtualMachine_CmdSet      0000000180037650     VirtualMachineImpl.obj
 0003:00000670       VirtualMachine_Commands    0000000180037670     VirtualMachineImpl.obj
 0003:000007fc       _fltused                   00000001800377fc     MSVCRT:fltused.obj
 0003:00000800       __security_cookie          0000000180037800     MSVCRT:gs_cookie.obj
 0003:00000808       __security_cookie_complement 0000000180037808     MSVCRT:gs_cookie.obj
 0003:00000810       __scrt_native_dllmain_reason 0000000180037810     MSVCRT:utility.obj
 0003:00000818       __isa_available            0000000180037818     MSVCRT:cpu_disp.obj
 0003:0000081c       __isa_enabled              000000018003781c     MSVCRT:cpu_disp.obj
 0003:00000820       __memset_fast_string_threshold 0000000180037820     MSVCRT:cpu_disp.obj
 0003:00000828       __memset_nt_threshold      0000000180037828     MSVCRT:cpu_disp.obj
 0003:00000830       __scrt_ucrt_dll_is_in_use  0000000180037830     MSVCRT:ucrt_stubs.obj
 0003:000010f0       gdata                      00000001800380f0     util.obj
 0003:00001170       __scrt_current_native_startup_state 0000000180038170     MSVCRT:utility.obj
 0003:00001178       __scrt_native_startup_lock 0000000180038178     MSVCRT:utility.obj
 0003:00001730       __favor                    0000000180038730     MSVCRT:cpu_disp.obj
 0003:00001734       __scrt_debugger_hook_flag  0000000180038734     MSVCRT:utility_desktop.obj
 0003:00001740       ?__type_info_root_node@@3U__type_info_node@@A 0000000180038740     MSVCRT:tncleanup.obj
 0003:00001750       ?_OptionsStorage@?1??__local_stdio_scanf_options@@9@4_KA 0000000180038750     MSVCRT:default_local_stdio_options.obj
 0003:00001758       ?_OptionsStorage@?1??__local_stdio_printf_options@@9@9 0000000180038758     <common>
 0003:00001760       __dyn_tls_init_callback    0000000180038760     <common>

 entry point at        0001:0002aa40

 Static symbols

 0000:fffc3000       .debug$S                   0000000180000000     jdwp.exp
 0000:fffc3000       .debug$S                   0000000180000000     vcruntime:VCRUNTIME140.dll
 0000:fffc3000       .debug$S                   0000000180000000     vcruntime:VCRUNTIME140.dll
 0000:fffc3000       .debug$S                   0000000180000000     vcruntime:VCRUNTIME140.dll
 0000:fffc3000       .debug$S                   0000000180000000     vcruntime:VCRUNTIME140.dll
 0000:fffc3000       .debug$S                   0000000180000000     vcruntime:VCRUNTIME140.dll
 0000:fffc3000       .debug$S                   0000000180000000     vcruntime:VCRUNTIME140.dll
 0000:fffc3000       .debug$S                   0000000180000000     vcruntime:VCRUNTIME140.dll
 0000:fffc3000       .debug$S                   0000000180000000     vcruntime:VCRUNTIME140.dll
 0000:fffc3000       .debug$S                   0000000180000000     vcruntime:VCRUNTIME140.dll
 0000:fffc3000       .debug$S                   0000000180000000     vcruntime:VCRUNTIME140.dll
 0000:fffc3000       .debug$S                   0000000180000000     ucrt:api-ms-win-crt-convert-l1-1-0.dll
 0000:fffc3000       .debug$S                   0000000180000000     ucrt:api-ms-win-crt-convert-l1-1-0.dll
 0000:fffc3000       .debug$S                   0000000180000000     ucrt:api-ms-win-crt-convert-l1-1-0.dll
 0000:fffc3000       .debug$S                   0000000180000000     ucrt:api-ms-win-crt-environment-l1-1-0.dll
 0000:fffc3000       .debug$S                   0000000180000000     ucrt:api-ms-win-crt-filesystem-l1-1-0.dll
 0000:fffc3000       .debug$S                   0000000180000000     ucrt:api-ms-win-crt-heap-l1-1-0.dll
 0000:fffc3000       .debug$S                   0000000180000000     ucrt:api-ms-win-crt-heap-l1-1-0.dll
 0000:fffc3000       .debug$S                   0000000180000000     ucrt:api-ms-win-crt-runtime-l1-1-0.dll
 0000:fffc3000       .debug$S                   0000000180000000     ucrt:api-ms-win-crt-runtime-l1-1-0.dll
 0000:fffc3000       .debug$S                   0000000180000000     ucrt:api-ms-win-crt-runtime-l1-1-0.dll
 0000:fffc3000       .debug$S                   0000000180000000     ucrt:api-ms-win-crt-runtime-l1-1-0.dll
 0000:fffc3000       .debug$S                   0000000180000000     ucrt:api-ms-win-crt-runtime-l1-1-0.dll
 0000:fffc3000       .debug$S                   0000000180000000     ucrt:api-ms-win-crt-runtime-l1-1-0.dll
 0000:fffc3000       .debug$S                   0000000180000000     ucrt:api-ms-win-crt-runtime-l1-1-0.dll
 0000:fffc3000       .debug$S                   0000000180000000     ucrt:api-ms-win-crt-runtime-l1-1-0.dll
 0000:fffc3000       .debug$S                   0000000180000000     ucrt:api-ms-win-crt-runtime-l1-1-0.dll
 0000:fffc3000       .debug$S                   0000000180000000     ucrt:api-ms-win-crt-runtime-l1-1-0.dll
 0000:fffc3000       .debug$S                   0000000180000000     ucrt:api-ms-win-crt-runtime-l1-1-0.dll
 0000:fffc3000       .debug$S                   0000000180000000     ucrt:api-ms-win-crt-runtime-l1-1-0.dll
 0000:fffc3000       .debug$S                   0000000180000000     ucrt:api-ms-win-crt-runtime-l1-1-0.dll
 0000:fffc3000       .debug$S                   0000000180000000     ucrt:api-ms-win-crt-runtime-l1-1-0.dll
 0000:fffc3000       .debug$S                   0000000180000000     ucrt:api-ms-win-crt-runtime-l1-1-0.dll
 0000:fffc3000       .debug$S                   0000000180000000     ucrt:api-ms-win-crt-runtime-l1-1-0.dll
 0000:fffc3000       .debug$S                   0000000180000000     ucrt:api-ms-win-crt-runtime-l1-1-0.dll
 0000:fffc3000       .debug$S                   0000000180000000     ucrt:api-ms-win-crt-stdio-l1-1-0.dll
 0000:fffc3000       .debug$S                   0000000180000000     ucrt:api-ms-win-crt-stdio-l1-1-0.dll
 0000:fffc3000       .debug$S                   0000000180000000     ucrt:api-ms-win-crt-stdio-l1-1-0.dll
 0000:fffc3000       .debug$S                   0000000180000000     ucrt:api-ms-win-crt-stdio-l1-1-0.dll
 0000:fffc3000       .debug$S                   0000000180000000     ucrt:api-ms-win-crt-stdio-l1-1-0.dll
 0000:fffc3000       .debug$S                   0000000180000000     ucrt:api-ms-win-crt-stdio-l1-1-0.dll
 0000:fffc3000       .debug$S                   0000000180000000     ucrt:api-ms-win-crt-stdio-l1-1-0.dll
 0000:fffc3000       .debug$S                   0000000180000000     ucrt:api-ms-win-crt-string-l1-1-0.dll
 0000:fffc3000       .debug$S                   0000000180000000     ucrt:api-ms-win-crt-string-l1-1-0.dll
 0000:fffc3000       .debug$S                   0000000180000000     ucrt:api-ms-win-crt-string-l1-1-0.dll
 0000:fffc3000       .debug$S                   0000000180000000     ucrt:api-ms-win-crt-string-l1-1-0.dll
 0000:fffc3000       .debug$S                   0000000180000000     ucrt:api-ms-win-crt-string-l1-1-0.dll
 0000:fffc3000       .debug$S                   0000000180000000     ucrt:api-ms-win-crt-string-l1-1-0.dll
 0000:fffc3000       .debug$S                   0000000180000000     ucrt:api-ms-win-crt-string-l1-1-0.dll
 0000:fffc3000       .debug$S                   0000000180000000     ucrt:api-ms-win-crt-string-l1-1-0.dll
 0000:fffc3000       .debug$S                   0000000180000000     ucrt:api-ms-win-crt-time-l1-1-0.dll
 0000:fffc3000       .debug$S                   0000000180000000     ucrt:api-ms-win-crt-time-l1-1-0.dll
 0000:fffc3000       .debug$S                   0000000180000000     ucrt:api-ms-win-crt-time-l1-1-0.dll
 0000:fffc3000       .debug$S                   0000000180000000     kernel32:KERNEL32.dll
 0000:fffc3000       .debug$S                   0000000180000000     kernel32:KERNEL32.dll
 0000:fffc3000       .debug$S                   0000000180000000     kernel32:KERNEL32.dll
 0000:fffc3000       .debug$S                   0000000180000000     kernel32:KERNEL32.dll
 0000:fffc3000       .debug$S                   0000000180000000     kernel32:KERNEL32.dll
 0000:fffc3000       .debug$S                   0000000180000000     kernel32:KERNEL32.dll
 0000:fffc3000       .debug$S                   0000000180000000     kernel32:KERNEL32.dll
 0000:fffc3000       .debug$S                   0000000180000000     kernel32:KERNEL32.dll
 0000:fffc3000       .debug$S                   0000000180000000     kernel32:KERNEL32.dll
 0000:fffc3000       .debug$S                   0000000180000000     kernel32:KERNEL32.dll
 0000:fffc3000       .debug$S                   0000000180000000     kernel32:KERNEL32.dll
 0000:fffc3000       .debug$S                   0000000180000000     kernel32:KERNEL32.dll
 0000:fffc3000       .debug$S                   0000000180000000     kernel32:KERNEL32.dll
 0000:fffc3000       .debug$S                   0000000180000000     kernel32:KERNEL32.dll
 0000:fffc3000       .debug$S                   0000000180000000     kernel32:KERNEL32.dll
 0000:fffc3000       .debug$S                   0000000180000000     kernel32:KERNEL32.dll
 0000:fffc3000       .debug$S                   0000000180000000     kernel32:KERNEL32.dll
 0000:fffc3000       .debug$S                   0000000180000000     kernel32:KERNEL32.dll
 0000:fffc3000       .debug$S                   0000000180000000     kernel32:KERNEL32.dll
 0000:fffc3000       .debug$S                   0000000180000000     kernel32:KERNEL32.dll
 0000:fffc3000       .debug$S                   0000000180000000     kernel32:KERNEL32.dll
 0000:fffc3000       .debug$S                   0000000180000000     kernel32:KERNEL32.dll
 0000:fffc3000       .debug$S                   0000000180000000     kernel32:KERNEL32.dll
 0000:fffc3000       .debug$S                   0000000180000000     kernel32:KERNEL32.dll
 0000:fffc3000       .debug$S                   0000000180000000     kernel32:KERNEL32.dll
 0000:fffc3000       .debug$S                   0000000180000000     kernel32:KERNEL32.dll
 0000:fffc3000       .debug$S                   0000000180000000     kernel32:KERNEL32.dll
 0000:fffc3000       .debug$S                   0000000180000000     kernel32:KERNEL32.dll
 0000:fffc3000       .debug$S                   0000000180000000     kernel32:KERNEL32.dll
 0000:fffc3000       .debug$S                   0000000180000000     jvm:jvm.dll
 0001:00000000       length                     0000000180001000 f   ArrayReferenceImpl.obj
 0001:000000ac       getValues                  00000001800010ac f   ArrayReferenceImpl.obj
 0001:00000358       setValues                  0000000180001358 f   ArrayReferenceImpl.obj
 0001:00000610       newComponents              0000000180001610 f   ArrayReferenceImpl.obj
 0001:0000067c       readBooleanComponents      000000018000167c f   ArrayReferenceImpl.obj
 0001:00000760       readByteComponents         0000000180001760 f   ArrayReferenceImpl.obj
 0001:00000844       readCharComponents         0000000180001844 f   ArrayReferenceImpl.obj
 0001:00000928       readComponents             0000000180001928 f   ArrayReferenceImpl.obj
 0001:00000c60       readDoubleComponents       0000000180001c60 f   ArrayReferenceImpl.obj
 0001:00000d44       readFloatComponents        0000000180001d44 f   ArrayReferenceImpl.obj
 0001:00000e28       readIntComponents          0000000180001e28 f   ArrayReferenceImpl.obj
 0001:00000f0c       readLongComponents         0000000180001f0c f   ArrayReferenceImpl.obj
 0001:00000ff0       readObjectComponents       0000000180001ff0 f   ArrayReferenceImpl.obj
 0001:00001108       readShortComponents        0000000180002108 f   ArrayReferenceImpl.obj
 0001:000011ec       writeBooleanComponents     00000001800021ec f   ArrayReferenceImpl.obj
 0001:000012c8       writeByteComponents        00000001800022c8 f   ArrayReferenceImpl.obj
 0001:000013a4       writeCharComponents        00000001800023a4 f   ArrayReferenceImpl.obj
 0001:00001484       writeComponents            0000000180002484 f   ArrayReferenceImpl.obj
 0001:000016c4       writeDoubleComponents      00000001800026c4 f   ArrayReferenceImpl.obj
 0001:000017a4       writeFloatComponents       00000001800027a4 f   ArrayReferenceImpl.obj
 0001:00001884       writeIntComponents         0000000180002884 f   ArrayReferenceImpl.obj
 0001:00001964       writeLongComponents        0000000180002964 f   ArrayReferenceImpl.obj
 0001:00001a44       writeObjectComponents      0000000180002a44 f   ArrayReferenceImpl.obj
 0001:00001bb0       writeShortComponents       0000000180002bb0 f   ArrayReferenceImpl.obj
 0001:00001c90       newInstance                0000000180002c90 f   ArrayTypeImpl.obj
 0001:00001e10       writeNewObjectArray        0000000180002e10 f   ArrayTypeImpl.obj
 0001:000020e8       writeNewPrimitiveArray     00000001800030e8 f   ArrayTypeImpl.obj
 0001:000024c0       visibleClasses             00000001800034c0 f   ClassLoaderReferenceImpl.obj
 0001:000025f0       reflectedType              00000001800035f0 f   ClassObjectReferenceImpl.obj
 0001:00002664       superclass                 0000000180003664 f   ClassTypeImpl.obj
 0001:0000276c       setValues                  000000018000376c f   ClassTypeImpl.obj
 0001:000028b0       invokeStatic               00000001800038b0 f   ClassTypeImpl.obj
 0001:000028b0       invokeStatic               00000001800038b0 f   InterfaceTypeImpl.obj
 0001:000028b0       invokeInstance             00000001800038b0 f   ObjectReferenceImpl.obj
 0001:000028b8       readStaticFieldValue       00000001800038b8 f   ClassTypeImpl.obj
 0001:00002da8       setCommand                 0000000180003da8 f   EventRequestImpl.obj
 0001:00002ed4       clearCommand               0000000180003ed4 f   EventRequestImpl.obj
 0001:00002f6c       clearAllBreakpoints        0000000180003f6c f   EventRequestImpl.obj
 0001:00002fa0       readAndSetFilters          0000000180003fa0 f   EventRequestImpl.obj
 0001:00003418       lineTable                  0000000180004418 f   MethodImpl.obj
 0001:000035b4       variableTable              00000001800045b4 f   MethodImpl.obj
 0001:000035bc       variableTableWithGenerics  00000001800045bc f   MethodImpl.obj
 0001:000035c8       bytecodes                  00000001800045c8 f   MethodImpl.obj
 0001:000036cc       isObsolete                 00000001800046cc f   MethodImpl.obj
 0001:0000373c       doVariableTable            000000018000473c f   MethodImpl.obj
 0001:00003970       getName                    0000000180004970 f   ModuleReferenceImpl.obj
 0001:00003c54       getClassLoader             0000000180004c54 f   ModuleReferenceImpl.obj
 0001:00003e84       referenceType              0000000180004e84 f   ObjectReferenceImpl.obj
 0001:00003fa4       getValues                  0000000180004fa4 f   ObjectReferenceImpl.obj
 0001:00003fb8       setValues                  0000000180004fb8 f   ObjectReferenceImpl.obj
 0001:000041a0       monitorInfo                00000001800051a0 f   ObjectReferenceImpl.obj
 0001:00004374       disableCollection          0000000180005374 f   ObjectReferenceImpl.obj
 0001:000043d0       enableCollection           00000001800053d0 f   ObjectReferenceImpl.obj
 0001:0000442c       isCollected                000000018000542c f   ObjectReferenceImpl.obj
 0001:000044c4       referringObjects           00000001800054c4 f   ObjectReferenceImpl.obj
 0001:00004638       readFieldValue             0000000180005638 f   ObjectReferenceImpl.obj
 0001:00004b34       signature                  0000000180005b34 f   ReferenceTypeImpl.obj
 0001:00004bcc       signatureWithGeneric       0000000180005bcc f   ReferenceTypeImpl.obj
 0001:00004c78       getClassLoader             0000000180005c78 f   ReferenceTypeImpl.obj
 0001:00004d04       getModule                  0000000180005d04 f   ReferenceTypeImpl.obj
 0001:00004db4       modifiers                  0000000180005db4 f   ReferenceTypeImpl.obj
 0001:00004e78       methods                    0000000180005e78 f   ReferenceTypeImpl.obj
 0001:00004e80       methodsWithGeneric         0000000180005e80 f   ReferenceTypeImpl.obj
 0001:00004e8c       instances                  0000000180005e8c f   ReferenceTypeImpl.obj
 0001:00005000       getClassVersion            0000000180006000 f   ReferenceTypeImpl.obj
 0001:000050d8       getConstantPool            00000001800060d8 f   ReferenceTypeImpl.obj
 0001:000051d8       fields                     00000001800061d8 f   ReferenceTypeImpl.obj
 0001:000051e0       fieldsWithGeneric          00000001800061e0 f   ReferenceTypeImpl.obj
 0001:000051ec       getValues                  00000001800061ec f   ReferenceTypeImpl.obj
 0001:00005200       sourceFile                 0000000180006200 f   ReferenceTypeImpl.obj
 0001:000052d4       sourceDebugExtension       00000001800062d4 f   ReferenceTypeImpl.obj
 0001:00005358       nestedTypes                0000000180006358 f   ReferenceTypeImpl.obj
 0001:00005490       getClassStatus             0000000180006490 f   ReferenceTypeImpl.obj
 0001:000054f0       interfaces                 00000001800064f0 f   ReferenceTypeImpl.obj
 0001:00005610       classObject                0000000180006610 f   ReferenceTypeImpl.obj
 0001:00005674       fields1                    0000000180006674 f   ReferenceTypeImpl.obj
 0001:000057ac       methods1                   00000001800067ac f   ReferenceTypeImpl.obj
 0001:000058e4       writeFieldInfo             00000001800068e4 f   ReferenceTypeImpl.obj
 0001:000059f8       writeMethodInfo            00000001800069f8 f   ReferenceTypeImpl.obj
 0001:00005c64       decode                     0000000180006c64 f   SDE.obj
 0001:00005e1c       ignoreLine                 0000000180006e1c f   SDE.obj
 0001:00005e50       lineSection                0000000180006e50 f   SDE.obj
 0001:00005f38       loadDebugInfo              0000000180006f38 f   SDE.obj
 0001:00006070       readLine                   0000000180007070 f   SDE.obj
 0001:00006118       readNumber                 0000000180007118 f   SDE.obj
 0001:00006174       sdePeek                    0000000180007174 f   SDE.obj
 0001:00006198       sdeRead                    0000000180007198 f   SDE.obj
 0001:00006358       storeFile                  0000000180007358 f   SDE.obj
 0001:000064a8       storeLine                  00000001800074a8 f   SDE.obj
 0001:00006618       storeStratum               0000000180007618 f   SDE.obj
 0001:00006798       stratumTableIndex          0000000180007798 f   SDE.obj
 0001:00006820       syntax                     0000000180007820 f   SDE.obj
 0001:0000688c       getValues                  000000018000788c f   StackFrameImpl.obj
 0001:000069d0       setValues                  00000001800079d0 f   StackFrameImpl.obj
 0001:00006b08       thisObject                 0000000180007b08 f   StackFrameImpl.obj
 0001:00006d48       popFrames                  0000000180007d48 f   StackFrameImpl.obj
 0001:00006e08       readVariableValue          0000000180007e08 f   StackFrameImpl.obj
 0001:000071b4       validateThreadFrame        00000001800081b4 f   StackFrameImpl.obj
 0001:00007200       writeVariableValue         0000000180008200 f   StackFrameImpl.obj
 0001:00007750       value                      0000000180008750 f   StringReferenceImpl.obj
 0001:000078bc       name                       00000001800088bc f   ThreadGroupReferenceImpl.obj
 0001:000079b4       parent                     00000001800089b4 f   ThreadGroupReferenceImpl.obj
 0001:00007aa0       children                   0000000180008aa0 f   ThreadGroupReferenceImpl.obj
 0001:00007c54       name                       0000000180008c54 f   ThreadReferenceImpl.obj
 0001:00007dbc       suspend                    0000000180008dbc f   ThreadReferenceImpl.obj
 0001:00007e38       resume                     0000000180008e38 f   ThreadReferenceImpl.obj
 0001:00007eb4       status                     0000000180008eb4 f   ThreadReferenceImpl.obj
 0001:00007f50       threadGroup                0000000180008f50 f   ThreadReferenceImpl.obj
 0001:000080b8       frames                     00000001800090b8 f   ThreadReferenceImpl.obj
 0001:000083b0       getFrameCount              00000001800093b0 f   ThreadReferenceImpl.obj
 0001:00008498       ownedMonitors              0000000180009498 f   ThreadReferenceImpl.obj
 0001:0000864c       currentContendedMonitor    000000018000964c f   ThreadReferenceImpl.obj
 0001:000087cc       stop                       00000001800097cc f   ThreadReferenceImpl.obj
 0001:0000887c       interrupt                  000000018000987c f   ThreadReferenceImpl.obj
 0001:000088f4       suspendCount               00000001800098f4 f   ThreadReferenceImpl.obj
 0001:00008980       ownedMonitorsWithStackDepth 0000000180009980 f   ThreadReferenceImpl.obj
 0001:00008b60       forceEarlyReturn           0000000180009b60 f   ThreadReferenceImpl.obj
 0001:00008f64       isVirtual                  0000000180009f64 f   ThreadReferenceImpl.obj
 0001:0000902c       validateSuspendedThread    000000018000a02c f   ThreadReferenceImpl.obj
 0001:00009078       version                    000000018000a078 f   VirtualMachineImpl.obj
 0001:000091c4       classesForSignature        000000018000a1c4 f   VirtualMachineImpl.obj
 0001:000093f8       allModules                 000000018000a3f8 f   VirtualMachineImpl.obj
 0001:00009550       allClasses                 000000018000a550 f   VirtualMachineImpl.obj
 0001:00009558       allClassesWithGeneric      000000018000a558 f   VirtualMachineImpl.obj
 0001:00009564       instanceCounts             000000018000a564 f   VirtualMachineImpl.obj
 0001:00009720       redefineClasses            000000018000a720 f   VirtualMachineImpl.obj
 0001:00009958       setDefaultStratum          000000018000a958 f   VirtualMachineImpl.obj
 0001:000099b4       getAllThreads              000000018000a9b4 f   VirtualMachineImpl.obj
 0001:00009b30       topLevelThreadGroups       000000018000ab30 f   VirtualMachineImpl.obj
 0001:00009c84       dispose                    000000018000ac84 f   VirtualMachineImpl.obj
 0001:00009c88       idSizes                    000000018000ac88 f   VirtualMachineImpl.obj
 0001:00009cdc       suspend                    000000018000acdc f   VirtualMachineImpl.obj
 0001:00009d20       resume                     000000018000ad20 f   VirtualMachineImpl.obj
 0001:00009d64       doExit                     000000018000ad64 f   VirtualMachineImpl.obj
 0001:00009e08       createString               000000018000ae08 f   VirtualMachineImpl.obj
 0001:00009fa8       capabilities               000000018000afa8 f   VirtualMachineImpl.obj
 0001:0000a08c       capabilitiesNew            000000018000b08c f   VirtualMachineImpl.obj
 0001:0000a2a0       classPaths                 000000018000b2a0 f   VirtualMachineImpl.obj
 0001:0000a3f0       disposeObjects             000000018000b3f0 f   VirtualMachineImpl.obj
 0001:0000a49c       holdEvents                 000000018000b49c f   VirtualMachineImpl.obj
 0001:0000a4ac       releaseEvents              000000018000b4ac f   VirtualMachineImpl.obj
 0001:0000a4bc       allClasses1                000000018000b4bc f   VirtualMachineImpl.obj
 0001:0000a8d0       addPreparedClass           000000018000b8d0 f   classTrack.obj
 0001:0000adf4       is_wrong_phase             000000018000bdf4 f   classTrack.obj
 0001:0000ae38       setupEvents                000000018000be38 f   classTrack.obj
 0001:0000b944       createNode                 000000018000c944 f   commonRef.obj
 0001:0000bbb0       deleteNode                 000000018000cbb0 f   commonRef.obj
 0001:0000bd2c       deleteNodeByID             000000018000cd2c f   commonRef.obj
 0001:0000be60       initializeObjectsByID      000000018000ce60 f   commonRef.obj
 0001:0000beb8       newCommonRef               000000018000ceb8 f   commonRef.obj
 0001:0000bfd0       strengthenNode             000000018000cfd0 f   commonRef.obj
 0001:0000c154       weakenNode                 000000018000d154 f   commonRef.obj
 0001:0000cae4       atexit_finish_logging      000000018000dae4 f   debugInit.obj
 0001:0000caec       cbEarlyException           000000018000daec f   debugInit.obj
 0001:0000cfac       cbEarlyVMDeath             000000018000dfac f   debugInit.obj
 0001:0000d0d0       cbEarlyVMInit              000000018000e0d0 f   debugInit.obj
 0001:0000d1f8       checkAddress               000000018000e1f8 f   debugInit.obj
 0001:0000d4c4       disposeEnvironment         000000018000e4c4 f   debugInit.obj
 0001:0000d5a4       get_boolean                000000018000e5a4 f   debugInit.obj
 0001:0000d628       get_tok                    000000018000e628 f   debugInit.obj
 0001:0000d698       initialize                 000000018000e698 f   debugInit.obj
 0001:0000dcc0       jniFatalError              000000018000ecc0 f   debugInit.obj
 0001:0000ddd8       parseOptions               000000018000edd8 f   debugInit.obj
 0001:0000e91c       printUsage                 000000018000f91c f   debugInit.obj
 0001:0000e93c       set_event_notification     000000018000f93c f   debugInit.obj
 0001:0000ea44       signalInitComplete         000000018000fa44 f   debugInit.obj
 0001:0000eaac       startTransport             000000018000faac f   debugInit.obj
 0001:0000ef0c       reader                     000000018000ff0c f   debugLoop.obj
 0001:0000fd08       vprint_message             0000000180010d08 f   error_messages.obj
 0001:0000fdd0       clearBreakpoint            0000000180010dd0 f   eventFilter.obj
 0001:0000fecc       clearWatchpoint            0000000180010ecc f   eventFilter.obj
 0001:00011190       eventInstance              0000000180012190 f   eventFilter.obj
 0001:000113d4       matchBreakpoint            00000001800123d4 f   eventFilter.obj
 0001:00011460       matchThread                0000000180012460 f   eventFilter.obj
 0001:00011494       matchWatchpoint            0000000180012494 f   eventFilter.obj
 0001:00011510       patternStringMatch         0000000180012510 f   eventFilter.obj
 0001:0001159c       setBreakpoint              000000018001259c f   eventFilter.obj
 0001:00011698       setWatchpoint              0000000180012698 f   eventFilter.obj
 0001:000117cc       cbBreakpoint               00000001800127cc f   eventHandler.obj
 0001:000119d4       cbClassLoad                00000001800129d4 f   eventHandler.obj
 0001:00011bb4       cbClassPrepare             0000000180012bb4 f   eventHandler.obj
 0001:00011d94       cbDataDump                 0000000180012d94 f   eventHandler.obj
 0001:00011dcc       cbException                0000000180012dcc f   eventHandler.obj
 0001:00012018       cbExceptionCatch           0000000180013018 f   eventHandler.obj
 0001:00012230       cbFieldAccess              0000000180013230 f   eventHandler.obj
 0001:00012468       cbFieldModification        0000000180013468 f   eventHandler.obj
 0001:0001268c       cbFramePop                 000000018001368c f   eventHandler.obj
 0001:00012894       cbGarbageCollectionFinish  0000000180013894 f   eventHandler.obj
 0001:00012910       cbMethodEntry              0000000180013910 f   eventHandler.obj
 0001:00012b0c       cbMethodExit               0000000180013b0c f   eventHandler.obj
 0001:00012d24       cbMonitorContendedEnter    0000000180013d24 f   eventHandler.obj
 0001:00012f90       cbMonitorContendedEntered  0000000180013f90 f   eventHandler.obj
 0001:000131fc       cbMonitorWait              00000001800141fc f   eventHandler.obj
 0001:0001346c       cbMonitorWaited            000000018001446c f   eventHandler.obj
 0001:000136dc       cbSingleStep               00000001800146dc f   eventHandler.obj
 0001:000138e4       cbThreadEnd                00000001800148e4 f   eventHandler.obj
 0001:00013ab0       cbThreadStart              0000000180014ab0 f   eventHandler.obj
 0001:00013c7c       cbVMDeath                  0000000180014c7c f   eventHandler.obj
 0001:00013e84       cbVMInit                   0000000180014e84 f   eventHandler.obj
 0001:0001404c       cbVThreadEnd               000000018001504c f   eventHandler.obj
 0001:00014244       cbVThreadStart             0000000180015244 f   eventHandler.obj
 0001:0001443c       createInternal             000000018001543c f   eventHandler.obj
 0001:00014504       deferEventReport           0000000180015504 f   eventHandler.obj
 0001:00015684       event_callback             0000000180016684 f   eventHandler.obj
 0001:000158b4       filterAndHandleEvent       00000001800168b4 f   eventHandler.obj
 0001:00015a48       freeHandler                0000000180016a48 f   eventHandler.obj
 0001:00015abc       getHandlerChain            0000000180016abc f   eventHandler.obj
 0001:00015c18       getObjectClass             0000000180016c18 f   eventHandler.obj
 0001:00015c84       installHandler             0000000180016c84 f   eventHandler.obj
 0001:00015d24       reportEvents               0000000180016d24 f   eventHandler.obj
 0001:00015e98       skipEventReport            0000000180016e98 f   eventHandler.obj
 0001:00015f58       commandLoop                0000000180016f58 f   eventHelper.obj
 0001:0001639c       completeCommand            000000018001739c f   eventHelper.obj
 0001:000163f8       enqueueCommand             00000001800173f8 f   eventHelper.obj
 0001:00016544       enumForCombinedSuspendPolicy 0000000180017544 f   eventHelper.obj
 0001:00016580       enumForCopyingSingles      0000000180017580 f   eventHelper.obj
 0001:000165b8       enumForVMDeath             00000001800175b8 f   eventHelper.obj
 0001:00016eb0       handleEventCommandSingle   0000000180017eb0 f   eventHelper.obj
 0001:00017228       handleReportEventCompositeCommand 0000000180018228 f   eventHelper.obj
 0001:0001749c       handleReportVMInitCommand  000000018001849c f   eventHelper.obj
 0001:00017570       saveEventInfoRefs          0000000180018570 f   eventHelper.obj
 0001:000177a8       writeClassEvent            00000001800187a8 f   eventHelper.obj
 0001:000178d4       writeFieldModificationEvent 00000001800188d4 f   eventHelper.obj
 0001:0001798c       writeMonitorEvent          000000018001898c f   eventHelper.obj
 0001:00017b20       deleteRef                  0000000180018b20 f   inStream.obj
 0001:000181fc       readBytes                  00000001800191fc f   inStream.obj
 0001:0001825c       check_methodClass          000000018001925c f   invoker.obj
 0001:000183c0       createGlobalRefs           00000001800193c0 f   invoker.obj
 0001:000186b8       fillInvokeRequest          00000001800196b8 f   invoker.obj
 0001:000187c0       invokeConstructor          00000001800197c0 f   invoker.obj
 0001:00018878       invokeNonvirtual           0000000180019878 f   invoker.obj
 0001:00018e00       invokeStatic               0000000180019e00 f   invoker.obj
 0001:000192f8       invokeVirtual              000000018001a2f8 f   invoker.obj
 0001:0001a25c       saveGlobalRefHelper        000000018001b25c f   invoker.obj
 0001:0001a5d0       dll_build_name             000000018001b5d0 f   linker_md.obj
 0001:0001a768       get_time_stamp             000000018001b768 f   log_messages.obj
 0001:0001ab40       commonInit                 000000018001bb40 f   outStream.obj
 0001:0001ac94       outStream_send             000000018001bc94 f   outStream.obj
 0001:0001b508       releaseID                  000000018001c508 f   outStream.obj
 0001:0001b52c       writeBytes                 000000018001c52c f   outStream.obj
 0001:0001b934       genericHandler             000000018001c934 f   standardHandlers.obj
 0001:0001b948       handleClassPrepare         000000018001c948 f   standardHandlers.obj
 0001:0001b99c       handleClassUnload          000000018001c99c f   standardHandlers.obj
 0001:0001b9d0       handleFrameEvent           000000018001c9d0 f   standardHandlers.obj
 0001:0001bbc4       clearStep                  000000018001cbc4 f   stepControl.obj
 0001:0001bebc       completeStep               000000018001cebc f   stepControl.obj
 0001:0001bfb0       disableStepping            000000018001cfb0 f   stepControl.obj
 0001:0001c080       enableStepping             000000018001d080 f   stepControl.obj
 0001:0001c150       getFrameCount              000000018001d150 f   stepControl.obj
 0001:0001c238       getFrameLocation           000000018001d238 f   stepControl.obj
 0001:0001c2ec       getLineNumberTable         000000018001d2ec f   stepControl.obj
 0001:0001c390       getThreadState             000000018001d390 f   stepControl.obj
 0001:0001c47c       handleExceptionCatchEvent  000000018001d47c f   stepControl.obj
 0001:0001c5d8       handleFramePopEvent        000000018001d5d8 f   stepControl.obj
 0001:0001c864       handleMethodEnterEvent     000000018001d864 f   stepControl.obj
 0001:0001ca14       initEvents                 000000018001da14 f   stepControl.obj
 0001:0001cb90       initState                  000000018001db90 f   stepControl.obj
 0001:0001d9c8       addNode                    000000018001e9c8 f   threadControl.obj
 0001:0001da18       clearThread                000000018001ea18 f   threadControl.obj
 0001:0001da84       commonResumeList           000000018001ea84 f   threadControl.obj
 0001:0001dddc       commonSuspend              000000018001eddc f   threadControl.obj
 0001:0001deb8       commonSuspendByNode        000000018001eeb8 f   threadControl.obj
 0001:0001df94       commonSuspendList          000000018001ef94 f   threadControl.obj
 0001:0001e2d4       detachHelper               000000018001f2d4 f   threadControl.obj
 0001:0001e2e8       doPendingTasks             000000018001f2e8 f   threadControl.obj
 0001:0001e3b0       dumpThreadList             000000018001f3b0 f   threadControl.obj
 0001:0001e3f4       enumerateOverThreadList    000000018001f3f4 f   threadControl.obj
 0001:0001e448       excludeCopyHelper          000000018001f448 f   threadControl.obj
 0001:0001e4a8       excludeCountHelper         000000018001f4a8 f   threadControl.obj
 0001:0001e500       findRunningThread          000000018001f500 f   threadControl.obj
 0001:0001e530       findThread                 000000018001f530 f   threadControl.obj
 0001:0001e788       incrementSuspendCountHelper 000000018001f788 f   threadControl.obj
 0001:0001e794       insertThread               000000018001f794 f   threadControl.obj
 0001:0001ea3c       newArray                   000000018001fa3c f   threadControl.obj
 0001:0001ea88       nonTlsSearch               000000018001fa88 f   threadControl.obj
 0001:0001ead4       popFrameCompleteEvent      000000018001fad4 f   threadControl.obj
 0001:0001ec08       popOneFrame                000000018001fc08 f   threadControl.obj
 0001:0001ee94       processDeferredEventModes  000000018001fe94 f   threadControl.obj
 0001:0001efe8       removeNode                 000000018001ffe8 f   threadControl.obj
 0001:0001f048       removeResumed              0000000180020048 f   threadControl.obj
 0001:0001f090       resetHelper                0000000180020090 f   threadControl.obj
 0001:0001f150       resumeCopyHelper           0000000180020150 f   threadControl.obj
 0001:0001f210       resumeCountHelper          0000000180020210 f   threadControl.obj
 0001:0001f268       resumeHelper               0000000180020268 f   threadControl.obj
 0001:0001f270       resumeThreadByNode         0000000180020270 f   threadControl.obj
 0001:0001f3a0       setPopFrameEvent           00000001800203a0 f   threadControl.obj
 0001:0001f46c       setPopFrameProceed         000000018002046c f   threadControl.obj
 0001:0001f534       setPopFrameThread          0000000180020534 f   threadControl.obj
 0001:0001f5fc       setThreadLocalStorage      00000001800205fc f   threadControl.obj
 0001:0001f6e8       suspendAllHelper           00000001800206e8 f   threadControl.obj
 0001:00020698       threadControl_removeDebugThread 0000000180021698 f   threadControl.obj
 0001:00021448       threadSetEventNotificationMode 0000000180022448 f   threadControl.obj
 0001:000214ec       threadState                00000001800224ec f   threadControl.obj
 0001:00021560       acceptThread               0000000180022560 f   transport.obj
 0001:000216c0       attachThread               00000001800226c0 f   transport.obj
 0001:0002174c       connectionInitiated        000000018002274c f   transport.obj
 0001:000217ec       freeTransportInfo          00000001800227ec f   transport.obj
 0001:00021824       launch                     0000000180022824 f   transport.obj
 0001:00021930       loadTransport              0000000180022930 f   transport.obj
 0001:00021cc4       loadTransportLibrary       0000000180022cc4 f   transport.obj
 0001:00021d80       printLastError             0000000180022d80 f   transport.obj
 0001:00022420       getCodepage                0000000180023420 f   utf_util.obj
 0001:0002248c       getWideString              000000018002348c f   utf_util.obj
 0001:00022dd8       utfError                   0000000180023dd8 f   utf_util.obj
 0001:00023520       cbObjectCounter            0000000180024520 f   util.obj
 0001:00023564       cbObjectCounterFromRef     0000000180024564 f   util.obj
 0001:000235dc       cbObjectTagInstance        00000001800245dc f   util.obj
 0001:00023614       cbObjectTagReferrer        0000000180024614 f   util.obj
 0001:00025490       getPropertyUTF8            0000000180026490 f   util.obj
 0001:000256c4       getPropertyValue           00000001800266c4 f   util.obj
 0001:00025a10       getStaticMethod            0000000180026a10 f   util.obj
 0001:00025d8c       ignore_vm_death            0000000180026d8c f   util.obj
 0001:00025eac       isArrayClass               0000000180026eac f   util.obj
 0001:00026510       is_a_nested_class          0000000180027510 f   util.obj
 0001:00026948       jvmtiVersion               0000000180027948 f   util.obj
 0001:0002973c       writeFieldValue            000000018002a73c f   util.obj
 0001:00029d48       writeStaticFieldValue      000000018002ad48 f   util.obj
 0001:0002a370       $$000000                   000000018002b370     MSVCRT:amdsecgs.obj
 0001:0002a720       ?dllmain_crt_dispatch@@YAHQEAUHINSTANCE__@@KQEAX@Z 000000018002b720 f   MSVCRT:dll_dllmain.obj
 0001:0002a770       ?dllmain_crt_process_attach@@YAHQEAUHINSTANCE__@@QEAX@Z 000000018002b770 f   MSVCRT:dll_dllmain.obj
 0001:0002a888       ?dllmain_crt_process_detach@@YAH_N@Z 000000018002b888 f   MSVCRT:dll_dllmain.obj
 0001:0002a90c       ?dllmain_dispatch@@YAHQEAUHINSTANCE__@@KQEAX@Z 000000018002b90c f   MSVCRT:dll_dllmain.obj
 0001:0002ab88       capture_previous_context   000000018002bb88 f   MSVCRT:gs_report.obj
 0001:0002b130       $$000000                   000000018002c130     MSVCRT:guard_dispatch.obj
 0001:0002b150       $$000000                   000000018002c150     MSVCRT:guard_xfg_dispatch.obj
 0001:0002b166       __scrt_is_nonwritable_in_current_image$filt$0 000000018002c166 f   MSVCRT:utility.obj
 0001:0002b17e       ?fin$0@?0??dllmain_crt_process_attach@@YAHQEAUHINSTANCE__@@QEAX@Z@4HA 000000018002c17e f   MSVCRT:dll_dllmain.obj
 0001:0002b195       ?fin$0@?0??dllmain_crt_process_detach@@YAH_N@Z@4HA 000000018002c195 f   MSVCRT:dll_dllmain.obj
 0001:0002b1ae       ?fin$1@?0??dllmain_crt_process_detach@@YAH_N@Z@4HA 000000018002c1ae f   MSVCRT:dll_dllmain.obj
 0001:0002b1c2       ?filt$0@?0??dllmain_dispatch@@YAHQEAUHINSTANCE__@@KQEAX@Z@4HA 000000018002c1c2 f   MSVCRT:dll_dllmain.obj
 0002:00007c78       GS_ExceptionPointers       0000000180034c78     MSVCRT:gs_report.obj
 0002:00008270       $unwind$length             0000000180035270     ArrayReferenceImpl.obj
 0002:00008270       $unwind$newComponents      0000000180035270     ArrayReferenceImpl.obj
 0002:00008270       $unwind$reflectedType      0000000180035270     ClassObjectReferenceImpl.obj
 0002:00008270       $unwind$superclass         0000000180035270     ClassTypeImpl.obj
 0002:00008270       $unwind$referenceType      0000000180035270     ObjectReferenceImpl.obj
 0002:00008270       $unwind$classObject        0000000180035270     ReferenceTypeImpl.obj
 0002:00008270       $unwind$getModule          0000000180035270     ReferenceTypeImpl.obj
 0002:00008270       $unwind$value              0000000180035270     StringReferenceImpl.obj
 0002:00008270       $unwind$doExit             0000000180035270     VirtualMachineImpl.obj
 0002:00008270       $unwind$commonRef_reset    0000000180035270     commonRef.obj
 0002:00008270       $unwind$eventFilterRestricted_install 0000000180035270     eventFilter.obj
 0002:00008270       $unwind$eventFilter_setInstanceOnlyFilter 0000000180035270     eventFilter.obj
 0002:00008270       $unwind$eventHandler_freeClassBreakpoints 0000000180035270     eventHandler.obj
 0002:00008270       $unwind$writeFieldModificationEvent 0000000180035270     eventHelper.obj
 0002:00008270       $unwind$writeMonitorEvent  0000000180035270     eventHelper.obj
 0002:00008270       $unwind$inStream_readObjectRef 0000000180035270     inStream.obj
 0002:00008270       $unwind$inStream_readString 0000000180035270     inStream.obj
 0002:00008270       $unwind$check_methodClass  0000000180035270     invoker.obj
 0002:00008270       $unwind$fillInvokeRequest  0000000180035270     invoker.obj
 0002:00008270       $unwind$saveGlobalRefHelper 0000000180035270     invoker.obj
 0002:00008270       $unwind$outStream_initCommand 0000000180035270     outStream.obj
 0002:00008270       $unwind$enumerateOverThreadList 0000000180035270     threadControl.obj
 0002:00008270       $unwind$threadControl_saveCLEInfo 0000000180035270     threadControl.obj
 0002:00008270       $unwind$threadControl_stop 0000000180035270     threadControl.obj
 0002:00008270       $unwind$threadSetEventNotificationMode 0000000180035270     threadControl.obj
 0002:00008270       $unwind$__scrt_dllmain_exception_filter 0000000180035270     MSVCRT:utility.obj
 0002:00008284       $unwind$writeBooleanComponents 0000000180035284     ArrayReferenceImpl.obj
 0002:00008284       $unwind$writeByteComponents 0000000180035284     ArrayReferenceImpl.obj
 0002:00008284       $unwind$writeCharComponents 0000000180035284     ArrayReferenceImpl.obj
 0002:00008284       $unwind$writeDoubleComponents 0000000180035284     ArrayReferenceImpl.obj
 0002:00008284       $unwind$writeFloatComponents 0000000180035284     ArrayReferenceImpl.obj
 0002:00008284       $unwind$writeIntComponents 0000000180035284     ArrayReferenceImpl.obj
 0002:00008284       $unwind$writeLongComponents 0000000180035284     ArrayReferenceImpl.obj
 0002:00008284       $unwind$writeShortComponents 0000000180035284     ArrayReferenceImpl.obj
 0002:00008284       $unwind$event_callback     0000000180035284     eventHandler.obj
 0002:00008284       $unwind$spawnNewThread     0000000180035284     util.obj
 0002:000082a0       $unwind$writeObjectComponents 00000001800352a0     ArrayReferenceImpl.obj
 0002:000082a0       $unwind$specificTypeKey    00000001800352a0     util.obj
 0002:000082b8       $unwind$writeComponents    00000001800352b8     ArrayReferenceImpl.obj
 0002:000082b8       $unwind$decode             00000001800352b8     SDE.obj
 0002:000082b8       $unwind$createInternal     00000001800352b8     eventHandler.obj
 0002:000082b8       $unwind$getWideString      00000001800352b8     utf_util.obj
 0002:000082d0       $unwind$getValues          00000001800352d0     ArrayReferenceImpl.obj
 0002:000082d0       $unwind$setValues          00000001800352d0     ArrayReferenceImpl.obj
 0002:000082d0       $unwind$getValues          00000001800352d0     StackFrameImpl.obj
 0002:000082d0       $unwind$setValues          00000001800352d0     StackFrameImpl.obj
 0002:000082ec       $unwind$readBooleanComponents 00000001800352ec     ArrayReferenceImpl.obj
 0002:000082ec       $unwind$readByteComponents 00000001800352ec     ArrayReferenceImpl.obj
 0002:000082ec       $unwind$readCharComponents 00000001800352ec     ArrayReferenceImpl.obj
 0002:000082ec       $unwind$readDoubleComponents 00000001800352ec     ArrayReferenceImpl.obj
 0002:000082ec       $unwind$readFloatComponents 00000001800352ec     ArrayReferenceImpl.obj
 0002:000082ec       $unwind$readIntComponents  00000001800352ec     ArrayReferenceImpl.obj
 0002:000082ec       $unwind$readLongComponents 00000001800352ec     ArrayReferenceImpl.obj
 0002:000082ec       $unwind$readShortComponents 00000001800352ec     ArrayReferenceImpl.obj
 0002:00008304       $unwind$readObjectComponents 0000000180035304     ArrayReferenceImpl.obj
 0002:00008320       $unwind$readComponents     0000000180035320     ArrayReferenceImpl.obj
 0002:00008320       $unwind$getClassLoader     0000000180035320     ModuleReferenceImpl.obj
 0002:00008320       $unwind$deleteNodeByID     0000000180035320     commonRef.obj
 0002:00008320       $unwind$eventHandlerRestricted_iterator 0000000180035320     eventHandler.obj
 0002:00008320       $unwind$eventHelper_reportInvokeDone 0000000180035320     eventHelper.obj
 0002:00008320       $unwind$eventHelper_suspendThread 0000000180035320     eventHelper.obj
 0002:00008338       $unwind$writeNewObjectArray 0000000180035338     ArrayTypeImpl.obj
 0002:00008350       $unwind$writeNewPrimitiveArray 0000000180035350     ArrayTypeImpl.obj
 0002:00008350       $unwind$disposeObjects     0000000180035350     VirtualMachineImpl.obj
 0002:00008350       $unwind$writeBytes         0000000180035350     outStream.obj
 0002:00008350       $unwind$suspendAllHelper   0000000180035350     threadControl.obj
 0002:00008350       $unwind$threadControl_removeDebugThread 0000000180035350     threadControl.obj
 0002:00008350       $unwind$filterDebugThreads 0000000180035350     util.obj
 0002:0000836c       $unwind$newInstance        000000018003536c     ArrayTypeImpl.obj
 0002:00008384       $unwind$visibleClasses     0000000180035384     ClassLoaderReferenceImpl.obj
 0002:00008384       $unwind$ownedMonitors      0000000180035384     ThreadReferenceImpl.obj
 0002:00008384       $unwind$ownedMonitorsWithStackDepth 0000000180035384     ThreadReferenceImpl.obj
 0002:00008398       $unwind$readStaticFieldValue 0000000180035398     ClassTypeImpl.obj
 0002:000083b8       $unwind$setValues          00000001800353b8     ClassTypeImpl.obj
 0002:000083b8       $unwind$doVariableTable    00000001800353b8     MethodImpl.obj
 0002:000083d0       $unwind$readAndSetFilters  00000001800353d0     EventRequestImpl.obj
 0002:000083d0       $unwind$eventFilter_setStepFilter 00000001800353d0     eventFilter.obj
 0002:000083ec       $unwind$setCommand         00000001800353ec     EventRequestImpl.obj
 0002:000083ec       $unwind$commonRef_pinAll   00000001800353ec     commonRef.obj
 0002:000083ec       $unwind$eventFilter_setExceptionOnlyFilter 00000001800353ec     eventFilter.obj
 0002:000083ec       $unwind$eventFilter_setFieldOnlyFilter 00000001800353ec     eventFilter.obj
 0002:000083ec       $unwind$eventFilter_setLocationOnlyFilter 00000001800353ec     eventFilter.obj
 0002:000083ec       $unwind$matchBreakpoint    00000001800353ec     eventFilter.obj
 0002:000083ec       $unwind$threadControl_popFrames 00000001800353ec     threadControl.obj
 0002:000083ec       $unwind$threadControl_setEventMode 00000001800353ec     threadControl.obj
 0002:00008404       $unwind$clearCommand       0000000180035404     EventRequestImpl.obj
 0002:00008404       $unwind$isCollected        0000000180035404     ObjectReferenceImpl.obj
 0002:00008404       $unwind$popFrames          0000000180035404     StackFrameImpl.obj
 0002:00008404       $unwind$stop               0000000180035404     ThreadReferenceImpl.obj
 0002:00008404       $unwind$createString       0000000180035404     VirtualMachineImpl.obj
 0002:00008404       $unwind$bagAdd             0000000180035404     bag.obj
 0002:00008404       $unwind$bagEnumerateOver   0000000180035404     bag.obj
 0002:00008404       $unwind$commonRef_compact  0000000180035404     commonRef.obj
 0002:00008404       $unwind$weakenNode         0000000180035404     commonRef.obj
 0002:00008404       $unwind$matchWatchpoint    0000000180035404     eventFilter.obj
 0002:00008404       $unwind$outStream_send     0000000180035404     outStream.obj
 0002:00008404       $unwind$outStream_writeString 0000000180035404     outStream.obj
 0002:00008404       $unwind$threadControl_cmpCLEInfo 0000000180035404     threadControl.obj
 0002:00008404       $unwind$threadControl_isDebugThread 0000000180035404     threadControl.obj
 0002:00008404       $unwind$launch             0000000180035404     transport.obj
 0002:00008404       $unwind$utf8sToUtf8m       0000000180035404     utf_util.obj
 0002:00008404       $unwind$writeCodeLocation  0000000180035404     util.obj
 0002:0000841c       $unwind$clearAllBreakpoints 000000018003541c     EventRequestImpl.obj
 0002:0000841c       $unwind$createFrameID      000000018003541c     FrameID.obj
 0002:0000841c       $unwind$validateFrameID    000000018003541c     FrameID.obj
 0002:0000841c       $unwind$readLine           000000018003541c     SDE.obj
 0002:0000841c       $unwind$readNumber         000000018003541c     SDE.obj
 0002:0000841c       $unwind$validateSuspendedThread 000000018003541c     ThreadReferenceImpl.obj
 0002:0000841c       $unwind$resume             000000018003541c     VirtualMachineImpl.obj
 0002:0000841c       $unwind$suspend            000000018003541c     VirtualMachineImpl.obj
 0002:0000841c       $unwind$cbTrackingObjectFree 000000018003541c     classTrack.obj
 0002:0000841c       $unwind$initializeObjectsByID 000000018003541c     commonRef.obj
 0002:0000841c       $unwind$checkAddress       000000018003541c     debugInit.obj
 0002:0000841c       $unwind$disposeEnvironment 000000018003541c     debugInit.obj
 0002:0000841c       $unwind$forceExit          000000018003541c     debugInit.obj
 0002:0000841c       $unwind$eventHandler_allocHandlerID 000000018003541c     eventHandler.obj
 0002:0000841c       $unwind$eventHandler_free  000000018003541c     eventHandler.obj
 0002:0000841c       $unwind$eventHandler_installExternal 000000018003541c     eventHandler.obj
 0002:0000841c       $unwind$completeCommand    000000018003541c     eventHelper.obj
 0002:0000841c       $unwind$eventHelper_reset  000000018003541c     eventHelper.obj
 0002:0000841c       $unwind$inStream_destroy   000000018003541c     inStream.obj
 0002:0000841c       $unwind$inStream_readBoolean 000000018003541c     inStream.obj
 0002:0000841c       $unwind$inStream_readBytes 000000018003541c     inStream.obj
 0002:0000841c       $unwind$inStream_readModuleRef 000000018003541c     inStream.obj
 0002:0000841c       $unwind$invoker_detach     000000018003541c     invoker.obj
 0002:0000841c       $unwind$commonInit         000000018003541c     outStream.obj
 0002:0000841c       $unwind$outStream_sendCommand 000000018003541c     outStream.obj
 0002:0000841c       $unwind$outStream_sendReply 000000018003541c     outStream.obj
 0002:0000841c       $unwind$outStream_writeObjectTag 000000018003541c     outStream.obj
 0002:0000841c       $unwind$releaseID          000000018003541c     outStream.obj
 0002:0000841c       $unwind$methodSignature_returnTag 000000018003541c     signature.obj
 0002:0000841c       $unwind$stepControl_endStep 000000018003541c     stepControl.obj
 0002:0000841c       $unwind$dumpThreadList     000000018003541c     threadControl.obj
 0002:0000841c       $unwind$findRunningThread  000000018003541c     threadControl.obj
 0002:0000841c       $unwind$resetHelper        000000018003541c     threadControl.obj
 0002:0000841c       $unwind$resumeCountHelper  000000018003541c     threadControl.obj
 0002:0000841c       $unwind$threadControl_allVThreads 000000018003541c     threadControl.obj
 0002:0000841c       $unwind$threadControl_currentThread 000000018003541c     threadControl.obj
 0002:0000841c       $unwind$threadControl_detachInvokes 000000018003541c     threadControl.obj
 0002:0000841c       $unwind$threadControl_interrupt 000000018003541c     threadControl.obj
 0002:0000841c       $unwind$threadControl_setPendingInterrupt 000000018003541c     threadControl.obj
 0002:0000841c       $unwind$attachThread       000000018003541c     transport.obj
 0002:0000841c       $unwind$getClassname       000000018003541c     util.obj
 0002:0000841c       $unwind$jvmtiGetCapabilities 000000018003541c     util.obj
 0002:0000841c       $unwind$__raise_securityfailure 000000018003541c     MSVCRT:gs_report.obj
 0002:0000841c       $unwind$__scrt_initialize_crt 000000018003541c     MSVCRT:utility.obj
 0002:0000841c       $unwind$__scrt_initialize_onexit_tables 000000018003541c     MSVCRT:utility.obj
 0002:0000841c       $unwind$__scrt_release_startup_lock 000000018003541c     MSVCRT:utility.obj
 0002:0000841c       $unwind$__scrt_uninitialize_crt 000000018003541c     MSVCRT:utility.obj
 0002:0000841c       $unwind$_onexit            000000018003541c     MSVCRT:utility.obj
 0002:00008424       $unwind$lineTable          0000000180035424     MethodImpl.obj
 0002:00008438       $unwind$bytecodes          0000000180035438     MethodImpl.obj
 0002:00008438       $unwind$signatureWithGeneric 0000000180035438     ReferenceTypeImpl.obj
 0002:00008448       $unwind$isObsolete         0000000180035448     MethodImpl.obj
 0002:00008448       $unwind$disableCollection  0000000180035448     ObjectReferenceImpl.obj
 0002:00008448       $unwind$enableCollection   0000000180035448     ObjectReferenceImpl.obj
 0002:00008448       $unwind$getClassStatus     0000000180035448     ReferenceTypeImpl.obj
 0002:00008448       $unwind$getClassVersion    0000000180035448     ReferenceTypeImpl.obj
 0002:00008448       $unwind$modifiers          0000000180035448     ReferenceTypeImpl.obj
 0002:00008448       $unwind$sourceDebugExtension 0000000180035448     ReferenceTypeImpl.obj
 0002:00008448       $unwind$sourceFile         0000000180035448     ReferenceTypeImpl.obj
 0002:00008448       $unwind$stratumTableIndex  0000000180035448     SDE.obj
 0002:00008448       $unwind$getFrameCount      0000000180035448     ThreadReferenceImpl.obj
 0002:00008448       $unwind$interrupt          0000000180035448     ThreadReferenceImpl.obj
 0002:00008448       $unwind$resume             0000000180035448     ThreadReferenceImpl.obj
 0002:00008448       $unwind$status             0000000180035448     ThreadReferenceImpl.obj
 0002:00008448       $unwind$suspend            0000000180035448     ThreadReferenceImpl.obj
 0002:00008448       $unwind$suspendCount       0000000180035448     ThreadReferenceImpl.obj
 0002:00008448       $unwind$bagCreateBag       0000000180035448     bag.obj
 0002:00008448       $unwind$commonRef_pin      0000000180035448     commonRef.obj
 0002:00008448       $unwind$commonRef_releaseMultiple 0000000180035448     commonRef.obj
 0002:00008448       $unwind$deleteNode         0000000180035448     commonRef.obj
 0002:00008448       $unwind$newCommonRef       0000000180035448     commonRef.obj
 0002:00008448       $unwind$debugInit_exit     0000000180035448     debugInit.obj
 0002:00008448       $unwind$set_event_notification 0000000180035448     debugInit.obj
 0002:00008448       $unwind$clearWatchpoint    0000000180035448     eventFilter.obj
 0002:00008448       $unwind$eventFilterRestricted_alloc 0000000180035448     eventFilter.obj
 0002:00008448       $unwind$eventFilter_setClassOnlyFilter 0000000180035448     eventFilter.obj
 0002:00008448       $unwind$eventFilter_setThreadOnlyFilter 0000000180035448     eventFilter.obj
 0002:00008448       $unwind$patternStringMatch 0000000180035448     eventFilter.obj
 0002:00008448       $unwind$setWatchpoint      0000000180035448     eventFilter.obj
 0002:00008448       $unwind$installHandler     0000000180035448     eventHandler.obj
 0002:00008448       $unwind$readBytes          0000000180035448     inStream.obj
 0002:00008448       $unwind$dbgsysLoadLibrary  0000000180035448     linker_md.obj
 0002:00008448       $unwind$outStream_destroy  0000000180035448     outStream.obj
 0002:00008448       $unwind$outStream_writeByteArray 0000000180035448     outStream.obj
 0002:00008448       $unwind$handleClassPrepare 0000000180035448     standardHandlers.obj
 0002:00008448       $unwind$getLineNumberTable 0000000180035448     stepControl.obj
 0002:00008448       $unwind$newArray           0000000180035448     threadControl.obj
 0002:00008448       $unwind$nonTlsSearch       0000000180035448     threadControl.obj
 0002:00008448       $unwind$threadControl_addDebugThread 0000000180035448     threadControl.obj
 0002:00008448       $unwind$threadControl_resumeThread 0000000180035448     threadControl.obj
 0002:00008448       $unwind$threadControl_suspendThread 0000000180035448     threadControl.obj
 0002:00008448       $unwind$allClassLoaderClasses 0000000180035448     util.obj
 0002:00008448       $unwind$allInterfaces      0000000180035448     util.obj
 0002:00008448       $unwind$fieldModifiers     0000000180035448     util.obj
 0002:00008448       $unwind$isFieldSynthetic   0000000180035448     util.obj
 0002:00008448       $unwind$methodLocation     0000000180035448     util.obj
 0002:00008448       $unwind$_DllMainCRTStartup 0000000180035448     MSVCRT:dll_dllmain.obj
 0002:00008458       $unwind$getName            0000000180035458     ModuleReferenceImpl.obj
 0002:00008474       $unwind$getValues          0000000180035474     ObjectReferenceImpl.obj
 0002:00008474       $unwind$getValues          0000000180035474     ReferenceTypeImpl.obj
 0002:00008474       $unwind$ignoreLine         0000000180035474     SDE.obj
 0002:00008474       $unwind$sdePeek            0000000180035474     SDE.obj
 0002:00008474       $unwind$sdeRead            0000000180035474     SDE.obj
 0002:00008474       $unwind$holdEvents         0000000180035474     VirtualMachineImpl.obj
 0002:00008474       $unwind$releaseEvents      0000000180035474     VirtualMachineImpl.obj
 0002:00008474       $unwind$is_wrong_phase     0000000180035474     classTrack.obj
 0002:00008474       $unwind$commonRef_initialize 0000000180035474     commonRef.obj
 0002:00008474       $unwind$Agent_OnUnload     0000000180035474     debugInit.obj
 0002:00008474       $unwind$debugInit_waitInitComplete 0000000180035474     debugInit.obj
 0002:00008474       $unwind$printUsage         0000000180035474     debugInit.obj
 0002:00008474       $unwind$signalInitComplete 0000000180035474     debugInit.obj
 0002:00008474       $unwind$debugLoop_initialize 0000000180035474     debugLoop.obj
 0002:00008474       $unwind$debugLoop_sync     0000000180035474     debugLoop.obj
 0002:00008474       $unwind$cbDataDump         0000000180035474     eventHandler.obj
 0002:00008474       $unwind$cbGarbageCollectionFinish 0000000180035474     eventHandler.obj
 0002:00008474       $unwind$eventHandler_waitForActiveCallbacks 0000000180035474     eventHandler.obj
 0002:00008474       $unwind$commandLoop_sync   0000000180035474     eventHelper.obj
 0002:00008474       $unwind$enumForCopyingSingles 0000000180035474     eventHelper.obj
 0002:00008474       $unwind$eventHelper_holdEvents 0000000180035474     eventHelper.obj
 0002:00008474       $unwind$eventHelper_initialize 0000000180035474     eventHelper.obj
 0002:00008474       $unwind$eventHelper_lock   0000000180035474     eventHelper.obj
 0002:00008474       $unwind$eventHelper_releaseEvents 0000000180035474     eventHelper.obj
 0002:00008474       $unwind$eventHelper_unlock 0000000180035474     eventHelper.obj
 0002:00008474       $unwind$unblockCommandLoop 0000000180035474     eventHelper.obj
 0002:00008474       $unwind$deleteRef          0000000180035474     inStream.obj
 0002:00008474       $unwind$inStream_readByte  0000000180035474     inStream.obj
 0002:00008474       $unwind$inStream_readChar  0000000180035474     inStream.obj
 0002:00008474       $unwind$inStream_readDouble 0000000180035474     inStream.obj
 0002:00008474       $unwind$inStream_readFloat 0000000180035474     inStream.obj
 0002:00008474       $unwind$inStream_readInt   0000000180035474     inStream.obj
 0002:00008474       $unwind$inStream_readLong  0000000180035474     inStream.obj
 0002:00008474       $unwind$inStream_readShort 0000000180035474     inStream.obj
 0002:00008474       $unwind$invoker_initialize 0000000180035474     invoker.obj
 0002:00008474       $unwind$finish_logging     0000000180035474     log_messages.obj
 0002:00008474       $unwind$outStream_writeBoolean 0000000180035474     outStream.obj
 0002:00008474       $unwind$outStream_writeChar 0000000180035474     outStream.obj
 0002:00008474       $unwind$outStream_writeInt 0000000180035474     outStream.obj
 0002:00008474       $unwind$outStream_writeLong 0000000180035474     outStream.obj
 0002:00008474       $unwind$outStream_writeShort 0000000180035474     outStream.obj
 0002:00008474       $unwind$handleClassUnload  0000000180035474     standardHandlers.obj
 0002:00008474       $unwind$stepControl_initialize 0000000180035474     stepControl.obj
 0002:00008474       $unwind$detachHelper       0000000180035474     threadControl.obj
 0002:00008474       $unwind$threadControl_dumpAllThreads 0000000180035474     threadControl.obj
 0002:00008474       $unwind$threadControl_initialize 0000000180035474     threadControl.obj
 0002:00008474       $unwind$transport_close    0000000180035474     transport.obj
 0002:00008474       $unwind$transport_initialize 0000000180035474     transport.obj
 0002:00008474       $unwind$transport_is_open  0000000180035474     transport.obj
 0002:00008474       $unwind$transport_reset    0000000180035474     transport.obj
 0002:00008474       $unwind$transport_waitForConnection 0000000180035474     transport.obj
 0002:00008474       $unwind$eventIndex2EventName 0000000180035474     util.obj
 0002:00008474       $unwind$eventIndexInit     0000000180035474     util.obj
 0002:00008474       $unwind$ignore_vm_death    0000000180035474     util.obj
 0002:00008474       $unwind$jvmtiMajorVersion  0000000180035474     util.obj
 0002:00008474       $unwind$jvmtiMicroVersion  0000000180035474     util.obj
 0002:00008474       $unwind$jvmtiMinorVersion  0000000180035474     util.obj
 0002:00008474       $unwind$__scrt_initialize_default_local_stdio_options 0000000180035474     MSVCRT:default_local_stdio_options.obj
 0002:00008474       $unwind$?dllmain_crt_dispatch@@YAHQEAUHINSTANCE__@@KQEAX@Z 0000000180035474     MSVCRT:dll_dllmain.obj
 0002:00008474       $unwind$DllMain            0000000180035474     MSVCRT:dll_dllmain_stub.obj
 0002:00008474       $unwind$__GSHandlerCheck   0000000180035474     MSVCRT:gshandler.obj
 0002:00008474       $unwind$__scrt_acquire_startup_lock 0000000180035474     MSVCRT:utility.obj
 0002:00008474       $unwind$__scrt_dllmain_after_initialize_c 0000000180035474     MSVCRT:utility.obj
 0002:00008474       $unwind$__scrt_dllmain_before_initialize_c 0000000180035474     MSVCRT:utility.obj
 0002:00008474       $unwind$__scrt_dllmain_crt_thread_attach 0000000180035474     MSVCRT:utility.obj
 0002:00008474       $unwind$__scrt_dllmain_crt_thread_detach 0000000180035474     MSVCRT:utility.obj
 0002:00008474       $unwind$__scrt_dllmain_uninitialize_c 0000000180035474     MSVCRT:utility.obj
 0002:00008474       $unwind$__scrt_dllmain_uninitialize_critical 0000000180035474     MSVCRT:utility.obj
 0002:00008474       $unwind$atexit             0000000180035474     MSVCRT:utility.obj
 0002:0000847c       $unwind$readFieldValue     000000018003547c     ObjectReferenceImpl.obj
 0002:0000849c       $unwind$setValues          000000018003549c     ObjectReferenceImpl.obj
 0002:000084b4       $unwind$monitorInfo        00000001800354b4     ObjectReferenceImpl.obj
 0002:000084cc       $unwind$referringObjects   00000001800354cc     ObjectReferenceImpl.obj
 0002:000084cc       $unwind$fields1            00000001800354cc     ReferenceTypeImpl.obj
 0002:000084cc       $unwind$instances          00000001800354cc     ReferenceTypeImpl.obj
 0002:000084cc       $unwind$methods1           00000001800354cc     ReferenceTypeImpl.obj
 0002:000084cc       $unwind$skipEventReport    00000001800354cc     eventHandler.obj
 0002:000084e4       $unwind$getClassLoader     00000001800354e4     ReferenceTypeImpl.obj
 0002:000084e4       $unwind$signature          00000001800354e4     ReferenceTypeImpl.obj
 0002:000084e4       $unwind$currentContendedMonitor 00000001800354e4     ThreadReferenceImpl.obj
 0002:000084f8       $unwind$writeMethodInfo    00000001800354f8     ReferenceTypeImpl.obj
 0002:0000850c       $unwind$getConstantPool    000000018003550c     ReferenceTypeImpl.obj
 0002:0000851c       $unwind$writeFieldInfo     000000018003551c     ReferenceTypeImpl.obj
 0002:00008534       $unwind$interfaces         0000000180035534     ReferenceTypeImpl.obj
 0002:00008534       $unwind$nestedTypes        0000000180035534     ReferenceTypeImpl.obj
 0002:00008534       $unwind$commonSuspend      0000000180035534     threadControl.obj
 0002:00008548       $unwind$snprintf           0000000180035548     SDE.obj
 0002:00008558       $unwind$convertLineNumberTable 0000000180035558     SDE.obj
 0002:00008558       $unwind$searchAllSourceNames 0000000180035558     SDE.obj
 0002:00008558       $unwind$classPaths         0000000180035558     VirtualMachineImpl.obj
 0002:00008558       $unwind$eventFilterRestricted_deinstall 0000000180035558     eventFilter.obj
 0002:00008558       $unwind$eventFilter_predictFiltering 0000000180035558     eventFilter.obj
 0002:00008558       $unwind$utf8mToUtf8s       0000000180035558     utf_util.obj
 0002:00008558       $unwind$sharedGetFieldValues 0000000180035558     util.obj
 0002:00008574       $unwind$loadDebugInfo      0000000180035574     SDE.obj
 0002:00008584       $unwind$syntax             0000000180035584     SDE.obj
 0002:00008594       $unwind$storeFile          0000000180035594     SDE.obj
 0002:00008594       $unwind$strengthenNode     0000000180035594     commonRef.obj
 0002:00008594       $unwind$eventHelper_recordEvent 0000000180035594     eventHelper.obj
 0002:00008594       $unwind$eventHelper_reportVMInit 0000000180035594     eventHelper.obj
 0002:000085b0       $unwind$storeLine          00000001800355b0     SDE.obj
 0002:000085b0       $unwind$eventHelper_recordFrameEvent 00000001800355b0     eventHelper.obj
 0002:000085b0       $unwind$getMethod          00000001800355b0     util.obj
 0002:000085b0       $unwind$getStaticMethod    00000001800355b0     util.obj
 0002:000085b0       $unwind$saveGlobalRef      00000001800355b0     util.obj
 0002:000085cc       $unwind$storeStratum       00000001800355cc     SDE.obj
 0002:000085cc       $unwind$eventHelper_recordClassUnload 00000001800355cc     eventHelper.obj
 0002:000085cc       $unwind$handleEventCommandSingle 00000001800355cc     eventHelper.obj
 0002:000085cc       $unwind$dbgsysBuildLibName 00000001800355cc     linker_md.obj
 0002:000085cc       $unwind$acceptThread       00000001800355cc     transport.obj
 0002:000085e4       $unwind$lineSection        00000001800355e4     SDE.obj
 0002:000085e4       $unwind$startTransport     00000001800355e4     debugInit.obj
 0002:000085e4       $unwind$log_message_begin  00000001800355e4     log_messages.obj
 0002:000085e4       $unwind$getFrameLocation   00000001800355e4     stepControl.obj
 0002:000085f8       $unwind$validateThreadFrame 00000001800355f8     StackFrameImpl.obj
 0002:000085f8       $unwind$idSizes            00000001800355f8     VirtualMachineImpl.obj
 0002:000085f8       $unwind$setDefaultStratum  00000001800355f8     VirtualMachineImpl.obj
 0002:000085f8       $unwind$bagDup             00000001800355f8     bag.obj
 0002:000085f8       $unwind$cbTrackingClassPrepare 00000001800355f8     classTrack.obj
 0002:000085f8       $unwind$commonRef_release  00000001800355f8     commonRef.obj
 0002:000085f8       $unwind$commonRef_unpin    00000001800355f8     commonRef.obj
 0002:000085f8       $unwind$debugInit_reset    00000001800355f8     debugInit.obj
 0002:000085f8       $unwind$do_pause           00000001800355f8     error_messages.obj
 0002:000085f8       $unwind$clearBreakpoint    00000001800355f8     eventFilter.obj
 0002:000085f8       $unwind$setBreakpoint      00000001800355f8     eventFilter.obj
 0002:000085f8       $unwind$eventHandler_alloc 00000001800355f8     eventHandler.obj
 0002:000085f8       $unwind$eventHandler_dumpAllHandlers 00000001800355f8     eventHandler.obj
 0002:000085f8       $unwind$eventHandler_freeAll 00000001800355f8     eventHandler.obj
 0002:000085f8       $unwind$eventHandler_freeByID 00000001800355f8     eventHandler.obj
 0002:000085f8       $unwind$freeHandler        00000001800355f8     eventHandler.obj
 0002:000085f8       $unwind$getObjectClass     00000001800355f8     eventHandler.obj
 0002:000085f8       $unwind$inStream_init      00000001800355f8     inStream.obj
 0002:000085f8       $unwind$inStream_readArrayRef 00000001800355f8     inStream.obj
 0002:000085f8       $unwind$inStream_readClassLoaderRef 00000001800355f8     inStream.obj
 0002:000085f8       $unwind$inStream_readClassRef 00000001800355f8     inStream.obj
 0002:000085f8       $unwind$inStream_readStringRef 00000001800355f8     inStream.obj
 0002:000085f8       $unwind$inStream_readThreadGroupRef 00000001800355f8     inStream.obj
 0002:000085f8       $unwind$inStream_readThreadRef 00000001800355f8     inStream.obj
 0002:000085f8       $unwind$invokeConstructor  00000001800355f8     invoker.obj
 0002:000085f8       $unwind$outStream_initReply 00000001800355f8     outStream.obj
 0002:000085f8       $unwind$outStream_setError 00000001800355f8     outStream.obj
 0002:000085f8       $unwind$methodSignature_init 00000001800355f8     signature.obj
 0002:000085f8       $unwind$stepControl_clearRequest 00000001800355f8     stepControl.obj
 0002:000085f8       $unwind$clearThread        00000001800355f8     threadControl.obj
 0002:000085f8       $unwind$commonSuspendByNode 00000001800355f8     threadControl.obj
 0002:000085f8       $unwind$doPendingTasks     00000001800355f8     threadControl.obj
 0002:000085f8       $unwind$excludeCopyHelper  00000001800355f8     threadControl.obj
 0002:000085f8       $unwind$excludeCountHelper 00000001800355f8     threadControl.obj
 0002:000085f8       $unwind$removeResumed      00000001800355f8     threadControl.obj
 0002:000085f8       $unwind$resumeCopyHelper   00000001800355f8     threadControl.obj
 0002:000085f8       $unwind$resumeThreadByNode 00000001800355f8     threadControl.obj
 0002:000085f8       $unwind$threadControl_clearCLEInfo 00000001800355f8     threadControl.obj
 0002:000085f8       $unwind$threadControl_getFrameGeneration 00000001800355f8     threadControl.obj
 0002:000085f8       $unwind$threadControl_getInstructionStepMode 00000001800355f8     threadControl.obj
 0002:000085f8       $unwind$threadControl_getInvokeRequest 00000001800355f8     threadControl.obj
 0002:000085f8       $unwind$threadControl_getStepRequest 00000001800355f8     threadControl.obj
 0002:000085f8       $unwind$threadState        00000001800355f8     threadControl.obj
 0002:000085f8       $unwind$connectionInitiated 00000001800355f8     transport.obj
 0002:000085f8       $unwind$transport_receivePacket 00000001800355f8     transport.obj
 0002:000085f8       $unwind$transport_sendPacket 00000001800355f8     transport.obj
 0002:000085f8       $unwind$allLoadedClasses   00000001800355f8     util.obj
 0002:000085f8       $unwind$classLoader        00000001800355f8     util.obj
 0002:000085f8       $unwind$getSourceDebugExtension 00000001800355f8     util.obj
 0002:000085f8       $unwind$isArray            00000001800355f8     util.obj
 0002:000085f8       $unwind$isClass            00000001800355f8     util.obj
 0002:000085f8       $unwind$isClassLoader      00000001800355f8     util.obj
 0002:000085f8       $unwind$isMethodSynthetic  00000001800355f8     util.obj
 0002:000085f8       $unwind$isString           00000001800355f8     util.obj
 0002:000085f8       $unwind$isThread           00000001800355f8     util.obj
 0002:000085f8       $unwind$isThreadGroup      00000001800355f8     util.obj
 0002:000085f8       $unwind$isVThread          00000001800355f8     util.obj
 0002:000085f8       $unwind$methodClass        00000001800355f8     util.obj
 0002:000085f8       $unwind$methodModifiers    00000001800355f8     util.obj
 0002:000085f8       $unwind$_RTC_Initialize    00000001800355f8     MSVCRT:initsect.obj
 0002:000085f8       $unwind$_RTC_Terminate     00000001800355f8     MSVCRT:initsect.obj
 0002:00008604       $unwind$writeVariableValue 0000000180035604     StackFrameImpl.obj
 0002:0000861c       $unwind$readVariableValue  000000018003561c     StackFrameImpl.obj
 0002:00008634       $unwind$thisObject         0000000180035634     StackFrameImpl.obj
 0002:00008648       $unwind$name               0000000180035648     ThreadGroupReferenceImpl.obj
 0002:00008648       $unwind$parent             0000000180035648     ThreadGroupReferenceImpl.obj
 0002:00008648       $unwind$name               0000000180035648     ThreadReferenceImpl.obj
 0002:00008648       $unwind$threadGroup        0000000180035648     ThreadReferenceImpl.obj
 0002:00008648       $unwind$dbgsysGetLastErrorString 0000000180035648     linker_md.obj
 0002:0000865c       $unwind$children           000000018003565c     ThreadGroupReferenceImpl.obj
 0002:00008670       $unwind$frames             0000000180035670     ThreadReferenceImpl.obj
 0002:00008688       $unwind$forceEarlyReturn   0000000180035688     ThreadReferenceImpl.obj
 0002:000086a4       $unwind$isVirtual          00000001800356a4     ThreadReferenceImpl.obj
 0002:000086a4       $unwind$methodSignature_nextArgumentExists 00000001800356a4     signature.obj
 0002:000086a4       $unwind$is_a_nested_class  00000001800356a4     util.obj
 0002:000086b8       $unwind$version            00000001800356b8     VirtualMachineImpl.obj
 0002:000086dc       $unwind$classesForSignature 00000001800356dc     VirtualMachineImpl.obj
 0002:000086f4       $unwind$allModules         00000001800356f4     VirtualMachineImpl.obj
 0002:000086f4       $unwind$topLevelThreadGroups 00000001800356f4     VirtualMachineImpl.obj
 0002:00008704       $unwind$allClasses1        0000000180035704     VirtualMachineImpl.obj
 0002:0000871c       $unwind$instanceCounts     000000018003571c     VirtualMachineImpl.obj
 0002:0000871c       $unwind$eventHandler_synthesizeUnloadEvent 000000018003571c     eventHandler.obj
 0002:00008738       $unwind$redefineClasses    0000000180035738     VirtualMachineImpl.obj
 0002:00008750       $unwind$getAllThreads      0000000180035750     VirtualMachineImpl.obj
 0002:00008768       $unwind$capabilities       0000000180035768     VirtualMachineImpl.obj
 0002:00008778       $unwind$capabilitiesNew    0000000180035778     VirtualMachineImpl.obj
 0002:0000878c       $unwind$bagDestroyBag      000000018003578c     bag.obj
 0002:0000878c       $unwind$freeTransportInfo  000000018003578c     transport.obj
 0002:00008794       $unwind$classTrack_initialize 0000000180035794     classTrack.obj
 0002:000087a8       $unwind$addPreparedClass   00000001800357a8     classTrack.obj
 0002:000087a8       $unwind$getPropertyUTF8    00000001800357a8     util.obj
 0002:000087bc       $unwind$setupEvents        00000001800357bc     classTrack.obj
 0002:000087cc       $unwind$commonRef_idToRef  00000001800357cc     commonRef.obj
 0002:000087cc       $unwind$commonRef_refToID  00000001800357cc     commonRef.obj
 0002:000087dc       $unwind$commonRef_idToRef_delete 00000001800357dc     commonRef.obj
 0002:000087e4       $unwind$commonRef_unpinAll 00000001800357e4     commonRef.obj
 0002:000087e4       $unwind$eventFilterRestricted_passesUnloadFilter 00000001800357e4     eventFilter.obj
 0002:000087e4       $unwind$handleFramePopEvent 00000001800357e4     stepControl.obj
 0002:000087e4       $unwind$findClass          00000001800357e4     util.obj
 0002:000087fc       $unwind$createNode         00000001800357fc     commonRef.obj
 0002:00008814       $unwind$debugDispatch_initialize 0000000180035814     debugDispatch.obj
 0002:00008814       $unwind$cbEarlyVMDeath     0000000180035814     debugInit.obj
 0002:00008814       $unwind$standardHandlers_onConnect 0000000180035814     standardHandlers.obj
 0002:00008814       $unwind$setPopFrameEvent   0000000180035814     threadControl.obj
 0002:00008814       $unwind$setPopFrameProceed 0000000180035814     threadControl.obj
 0002:00008814       $unwind$setPopFrameThread  0000000180035814     threadControl.obj
 0002:00008820       $unwind$Agent_OnLoad       0000000180035820     debugInit.obj
 0002:0000883c       $unwind$cbEarlyVMInit      000000018003583c     debugInit.obj
 0002:0000884c       $unwind$cbEarlyException   000000018003584c     debugInit.obj
 0002:0000886c       $unwind$initialize         000000018003586c     debugInit.obj
 0002:0000886c       $unwind$invoker_requestInvoke 000000018003586c     invoker.obj
 0002:0000886c       $unwind$threadControl_onEventHandlerExit 000000018003586c     threadControl.obj
 0002:0000886c       $unwind$writeStaticFieldValue 000000018003586c     util.obj
 0002:00008888       $unwind$parseOptions       0000000180035888     debugInit.obj
 0002:000088ac       $unwind$jniFatalError      00000001800358ac     debugInit.obj
 0002:000088c4       $unwind$get_tok            00000001800358c4     debugInit.obj
 0002:000088d0       $unwind$get_boolean        00000001800358d0     debugInit.obj
 0002:000088e0       $unwind$debugLoop_run      00000001800358e0     debugLoop.obj
 0002:00008908       $unwind$reader             0000000180035908     debugLoop.obj
 0002:0000891c       $unwind$fprintf            000000018003591c     error_messages.obj
 0002:00008928       $unwind$print_message      0000000180035928     error_messages.obj
 0002:00008928       $unwind$__report_gsfailure 0000000180035928     MSVCRT:gs_report.obj
 0002:00008930       $unwind$error_message      0000000180035930     error_messages.obj
 0002:0000893c       $unwind$tty_message        000000018003593c     error_messages.obj
 0002:00008944       $unwind$jdiAssertionFailed 0000000180035944     error_messages.obj
 0002:00008944       $unwind$saveEventInfoRefs  0000000180035944     eventHelper.obj
 0002:00008944       $unwind$completeStep       0000000180035944     stepControl.obj
 0002:00008944       $unwind$stepControl_resetRequest 0000000180035944     stepControl.obj
 0002:00008958       $unwind$vprint_message     0000000180035958     error_messages.obj
 0002:00008974       $unwind$isBreakpointSet    0000000180035974     eventFilter.obj
 0002:0000897c       $unwind$eventFilter_dumpHandlerFilters 000000018003597c     eventFilter.obj
 0002:00008988       $unwind$eventFilterRestricted_passesFilter 0000000180035988     eventFilter.obj
 0002:000089a0       $unwind$eventInstance      00000001800359a0     eventFilter.obj
 0002:000089ac       $unwind$eventHandler_createInternalThreadOnly 00000001800359ac     eventHandler.obj
 0002:000089ac       $unwind$eventHandler_createPermanentInternal 00000001800359ac     eventHandler.obj
 0002:000089b4       $unwind$eventHandler_initialize 00000001800359b4     eventHandler.obj
 0002:000089d0       $unwind$eventHandler_onConnect 00000001800359d0     eventHandler.obj
 0002:000089e4       $unwind$eventHandler_reset 00000001800359e4     eventHandler.obj
 0002:000089e4       $unwind$invoker_doInvoke   00000001800359e4     invoker.obj
 0002:000089e4       $unwind$threadControl_reset 00000001800359e4     threadControl.obj
 0002:000089fc       $unwind$getMethodClass     00000001800359fc     eventHandler.obj
 0002:000089fc       $unwind$getFrameCount      00000001800359fc     stepControl.obj
 0002:000089fc       $unwind$getThreadState     00000001800359fc     stepControl.obj
 0002:000089fc       $unwind$classStatus        00000001800359fc     util.obj
 0002:000089fc       $unwind$debugMonitorCreate 00000001800359fc     util.obj
 0002:000089fc       $unwind$isArrayClass       00000001800359fc     util.obj
 0002:000089fc       $unwind$isMethodNative     00000001800359fc     util.obj
 0002:000089fc       $unwind$jvmtiAllocate      00000001800359fc     util.obj
 0002:00008a0c       $unwind$eventHandler_dumpHandlers 0000000180035a0c     eventHandler.obj
 0002:00008a0c       $unwind$utfError           0000000180035a0c     utf_util.obj
 0002:00008a1c       $unwind$getHandlerChain    0000000180035a1c     eventHandler.obj
 0002:00008a1c       $unwind$invokeNonvirtual   0000000180035a1c     invoker.obj
 0002:00008a1c       $unwind$invokeStatic       0000000180035a1c     invoker.obj
 0002:00008a1c       $unwind$invokeVirtual      0000000180035a1c     invoker.obj
 0002:00008a1c       $unwind$invoker_enableInvokeRequests 0000000180035a1c     invoker.obj
 0002:00008a1c       $unwind$invoker_isEnabled  0000000180035a1c     invoker.obj
 0002:00008a1c       $unwind$disableStepping    0000000180035a1c     stepControl.obj
 0002:00008a1c       $unwind$enableStepping     0000000180035a1c     stepControl.obj
 0002:00008a1c       $unwind$setThreadLocalStorage 0000000180035a1c     threadControl.obj
 0002:00008a1c       $unwind$debugMonitorEnter  0000000180035a1c     util.obj
 0002:00008a1c       $unwind$debugMonitorExit   0000000180035a1c     util.obj
 0002:00008a1c       $unwind$debugMonitorNotify 0000000180035a1c     util.obj
 0002:00008a1c       $unwind$debugMonitorNotifyAll 0000000180035a1c     util.obj
 0002:00008a1c       $unwind$debugMonitorWait   0000000180035a1c     util.obj
 0002:00008a1c       $unwind$eventIndex2jdwp    0000000180035a1c     util.obj
 0002:00008a1c       $unwind$eventIndex2jvmti   0000000180035a1c     util.obj
 0002:00008a1c       $unwind$jvmtiVersion       0000000180035a1c     util.obj
 0002:00008a1c       $unwind$threadGroupInfo    0000000180035a1c     util.obj
 0002:00008a2c       $unwind$deferEventReport   0000000180035a2c     eventHandler.obj
 0002:00008a44       $unwind$reportEvents       0000000180035a44     eventHandler.obj
 0002:00008a5c       $unwind$filterAndHandleEvent 0000000180035a5c     eventHandler.obj
 0002:00008a78       $unwind$cbBreakpoint       0000000180035a78     eventHandler.obj
 0002:00008a78       $unwind$cbException        0000000180035a78     eventHandler.obj
 0002:00008a78       $unwind$cbExceptionCatch   0000000180035a78     eventHandler.obj
 0002:00008a78       $unwind$cbFieldAccess      0000000180035a78     eventHandler.obj
 0002:00008a78       $unwind$cbFramePop         0000000180035a78     eventHandler.obj
 0002:00008a78       $unwind$cbMethodEntry      0000000180035a78     eventHandler.obj
 0002:00008a78       $unwind$cbMethodExit       0000000180035a78     eventHandler.obj
 0002:00008a78       $unwind$cbSingleStep       0000000180035a78     eventHandler.obj
 0002:00008a94       $unwind$cbThreadEnd        0000000180035a94     eventHandler.obj
 0002:00008a94       $unwind$cbThreadStart      0000000180035a94     eventHandler.obj
 0002:00008a94       $unwind$cbVMInit           0000000180035a94     eventHandler.obj
 0002:00008a94       $unwind$cbVThreadEnd       0000000180035a94     eventHandler.obj
 0002:00008a94       $unwind$cbVThreadStart     0000000180035a94     eventHandler.obj
 0002:00008aa8       $unwind$cbClassLoad        0000000180035aa8     eventHandler.obj
 0002:00008aa8       $unwind$cbClassPrepare     0000000180035aa8     eventHandler.obj
 0002:00008ac0       $unwind$cbFieldModification 0000000180035ac0     eventHandler.obj
 0002:00008adc       $unwind$cbMonitorContendedEnter 0000000180035adc     eventHandler.obj
 0002:00008adc       $unwind$cbMonitorContendedEntered 0000000180035adc     eventHandler.obj
 0002:00008af8       $unwind$cbMonitorWait      0000000180035af8     eventHandler.obj
 0002:00008af8       $unwind$cbMonitorWaited    0000000180035af8     eventHandler.obj
 0002:00008b14       $unwind$cbVMDeath          0000000180035b14     eventHandler.obj
 0002:00008b30       $unwind$enqueueCommand     0000000180035b30     eventHelper.obj
 0002:00008b48       $unwind$writeClassEvent    0000000180035b48     eventHelper.obj
 0002:00008b60       $unwind$handleReportEventCompositeCommand 0000000180035b60     eventHelper.obj
 0002:00008b84       $unwind$handleReportVMInitCommand 0000000180035b84     eventHelper.obj
 0002:00008b9c       $unwind$commandLoop        0000000180035b9c     eventHelper.obj
 0002:00008b9c       $unwind$clearStep          0000000180035b9c     stepControl.obj
 0002:00008b9c       $unwind$stepControl_beginStep 0000000180035b9c     stepControl.obj
 0002:00008b9c       $unwind$tossGlobalRef      0000000180035b9c     util.obj
 0002:00008bb8       $unwind$commandLoop_exitVmDeathLockOnError 0000000180035bb8     eventHelper.obj
 0002:00008bc0       $unwind$eventHelper_reportEvents 0000000180035bc0     eventHelper.obj
 0002:00008bc0       $unwind$initState          0000000180035bc0     stepControl.obj
 0002:00008bd4       $unwind$dbgsysExec         0000000180035bd4     exec_md.obj
 0002:00008be0       $unwind$inStream_readValue 0000000180035be0     inStream.obj
 0002:00008bf0       $unwind$invoker_completeInvokeRequest 0000000180035bf0     invoker.obj
 0002:00008c18       $unwind$createGlobalRefs   0000000180035c18     invoker.obj
 0002:00008c30       $unwind$dll_build_name     0000000180035c30     linker_md.obj
 0002:00008c48       $unwind$setup_logging      0000000180035c48     log_messages.obj
 0002:00008c54       $unwind$log_message_end    0000000180035c54     log_messages.obj
 0002:00008c68       $unwind$get_time_stamp     0000000180035c68     log_messages.obj
 0002:00008c84       $unwind$outStream_writeByte 0000000180035c84     outStream.obj
 0002:00008c8c       $unwind$outStream_writeDouble 0000000180035c8c     outStream.obj
 0002:00008c8c       $unwind$outStream_writeFloat 0000000180035c8c     outStream.obj
 0002:00008c94       $unwind$outStream_writeObjectRef 0000000180035c94     outStream.obj
 0002:00008cac       $unwind$outStream_writeValue 0000000180035cac     outStream.obj
 0002:00008cc0       $unwind$componentTypeSignature 0000000180035cc0     signature.obj
 0002:00008ccc       $unwind$handleFrameEvent   0000000180035ccc     standardHandlers.obj
 0002:00008cdc       $unwind$stepControl_handleStep 0000000180035cdc     stepControl.obj
 0002:00008cf4       $unwind$handleExceptionCatchEvent 0000000180035cf4     stepControl.obj
 0002:00008cf4       $unwind$popOneFrame        0000000180035cf4     threadControl.obj
 0002:00008cf4       $unwind$createLocalRefSpace 0000000180035cf4     util.obj
 0002:00008d0c       $unwind$handleMethodEnterEvent 0000000180035d0c     stepControl.obj
 0002:00008d24       $unwind$initEvents         0000000180035d24     stepControl.obj
 0002:00008d3c       $unwind$threadControl_onHook 0000000180035d3c     threadControl.obj
 0002:00008d50       $unwind$threadControl_onEventHandlerEntry 0000000180035d50     threadControl.obj
 0002:00008d6c       $unwind$threadControl_suspendCount 0000000180035d6c     threadControl.obj
 0002:00008d6c       $unwind$methodReturnType   0000000180035d6c     util.obj
 0002:00008d80       $unwind$threadControl_suspendAll 0000000180035d80     threadControl.obj
 0002:00008d94       $unwind$threadControl_resumeAll 0000000180035d94     threadControl.obj
 0002:00008da8       $unwind$threadControl_applicationThreadStatus 0000000180035da8     threadControl.obj
 0002:00008dbc       $unwind$findThread         0000000180035dbc     threadControl.obj
 0002:00008dd4       $unwind$insertThread       0000000180035dd4     threadControl.obj
 0002:00008dec       $unwind$processDeferredEventModes 0000000180035dec     threadControl.obj
 0002:00008e08       $unwind$commonResumeList   0000000180035e08     threadControl.obj
 0002:00008e20       $unwind$commonSuspendList  0000000180035e20     threadControl.obj
 0002:00008e38       $unwind$popFrameCompleteEvent 0000000180035e38     threadControl.obj
 0002:00008e4c       $unwind$transport_startTransport 0000000180035e4c     transport.obj
 0002:00008e70       $unwind$printLastError     0000000180035e70     transport.obj
 0002:00008e84       $unwind$loadTransportLibrary 0000000180035e84     transport.obj
 0002:00008e9c       $unwind$loadTransport      0000000180035e9c     transport.obj
 0002:00008eb0       $unwind$utf8sToUtf8mLength 0000000180035eb0     utf_util.obj
 0002:00008eb8       $unwind$utf8mToUtf8sLength 0000000180035eb8     utf_util.obj
 0002:00008ecc       $unwind$utf8FromPlatform   0000000180035ecc     utf_util.obj
 0002:00008ecc       $unwind$utf8ToPlatform     0000000180035ecc     utf_util.obj
 0002:00008ee0       $unwind$getCodepage        0000000180035ee0     utf_util.obj
 0002:00008ef0       $unwind$util_initialize    0000000180035ef0     util.obj
 0002:00008f08       $unwind$referenceTypeTag   0000000180035f08     util.obj
 0002:00008f1c       $unwind$classInstances     0000000180035f1c     util.obj
 0002:00008f38       $unwind$classInstanceCounts 0000000180035f38     util.obj
 0002:00008f58       $unwind$objectReferrers    0000000180035f58     util.obj
 0002:00008f78       $unwind$sharedInvoke       0000000180035f78     util.obj
 0002:00008f90       $unwind$fieldSignature     0000000180035f90     util.obj
 0002:00008fa4       $unwind$methodSignature    0000000180035fa4     util.obj
 0002:00008fb8       $unwind$getEnv             0000000180035fb8     util.obj
 0002:00008fc4       $unwind$allThreads         0000000180035fc4     util.obj
 0002:00008fd4       $unwind$classSignature     0000000180035fd4     util.obj
 0002:00008fe8       $unwind$isMethodObsolete   0000000180035fe8     util.obj
 0002:00008ff4       $unwind$allNestedClasses   0000000180035ff4     util.obj
 0002:0000900c       $unwind$setAgentPropertyValue 000000018003600c     util.obj
 0002:00009028       $unwind$jvmtiDeallocate    0000000180036028     util.obj
 0002:00009038       $unwind$log_debugee_location 0000000180036038     util.obj
 0002:00009054       $unwind$getSpecialJvmti    0000000180036054     util.obj
 0002:00009064       $unwind$writeFieldValue    0000000180036064     util.obj
 0002:00009080       $unwind$getPropertyValue   0000000180036080     util.obj
 0002:00009098       $unwind$__GSHandlerCheckCommon 0000000180036098     MSVCRT:gshandler.obj
 0002:000090a0       $xdatasym                  00000001800360a0     MSVCRT:amdsecgs.obj
 0002:000090a4       $unwind$__scrt_is_nonwritable_in_current_image 00000001800360a4     MSVCRT:utility.obj
 0002:000090c4       $unwind$__scrt_is_nonwritable_in_current_image$filt$0 00000001800360c4     MSVCRT:utility.obj
 0002:000090cc       $unwind$?dllmain_crt_process_attach@@YAHQEAUHINSTANCE__@@QEAX@Z 00000001800360cc     MSVCRT:dll_dllmain.obj
 0002:00009108       $unwind$?fin$0@?0??dllmain_crt_process_attach@@YAHQEAUHINSTANCE__@@QEAX@Z@4HA 0000000180036108     MSVCRT:dll_dllmain.obj
 0002:00009108       $unwind$?fin$0@?0??dllmain_crt_process_detach@@YAH_N@Z@4HA 0000000180036108     MSVCRT:dll_dllmain.obj
 0002:00009108       $unwind$?fin$1@?0??dllmain_crt_process_detach@@YAH_N@Z@4HA 0000000180036108     MSVCRT:dll_dllmain.obj
 0002:00009110       $unwind$?dllmain_crt_process_detach@@YAH_N@Z 0000000180036110     MSVCRT:dll_dllmain.obj
 0002:00009164       $unwind$?dllmain_dispatch@@YAHQEAUHINSTANCE__@@KQEAX@Z 0000000180036164     MSVCRT:dll_dllmain.obj
 0002:0000918c       $unwind$?filt$0@?0??dllmain_dispatch@@YAHQEAUHINSTANCE__@@KQEAX@Z@4HA 000000018003618c     MSVCRT:dll_dllmain.obj
 0002:00009194       $unwind$capture_previous_context 0000000180036194     MSVCRT:gs_report.obj
 0002:000091a0       $unwind$__isa_available_init 00000001800361a0     MSVCRT:cpu_disp.obj
 0002:000091b0       $unwind$__scrt_fastfail    00000001800361b0     MSVCRT:utility_desktop.obj
 0002:000091c0       $unwind$__security_init_cookie 00000001800361c0     MSVCRT:gs_support.obj
 0002:000091d0       $xdatasym                  00000001800361d0     MSVCRT:guard_dispatch.obj
 0002:000091d8       $xdatasym                  00000001800361d8     MSVCRT:guard_xfg_dispatch.obj
 0002:000091e0       .edata                     00000001800361e0     jdwp.exp
 0002:00009208       rgpv                       0000000180036208     jdwp.exp
 0002:00009210       rgszName                   0000000180036210     jdwp.exp
 0002:00009218       rgwOrd                     0000000180036218     jdwp.exp
 0002:0000921c       szName                     000000018003621c     jdwp.exp
 0002:00009225       $N00001                    0000000180036225     jdwp.exp
 0002:00009232       $N00002                    0000000180036232     jdwp.exp
 0002:00009602       .idata$6                   0000000180036602     jvm:jvm.dll
 0002:0000982c       .idata$6                   000000018003682c     kernel32:KERNEL32.dll
 0002:000098ba       .idata$6                   00000001800368ba     vcruntime:VCRUNTIME140.dll
 0002:00009af0       .idata$6                   0000000180036af0     ucrt:api-ms-win-crt-stdio-l1-1-0.dll
 0002:00009b10       .idata$6                   0000000180036b10     ucrt:api-ms-win-crt-string-l1-1-0.dll
 0002:00009b32       .idata$6                   0000000180036b32     ucrt:api-ms-win-crt-runtime-l1-1-0.dll
 0002:00009b54       .idata$6                   0000000180036b54     ucrt:api-ms-win-crt-convert-l1-1-0.dll
 0002:00009b76       .idata$6                   0000000180036b76     ucrt:api-ms-win-crt-environment-l1-1-0.dll
 0002:00009b9c       .idata$6                   0000000180036b9c     ucrt:api-ms-win-crt-filesystem-l1-1-0.dll
 0002:00009bc2       .idata$6                   0000000180036bc2     ucrt:api-ms-win-crt-time-l1-1-0.dll
 0002:00009be2       .idata$6                   0000000180036be2     ucrt:api-ms-win-crt-heap-l1-1-0.dll
 0003:00000668       versionName                0000000180037668     VirtualMachineImpl.obj
 0003:000007d0       initOnStartup              00000001800377d0     debugInit.obj
 0003:000007d1       suspendOnInit              00000001800377d1     debugInit.obj
 0003:000007d4       p                          00000001800377d4     error_messages.obj
 0003:000007d8       maxQueueSize               00000001800377d8     eventHelper.obj
 0003:000007e0       transportVersion           00000001800377e0     transport.obj
 0003:000007e8       callback                   00000001800377e8     transport.obj
 0003:000007f8       ?intCodePage@?1??getCodepage@@9@9 00000001800377f8     utf_util.obj
 0003:00000840       ?method@?1??getName@@9@9   0000000180037840     ModuleReferenceImpl.obj
 0003:00000848       ?method@?1??getClassLoader@@9@9 0000000180037848     ModuleReferenceImpl.obj
 0003:00000850       globalDefaultStratumId     0000000180037850     SDE.obj
 0003:00000858       defaultStratumId           0000000180037858     SDE.obj
 0003:00000860       cachedClass                0000000180037860     SDE.obj
 0003:00000868       fileTable                  0000000180037868     SDE.obj
 0003:00000870       lineTable                  0000000180037870     SDE.obj
 0003:00000878       stratumTable               0000000180037878     SDE.obj
 0003:00000880       fileTableSize              0000000180037880     SDE.obj
 0003:00000884       lineTableSize              0000000180037884     SDE.obj
 0003:00000888       stratumTableSize           0000000180037888     SDE.obj
 0003:0000088c       fileIndex                  000000018003788c     SDE.obj
 0003:00000890       lineIndex                  0000000180037890     SDE.obj
 0003:00000894       stratumIndex               0000000180037894     SDE.obj
 0003:00000898       currentFileId              0000000180037898     SDE.obj
 0003:0000089c       defaultStratumIndex        000000018003789c     SDE.obj
 0003:000008a0       baseStratumIndex           00000001800378a0     SDE.obj
 0003:000008a4       sourceMapIsValid           00000001800378a4     SDE.obj
 0003:000008a8       sdePos                     00000001800378a8     SDE.obj
 0003:000008b0       jplsFilename               00000001800378b0     SDE.obj
 0003:000008b8       NullString                 00000001800378b8     SDE.obj
 0003:000008c0       sourceDebugExtension       00000001800378c0     SDE.obj
 0003:000008d0       jmp_buf_env                00000001800378d0     SDE.obj
 0003:000009d0       trackingEnv                00000001800379d0     classTrack.obj
 0003:000009d8       cmdSetsArray               00000001800379d8     debugDispatch.obj
 0003:000009e0       vmInitialized              00000001800379e0     debugInit.obj
 0003:000009e1       initComplete               00000001800379e1     debugInit.obj
 0003:000009e2       currentSessionID           00000001800379e2     debugInit.obj
 0003:000009e3       isServer                   00000001800379e3     debugInit.obj
 0003:000009e4       isStrict                   00000001800379e4     debugInit.obj
 0003:000009e5       useStandardAlloc           00000001800379e5     debugInit.obj
 0003:000009e6       initOnUncaught             00000001800379e6     debugInit.obj
 0003:000009e7       dopause                    00000001800379e7     debugInit.obj
 0003:000009e8       initMonitor                00000001800379e8     debugInit.obj
 0003:000009f0       transports                 00000001800379f0     debugInit.obj
 0003:000009f8       initOnException            00000001800379f8     debugInit.obj
 0003:00000a00       launchOnInit               0000000180037a00     debugInit.obj
 0003:00000a08       docoredump                 0000000180037a08     debugInit.obj
 0003:00000a10       logfile                    0000000180037a10     debugInit.obj
 0003:00000a18       logflags                   0000000180037a18     debugInit.obj
 0003:00000a20       names                      0000000180037a20     debugInit.obj
 0003:00000a30       ?s@?1??get_gdata@@9@9      0000000180037a30     debugInit.obj
 0003:00000c78       cmdQueue                   0000000180037c78     debugLoop.obj
 0003:00000c80       cmdQueueLock               0000000180037c80     debugLoop.obj
 0003:00000c88       vmDeathLock                0000000180037c88     debugLoop.obj
 0003:00000c90       transportError             0000000180037c90     debugLoop.obj
 0003:00000c91       ?got_version@?1??eventInstance@@9@9 0000000180037c91     eventFilter.obj
 0003:00000c92       ?is_version_gte_12x@?1??eventInstance@@9@9 0000000180037c92     eventFilter.obj
 0003:00000ca0       requestIdCounter           0000000180037ca0     eventHandler.obj
 0003:00000ca4       currentSessionID           0000000180037ca4     eventHandler.obj
 0003:00000ca5       vm_death_callback_active   0000000180037ca5     eventHandler.obj
 0003:00000ca8       active_callbacks           0000000180037ca8     eventHandler.obj
 0003:00000cac       garbageCollected           0000000180037cac     eventHandler.obj
 0003:00000cb0       callbackLock               0000000180037cb0     eventHandler.obj
 0003:00000cb8       callbackBlock              0000000180037cb8     eventHandler.obj
 0003:00000cc0       handlerLock                0000000180037cc0     eventHandler.obj
 0003:00000cd0       __handlers                 0000000180037cd0     eventHandler.obj
 0003:00000d80       commandQueue               0000000180037d80     eventHelper.obj
 0003:00000d90       commandQueueLock           0000000180037d90     eventHelper.obj
 0003:00000d98       commandCompleteLock        0000000180037d98     eventHelper.obj
 0003:00000da0       blockCommandLoopLock       0000000180037da0     eventHelper.obj
 0003:00000da8       vmDeathLock                0000000180037da8     eventHelper.obj
 0003:00000db0       commandLoopEnteredVmDeathLock 0000000180037db0     eventHelper.obj
 0003:00000db1       holdEvents                 0000000180037db1     eventHelper.obj
 0003:00000db2       ?vmDeathReported@?1??enqueueCommand@@9@9 0000000180037db2     eventHelper.obj
 0003:00000db3       blockCommandLoop           0000000180037db3     eventHelper.obj
 0003:00000db4       currentQueueSize           0000000180037db4     eventHelper.obj
 0003:00000db8       currentSessionID           0000000180037db8     eventHelper.obj
 0003:00000dc0       invokerLock                0000000180037dc0     invoker.obj
 0003:00000dd0       logging                    0000000180037dd0     log_messages.obj
 0003:00000dd4       processPid                 0000000180037dd4     log_messages.obj
 0003:00000dd8       log_file                   0000000180037dd8     log_messages.obj
 0003:00000de0       logging_filename           0000000180037de0     log_messages.obj
 0003:00000ef0       location_stamp             0000000180037ef0     log_messages.obj
 0003:00001018       open_count                 0000000180038018     log_messages.obj
 0003:00001020       stepLock                   0000000180038020     stepControl.obj
 0003:00001030       suspendAllCount            0000000180038030     threadControl.obj
 0003:00001034       numRunningVThreads         0000000180038034     threadControl.obj
 0003:00001038       popFrameEventLock          0000000180038038     threadControl.obj
 0003:00001040       popFrameProceedLock        0000000180038040     threadControl.obj
 0003:00001048       threadLock                 0000000180038048     threadControl.obj
 0003:00001050       runningThreads             0000000180038050     threadControl.obj
 0003:00001058       otherThreads               0000000180038058     threadControl.obj
 0003:00001060       runningVThreads            0000000180038060     threadControl.obj
 0003:00001068       debugThreadCount           0000000180038068     threadControl.obj
 0003:00001070       debugThreads               0000000180038070     threadControl.obj
 0003:000010c0       deferredEventModes         00000001800380c0     threadControl.obj
 0003:000010d0       transport                  00000001800380d0     transport.obj
 0003:000010d8       listenerLock               00000001800380d8     transport.obj
 0003:000010e0       sendLock                   00000001800380e0     transport.obj
 0003:000010f8       ?currentID@?1??uniqueID@@9@9 00000001800380f8     util.obj
 0003:00001100       index2jvmti                0000000180038100     util.obj
 0003:00001158       index2jdwp                 0000000180038158     util.obj
 0003:00001180       ?is_initialized_as_dll@@3_NA 0000000180038180     MSVCRT:utility.obj
 0003:00001181       ?module_local_atexit_table_initialized@@3_NA 0000000180038181     MSVCRT:utility.obj
 0003:00001188       ?module_local_atexit_table@@3U_onexit_table_t@@A 0000000180038188     MSVCRT:utility.obj
 0003:000011a0       ?module_local_at_quick_exit_table@@3U_onexit_table_t@@A 00000001800381a0     MSVCRT:utility.obj
 0003:000011b8       ?__proc_attached@@3HA      00000001800381b8     MSVCRT:dll_dllmain.obj
 0003:000011c0       GS_ExceptionRecord         00000001800381c0     MSVCRT:gs_report.obj
 0003:00001260       GS_ContextRecord           0000000180038260     MSVCRT:gs_report.obj
 0005:00000060       $R000000                   000000018003b060     jdwp.dll.res
